Component: ARM Compiler 5.06 update 4 (build 422) Tool: armlink [4d35d2]

==============================================================================

Section Cross References

    system_stm32f4xx.o(i.SystemCoreClockUpdate) refers to system_stm32f4xx.o(.data) for .data
    tcp_in.o(i.tcp_input) refers to pbuf.o(i.pbuf_header) for pbuf_header
    tcp_in.o(i.tcp_input) refers to ip_addr.o(i.ip4_addr_isbroadcast) for ip4_addr_isbroadcast
    tcp_in.o(i.tcp_input) refers to def.o(i.lwip_ntohs) for lwip_ntohs
    tcp_in.o(i.tcp_input) refers to def.o(i.lwip_ntohl) for lwip_ntohl
    tcp_in.o(i.tcp_input) refers to tcp.o(i.tcp_process_refused_data) for tcp_process_refused_data
    tcp_in.o(i.tcp_input) refers to tcp_in.o(i.tcp_timewait_input) for tcp_timewait_input
    tcp_in.o(i.tcp_input) refers to tcp_in.o(i.tcp_listen_input) for tcp_listen_input
    tcp_in.o(i.tcp_input) refers to tcp_in.o(i.tcp_process) for tcp_process
    tcp_in.o(i.tcp_input) refers to tcp.o(i.tcp_pcb_remove) for tcp_pcb_remove
    tcp_in.o(i.tcp_input) refers to memp.o(i.memp_free) for memp_free
    tcp_in.o(i.tcp_input) refers to pbuf.o(i.pbuf_free) for pbuf_free
    tcp_in.o(i.tcp_input) refers to tcp.o(i.tcp_abort) for tcp_abort
    tcp_in.o(i.tcp_input) refers to tcp.o(i.tcp_recv_null) for tcp_recv_null
    tcp_in.o(i.tcp_input) refers to tcp_out.o(i.tcp_output) for tcp_output
    tcp_in.o(i.tcp_input) refers to tcp_out.o(i.tcp_rst) for tcp_rst
    tcp_in.o(i.tcp_input) refers to tcp_in.o(.data) for .data
    tcp_in.o(i.tcp_input) refers to ip.o(.data) for current_iphdr_dest
    tcp_in.o(i.tcp_input) refers to tcp.o(.data) for tcp_active_pcbs
    tcp_in.o(i.tcp_input) refers to tcp_in.o(.bss) for .bss
    tcp_in.o(i.tcp_listen_input) refers to tcp_out.o(i.tcp_rst) for tcp_rst
    tcp_in.o(i.tcp_listen_input) refers to tcp.o(i.tcp_alloc) for tcp_alloc
    tcp_in.o(i.tcp_listen_input) refers to lwip_timers.o(i.tcp_timer_needed) for tcp_timer_needed
    tcp_in.o(i.tcp_listen_input) refers to tcp_in.o(i.tcp_parseopt) for tcp_parseopt
    tcp_in.o(i.tcp_listen_input) refers to tcp.o(i.tcp_eff_send_mss) for tcp_eff_send_mss
    tcp_in.o(i.tcp_listen_input) refers to tcp_out.o(i.tcp_enqueue_flags) for tcp_enqueue_flags
    tcp_in.o(i.tcp_listen_input) refers to tcp.o(i.tcp_abandon) for tcp_abandon
    tcp_in.o(i.tcp_listen_input) refers to tcp_out.o(i.tcp_output) for tcp_output
    tcp_in.o(i.tcp_listen_input) refers to tcp_in.o(.data) for .data
    tcp_in.o(i.tcp_listen_input) refers to ip.o(.data) for current_iphdr_src
    tcp_in.o(i.tcp_listen_input) refers to tcp.o(.data) for tcp_active_pcbs
    tcp_in.o(i.tcp_parseopt) refers to def.o(i.lwip_ntohs) for lwip_ntohs
    tcp_in.o(i.tcp_parseopt) refers to tcp_in.o(.data) for .data
    tcp_in.o(i.tcp_process) refers to tcp_in.o(i.tcp_parseopt) for tcp_parseopt
    tcp_in.o(i.tcp_process) refers to def.o(i.lwip_ntohl) for lwip_ntohl
    tcp_in.o(i.tcp_process) refers to tcp.o(i.tcp_eff_send_mss) for tcp_eff_send_mss
    tcp_in.o(i.tcp_process) refers to tcp.o(i.tcp_seg_free) for tcp_seg_free
    tcp_in.o(i.tcp_process) refers to tcp.o(i.tcp_abort) for tcp_abort
    tcp_in.o(i.tcp_process) refers to tcp_in.o(i.tcp_receive) for tcp_receive
    tcp_in.o(i.tcp_process) refers to tcp_out.o(i.tcp_rst) for tcp_rst
    tcp_in.o(i.tcp_process) refers to tcp_out.o(i.tcp_rexmit) for tcp_rexmit
    tcp_in.o(i.tcp_process) refers to tcp.o(i.tcp_pcb_purge) for tcp_pcb_purge
    tcp_in.o(i.tcp_process) refers to lwip_timers.o(i.tcp_timer_needed) for tcp_timer_needed
    tcp_in.o(i.tcp_process) refers to tcp_in.o(.data) for .data
    tcp_in.o(i.tcp_process) refers to tcp.o(.data) for tcp_ticks
    tcp_in.o(i.tcp_process) refers to ip.o(.data) for current_iphdr_src
    tcp_in.o(i.tcp_receive) refers to tcp_out.o(i.tcp_rexmit_fast) for tcp_rexmit_fast
    tcp_in.o(i.tcp_receive) refers to pbuf.o(i.pbuf_clen) for pbuf_clen
    tcp_in.o(i.tcp_receive) refers to def.o(i.lwip_ntohs) for lwip_ntohs
    tcp_in.o(i.tcp_receive) refers to tcp.o(i.tcp_seg_free) for tcp_seg_free
    tcp_in.o(i.tcp_receive) refers to def.o(i.lwip_ntohl) for lwip_ntohl
    tcp_in.o(i.tcp_receive) refers to pbuf.o(i.pbuf_header) for pbuf_header
    tcp_in.o(i.tcp_receive) refers to def.o(i.lwip_htons) for lwip_htons
    tcp_in.o(i.tcp_receive) refers to pbuf.o(i.pbuf_realloc) for pbuf_realloc
    tcp_in.o(i.tcp_receive) refers to tcp.o(i.tcp_update_rcv_ann_wnd) for tcp_update_rcv_ann_wnd
    tcp_in.o(i.tcp_receive) refers to tcp_out.o(i.tcp_send_empty_ack) for tcp_send_empty_ack
    tcp_in.o(i.tcp_receive) refers to tcp_in.o(.data) for .data
    tcp_in.o(i.tcp_receive) refers to tcp.o(.data) for tcp_ticks
    tcp_in.o(i.tcp_receive) refers to tcp_in.o(.bss) for .bss
    tcp_in.o(i.tcp_timewait_input) refers to tcp_out.o(i.tcp_rst) for tcp_rst
    tcp_in.o(i.tcp_timewait_input) refers to tcp_out.o(i.tcp_output) for tcp_output
    tcp_in.o(i.tcp_timewait_input) refers to tcp_in.o(.data) for .data
    tcp_in.o(i.tcp_timewait_input) refers to ip.o(.data) for current_iphdr_src
    tcp_in.o(i.tcp_timewait_input) refers to tcp.o(.data) for tcp_ticks
    lwip_timers.o(i.arp_timer) refers to etharp.o(i.etharp_tmr) for etharp_tmr
    lwip_timers.o(i.arp_timer) refers to lwip_timers.o(i.sys_timeout) for sys_timeout
    lwip_timers.o(i.dhcp_timer_coarse) refers to dhcp.o(i.dhcp_coarse_tmr) for dhcp_coarse_tmr
    lwip_timers.o(i.dhcp_timer_coarse) refers to lwip_timers.o(i.sys_timeout) for sys_timeout
    lwip_timers.o(i.dhcp_timer_fine) refers to dhcp.o(i.dhcp_fine_tmr) for dhcp_fine_tmr
    lwip_timers.o(i.dhcp_timer_fine) refers to lwip_timers.o(i.sys_timeout) for sys_timeout
    lwip_timers.o(i.ip_reass_timer) refers to ip_frag.o(i.ip_reass_tmr) for ip_reass_tmr
    lwip_timers.o(i.ip_reass_timer) refers to lwip_timers.o(i.sys_timeout) for sys_timeout
    lwip_timers.o(i.sys_check_timeouts) refers to ethernetif.o(i.sys_now) for sys_now
    lwip_timers.o(i.sys_check_timeouts) refers to memp.o(i.memp_free) for memp_free
    lwip_timers.o(i.sys_check_timeouts) refers to lwip_timers.o(.data) for .data
    lwip_timers.o(i.sys_restart_timeouts) refers to ethernetif.o(i.sys_now) for sys_now
    lwip_timers.o(i.sys_restart_timeouts) refers to lwip_timers.o(.data) for .data
    lwip_timers.o(i.sys_timeout) refers to memp.o(i.memp_malloc) for memp_malloc
    lwip_timers.o(i.sys_timeout) refers to lwip_timers.o(.data) for .data
    lwip_timers.o(i.sys_timeouts_init) refers to lwip_timers.o(i.sys_timeout) for sys_timeout
    lwip_timers.o(i.sys_timeouts_init) refers to ethernetif.o(i.sys_now) for sys_now
    lwip_timers.o(i.sys_timeouts_init) refers to lwip_timers.o(i.ip_reass_timer) for ip_reass_timer
    lwip_timers.o(i.sys_timeouts_init) refers to lwip_timers.o(i.arp_timer) for arp_timer
    lwip_timers.o(i.sys_timeouts_init) refers to lwip_timers.o(i.dhcp_timer_coarse) for dhcp_timer_coarse
    lwip_timers.o(i.sys_timeouts_init) refers to lwip_timers.o(i.dhcp_timer_fine) for dhcp_timer_fine
    lwip_timers.o(i.sys_timeouts_init) refers to lwip_timers.o(.data) for .data
    lwip_timers.o(i.sys_untimeout) refers to memp.o(i.memp_free) for memp_free
    lwip_timers.o(i.sys_untimeout) refers to lwip_timers.o(.data) for .data
    lwip_timers.o(i.tcp_timer_needed) refers to lwip_timers.o(i.sys_timeout) for sys_timeout
    lwip_timers.o(i.tcp_timer_needed) refers to lwip_timers.o(.data) for .data
    lwip_timers.o(i.tcp_timer_needed) refers to tcp.o(.data) for tcp_active_pcbs
    lwip_timers.o(i.tcp_timer_needed) refers to lwip_timers.o(i.tcpip_tcp_timer) for tcpip_tcp_timer
    lwip_timers.o(i.tcpip_tcp_timer) refers to tcp.o(i.tcp_tmr) for tcp_tmr
    lwip_timers.o(i.tcpip_tcp_timer) refers to lwip_timers.o(i.sys_timeout) for sys_timeout
    lwip_timers.o(i.tcpip_tcp_timer) refers to tcp.o(.data) for tcp_active_pcbs
    lwip_timers.o(i.tcpip_tcp_timer) refers to lwip_timers.o(.data) for .data
    memp.o(i.memp_free) refers to memp.o(.bss) for .bss
    memp.o(i.memp_init) refers to memp.o(.bss) for .bss
    memp.o(i.memp_init) refers to memp.o(.constdata) for .constdata
    memp.o(i.memp_malloc) refers to memp.o(.bss) for .bss
    memp.o(.data) refers to memp.o(.conststring) for .conststring
    dhcp.o(i.dhcp_arp_reply) refers to dhcp.o(i.dhcp_decline) for dhcp_decline
    dhcp.o(i.dhcp_bind) refers to netif.o(i.netif_set_ipaddr) for netif_set_ipaddr
    dhcp.o(i.dhcp_bind) refers to netif.o(i.netif_set_netmask) for netif_set_netmask
    dhcp.o(i.dhcp_bind) refers to netif.o(i.netif_set_gw) for netif_set_gw
    dhcp.o(i.dhcp_bind) refers to netif.o(i.netif_set_up) for netif_set_up
    dhcp.o(i.dhcp_bind) refers to dhcp.o(i.dhcp_set_state) for dhcp_set_state
    dhcp.o(i.dhcp_check) refers to dhcp.o(i.dhcp_set_state) for dhcp_set_state
    dhcp.o(i.dhcp_check) refers to etharp.o(i.etharp_query) for etharp_query
    dhcp.o(i.dhcp_cleanup) refers to mem.o(i.mem_free) for mem_free
    dhcp.o(i.dhcp_coarse_tmr) refers to dhcp.o(i.dhcp_rebind) for dhcp_rebind
    dhcp.o(i.dhcp_coarse_tmr) refers to dhcp.o(i.dhcp_renew) for dhcp_renew
    dhcp.o(i.dhcp_coarse_tmr) refers to netif.o(.data) for netif_list
    dhcp.o(i.dhcp_create_msg) refers to pbuf.o(i.pbuf_alloc) for pbuf_alloc
    dhcp.o(i.dhcp_create_msg) refers to def.o(i.lwip_htonl) for lwip_htonl
    dhcp.o(i.dhcp_create_msg) refers to dhcp.o(i.dhcp_option) for dhcp_option
    dhcp.o(i.dhcp_create_msg) refers to dhcp.o(i.dhcp_option_byte) for dhcp_option_byte
    dhcp.o(i.dhcp_create_msg) refers to dhcp.o(.data) for .data
    dhcp.o(i.dhcp_decline) refers to dhcp.o(i.dhcp_set_state) for dhcp_set_state
    dhcp.o(i.dhcp_decline) refers to dhcp.o(i.dhcp_create_msg) for dhcp_create_msg
    dhcp.o(i.dhcp_decline) refers to dhcp.o(i.dhcp_option) for dhcp_option
    dhcp.o(i.dhcp_decline) refers to def.o(i.lwip_ntohl) for lwip_ntohl
    dhcp.o(i.dhcp_decline) refers to dhcp.o(i.dhcp_option_long) for dhcp_option_long
    dhcp.o(i.dhcp_decline) refers to dhcp.o(i.dhcp_option_trailer) for dhcp_option_trailer
    dhcp.o(i.dhcp_decline) refers to pbuf.o(i.pbuf_realloc) for pbuf_realloc
    dhcp.o(i.dhcp_decline) refers to udp.o(i.udp_sendto_if) for udp_sendto_if
    dhcp.o(i.dhcp_decline) refers to dhcp.o(i.dhcp_delete_msg) for dhcp_delete_msg
    dhcp.o(i.dhcp_decline) refers to ip_addr.o(.constdata) for ip_addr_broadcast
    dhcp.o(i.dhcp_delete_msg) refers to pbuf.o(i.pbuf_free) for pbuf_free
    dhcp.o(i.dhcp_discover) refers to dhcp.o(i.dhcp_set_state) for dhcp_set_state
    dhcp.o(i.dhcp_discover) refers to dhcp.o(i.dhcp_create_msg) for dhcp_create_msg
    dhcp.o(i.dhcp_discover) refers to dhcp.o(i.dhcp_option) for dhcp_option
    dhcp.o(i.dhcp_discover) refers to dhcp.o(i.dhcp_option_short) for dhcp_option_short
    dhcp.o(i.dhcp_discover) refers to dhcp.o(i.dhcp_option_byte) for dhcp_option_byte
    dhcp.o(i.dhcp_discover) refers to dhcp.o(i.dhcp_option_trailer) for dhcp_option_trailer
    dhcp.o(i.dhcp_discover) refers to pbuf.o(i.pbuf_realloc) for pbuf_realloc
    dhcp.o(i.dhcp_discover) refers to udp.o(i.udp_sendto_if) for udp_sendto_if
    dhcp.o(i.dhcp_discover) refers to dhcp.o(i.dhcp_delete_msg) for dhcp_delete_msg
    dhcp.o(i.dhcp_discover) refers to ip_addr.o(.constdata) for ip_addr_broadcast
    dhcp.o(i.dhcp_fine_tmr) refers to dhcp.o(i.dhcp_timeout) for dhcp_timeout
    dhcp.o(i.dhcp_fine_tmr) refers to netif.o(.data) for netif_list
    dhcp.o(i.dhcp_handle_ack) refers to def.o(i.lwip_htonl) for lwip_htonl
    dhcp.o(i.dhcp_handle_ack) refers to dhcp.o(.bss) for .bss
    dhcp.o(i.dhcp_inform) refers to memseta.o(.text) for __aeabi_memclr4
    dhcp.o(i.dhcp_inform) refers to dhcp.o(i.dhcp_set_state) for dhcp_set_state
    dhcp.o(i.dhcp_inform) refers to udp.o(i.udp_new) for udp_new
    dhcp.o(i.dhcp_inform) refers to udp.o(i.udp_bind) for udp_bind
    dhcp.o(i.dhcp_inform) refers to dhcp.o(i.dhcp_create_msg) for dhcp_create_msg
    dhcp.o(i.dhcp_inform) refers to dhcp.o(i.dhcp_option) for dhcp_option
    dhcp.o(i.dhcp_inform) refers to dhcp.o(i.dhcp_option_short) for dhcp_option_short
    dhcp.o(i.dhcp_inform) refers to dhcp.o(i.dhcp_option_trailer) for dhcp_option_trailer
    dhcp.o(i.dhcp_inform) refers to pbuf.o(i.pbuf_realloc) for pbuf_realloc
    dhcp.o(i.dhcp_inform) refers to udp.o(i.udp_sendto_if) for udp_sendto_if
    dhcp.o(i.dhcp_inform) refers to dhcp.o(i.dhcp_delete_msg) for dhcp_delete_msg
    dhcp.o(i.dhcp_inform) refers to udp.o(i.udp_remove) for udp_remove
    dhcp.o(i.dhcp_inform) refers to ip_addr.o(.constdata) for ip_addr_any
    dhcp.o(i.dhcp_inform) refers to ip_addr.o(.constdata) for ip_addr_broadcast
    dhcp.o(i.dhcp_network_changed) refers to dhcp.o(i.dhcp_discover) for dhcp_discover
    dhcp.o(i.dhcp_network_changed) refers to netif.o(i.netif_set_down) for netif_set_down
    dhcp.o(i.dhcp_network_changed) refers to dhcp.o(i.dhcp_reboot) for dhcp_reboot
    dhcp.o(i.dhcp_parse_reply) refers to memseta.o(.text) for __aeabi_memclr4
    dhcp.o(i.dhcp_parse_reply) refers to pbuf.o(i.pbuf_copy_partial) for pbuf_copy_partial
    dhcp.o(i.dhcp_parse_reply) refers to def.o(i.lwip_htonl) for lwip_htonl
    dhcp.o(i.dhcp_parse_reply) refers to def.o(i.lwip_ntohl) for lwip_ntohl
    dhcp.o(i.dhcp_parse_reply) refers to dhcp.o(.bss) for .bss
    dhcp.o(i.dhcp_rebind) refers to dhcp.o(i.dhcp_set_state) for dhcp_set_state
    dhcp.o(i.dhcp_rebind) refers to dhcp.o(i.dhcp_create_msg) for dhcp_create_msg
    dhcp.o(i.dhcp_rebind) refers to dhcp.o(i.dhcp_option) for dhcp_option
    dhcp.o(i.dhcp_rebind) refers to dhcp.o(i.dhcp_option_short) for dhcp_option_short
    dhcp.o(i.dhcp_rebind) refers to dhcp.o(i.dhcp_option_trailer) for dhcp_option_trailer
    dhcp.o(i.dhcp_rebind) refers to pbuf.o(i.pbuf_realloc) for pbuf_realloc
    dhcp.o(i.dhcp_rebind) refers to udp.o(i.udp_sendto_if) for udp_sendto_if
    dhcp.o(i.dhcp_rebind) refers to dhcp.o(i.dhcp_delete_msg) for dhcp_delete_msg
    dhcp.o(i.dhcp_rebind) refers to ip_addr.o(.constdata) for ip_addr_broadcast
    dhcp.o(i.dhcp_reboot) refers to dhcp.o(i.dhcp_set_state) for dhcp_set_state
    dhcp.o(i.dhcp_reboot) refers to dhcp.o(i.dhcp_create_msg) for dhcp_create_msg
    dhcp.o(i.dhcp_reboot) refers to dhcp.o(i.dhcp_option) for dhcp_option
    dhcp.o(i.dhcp_reboot) refers to dhcp.o(i.dhcp_option_short) for dhcp_option_short
    dhcp.o(i.dhcp_reboot) refers to def.o(i.lwip_ntohl) for lwip_ntohl
    dhcp.o(i.dhcp_reboot) refers to dhcp.o(i.dhcp_option_long) for dhcp_option_long
    dhcp.o(i.dhcp_reboot) refers to dhcp.o(i.dhcp_option_trailer) for dhcp_option_trailer
    dhcp.o(i.dhcp_reboot) refers to pbuf.o(i.pbuf_realloc) for pbuf_realloc
    dhcp.o(i.dhcp_reboot) refers to udp.o(i.udp_sendto_if) for udp_sendto_if
    dhcp.o(i.dhcp_reboot) refers to dhcp.o(i.dhcp_delete_msg) for dhcp_delete_msg
    dhcp.o(i.dhcp_reboot) refers to ip_addr.o(.constdata) for ip_addr_broadcast
    dhcp.o(i.dhcp_recv) refers to def.o(i.lwip_ntohl) for lwip_ntohl
    dhcp.o(i.dhcp_recv) refers to dhcp.o(i.dhcp_parse_reply) for dhcp_parse_reply
    dhcp.o(i.dhcp_recv) refers to dhcp.o(i.dhcp_handle_ack) for dhcp_handle_ack
    dhcp.o(i.dhcp_recv) refers to dhcp.o(i.dhcp_check) for dhcp_check
    dhcp.o(i.dhcp_recv) refers to dhcp.o(i.dhcp_bind) for dhcp_bind
    dhcp.o(i.dhcp_recv) refers to netif.o(i.netif_set_down) for netif_set_down
    dhcp.o(i.dhcp_recv) refers to netif.o(i.netif_set_ipaddr) for netif_set_ipaddr
    dhcp.o(i.dhcp_recv) refers to netif.o(i.netif_set_gw) for netif_set_gw
    dhcp.o(i.dhcp_recv) refers to netif.o(i.netif_set_netmask) for netif_set_netmask
    dhcp.o(i.dhcp_recv) refers to dhcp.o(i.dhcp_set_state) for dhcp_set_state
    dhcp.o(i.dhcp_recv) refers to dhcp.o(i.dhcp_discover) for dhcp_discover
    dhcp.o(i.dhcp_recv) refers to def.o(i.lwip_htonl) for lwip_htonl
    dhcp.o(i.dhcp_recv) refers to dhcp.o(i.dhcp_select) for dhcp_select
    dhcp.o(i.dhcp_recv) refers to pbuf.o(i.pbuf_free) for pbuf_free
    dhcp.o(i.dhcp_recv) refers to dhcp.o(.bss) for .bss
    dhcp.o(i.dhcp_recv) refers to ip_addr.o(.constdata) for ip_addr_any
    dhcp.o(i.dhcp_release) refers to dhcp.o(i.dhcp_set_state) for dhcp_set_state
    dhcp.o(i.dhcp_release) refers to dhcp.o(i.dhcp_create_msg) for dhcp_create_msg
    dhcp.o(i.dhcp_release) refers to dhcp.o(i.dhcp_option_trailer) for dhcp_option_trailer
    dhcp.o(i.dhcp_release) refers to pbuf.o(i.pbuf_realloc) for pbuf_realloc
    dhcp.o(i.dhcp_release) refers to udp.o(i.udp_sendto_if) for udp_sendto_if
    dhcp.o(i.dhcp_release) refers to dhcp.o(i.dhcp_delete_msg) for dhcp_delete_msg
    dhcp.o(i.dhcp_release) refers to netif.o(i.netif_set_down) for netif_set_down
    dhcp.o(i.dhcp_release) refers to netif.o(i.netif_set_ipaddr) for netif_set_ipaddr
    dhcp.o(i.dhcp_release) refers to netif.o(i.netif_set_gw) for netif_set_gw
    dhcp.o(i.dhcp_release) refers to netif.o(i.netif_set_netmask) for netif_set_netmask
    dhcp.o(i.dhcp_release) refers to ip_addr.o(.constdata) for ip_addr_any
    dhcp.o(i.dhcp_renew) refers to dhcp.o(i.dhcp_set_state) for dhcp_set_state
    dhcp.o(i.dhcp_renew) refers to dhcp.o(i.dhcp_create_msg) for dhcp_create_msg
    dhcp.o(i.dhcp_renew) refers to dhcp.o(i.dhcp_option) for dhcp_option
    dhcp.o(i.dhcp_renew) refers to dhcp.o(i.dhcp_option_short) for dhcp_option_short
    dhcp.o(i.dhcp_renew) refers to dhcp.o(i.dhcp_option_trailer) for dhcp_option_trailer
    dhcp.o(i.dhcp_renew) refers to pbuf.o(i.pbuf_realloc) for pbuf_realloc
    dhcp.o(i.dhcp_renew) refers to udp.o(i.udp_sendto_if) for udp_sendto_if
    dhcp.o(i.dhcp_renew) refers to dhcp.o(i.dhcp_delete_msg) for dhcp_delete_msg
    dhcp.o(i.dhcp_select) refers to dhcp.o(i.dhcp_set_state) for dhcp_set_state
    dhcp.o(i.dhcp_select) refers to dhcp.o(i.dhcp_create_msg) for dhcp_create_msg
    dhcp.o(i.dhcp_select) refers to dhcp.o(i.dhcp_option) for dhcp_option
    dhcp.o(i.dhcp_select) refers to dhcp.o(i.dhcp_option_short) for dhcp_option_short
    dhcp.o(i.dhcp_select) refers to def.o(i.lwip_ntohl) for lwip_ntohl
    dhcp.o(i.dhcp_select) refers to dhcp.o(i.dhcp_option_long) for dhcp_option_long
    dhcp.o(i.dhcp_select) refers to dhcp.o(i.dhcp_option_byte) for dhcp_option_byte
    dhcp.o(i.dhcp_select) refers to dhcp.o(i.dhcp_option_trailer) for dhcp_option_trailer
    dhcp.o(i.dhcp_select) refers to pbuf.o(i.pbuf_realloc) for pbuf_realloc
    dhcp.o(i.dhcp_select) refers to udp.o(i.udp_sendto_if) for udp_sendto_if
    dhcp.o(i.dhcp_select) refers to dhcp.o(i.dhcp_delete_msg) for dhcp_delete_msg
    dhcp.o(i.dhcp_select) refers to ip_addr.o(.constdata) for ip_addr_broadcast
    dhcp.o(i.dhcp_set_struct) refers to memseta.o(.text) for __aeabi_memclr4
    dhcp.o(i.dhcp_start) refers to udp.o(i.udp_remove) for udp_remove
    dhcp.o(i.dhcp_start) refers to memseta.o(.text) for __aeabi_memclr4
    dhcp.o(i.dhcp_start) refers to udp.o(i.udp_new) for udp_new
    dhcp.o(i.dhcp_start) refers to udp.o(i.udp_bind) for udp_bind
    dhcp.o(i.dhcp_start) refers to udp.o(i.udp_connect) for udp_connect
    dhcp.o(i.dhcp_start) refers to udp.o(i.udp_recv) for udp_recv
    dhcp.o(i.dhcp_start) refers to dhcp.o(i.dhcp_discover) for dhcp_discover
    dhcp.o(i.dhcp_start) refers to dhcp.o(i.dhcp_stop) for dhcp_stop
    dhcp.o(i.dhcp_start) refers to mem.o(i.mem_malloc) for mem_malloc
    dhcp.o(i.dhcp_start) refers to ip_addr.o(.constdata) for ip_addr_any
    dhcp.o(i.dhcp_start) refers to dhcp.o(i.dhcp_recv) for dhcp_recv
    dhcp.o(i.dhcp_stop) refers to udp.o(i.udp_remove) for udp_remove
    dhcp.o(i.dhcp_stop) refers to dhcp.o(i.dhcp_set_state) for dhcp_set_state
    dhcp.o(i.dhcp_timeout) refers to dhcp.o(i.dhcp_reboot) for dhcp_reboot
    dhcp.o(i.dhcp_timeout) refers to dhcp.o(i.dhcp_discover) for dhcp_discover
    dhcp.o(i.dhcp_timeout) refers to dhcp.o(i.dhcp_select) for dhcp_select
    dhcp.o(i.dhcp_timeout) refers to dhcp.o(i.dhcp_release) for dhcp_release
    dhcp.o(i.dhcp_timeout) refers to dhcp.o(i.dhcp_check) for dhcp_check
    dhcp.o(i.dhcp_timeout) refers to dhcp.o(i.dhcp_bind) for dhcp_bind
    dhcp.o(i.dhcp_timeout) refers to dhcp.o(i.dhcp_renew) for dhcp_renew
    dhcp.o(i.dhcp_timeout) refers to dhcp.o(i.dhcp_rebind) for dhcp_rebind
    udp.o(i.udp_bind) refers to udp.o(.data) for .data
    udp.o(i.udp_connect) refers to udp.o(i.udp_bind) for udp_bind
    udp.o(i.udp_connect) refers to udp.o(.data) for .data
    udp.o(i.udp_input) refers to pbuf.o(i.pbuf_header) for pbuf_header
    udp.o(i.udp_input) refers to ip_addr.o(i.ip4_addr_isbroadcast) for ip4_addr_isbroadcast
    udp.o(i.udp_input) refers to def.o(i.lwip_ntohs) for lwip_ntohs
    udp.o(i.udp_input) refers to icmp.o(i.icmp_dest_unreach) for icmp_dest_unreach
    udp.o(i.udp_input) refers to pbuf.o(i.pbuf_free) for pbuf_free
    udp.o(i.udp_input) refers to ip.o(.data) for current_iphdr_dest
    udp.o(i.udp_input) refers to udp.o(.data) for .data
    udp.o(i.udp_new) refers to memp.o(i.memp_malloc) for memp_malloc
    udp.o(i.udp_new) refers to memseta.o(.text) for __aeabi_memclr4
    udp.o(i.udp_remove) refers to memp.o(i.memp_free) for memp_free
    udp.o(i.udp_remove) refers to udp.o(.data) for .data
    udp.o(i.udp_send) refers to udp.o(i.udp_sendto) for udp_sendto
    udp.o(i.udp_sendto) refers to ip.o(i.ip_route) for ip_route
    udp.o(i.udp_sendto) refers to udp.o(i.udp_sendto_if) for udp_sendto_if
    udp.o(i.udp_sendto_if) refers to udp.o(i.udp_bind) for udp_bind
    udp.o(i.udp_sendto_if) refers to pbuf.o(i.pbuf_header) for pbuf_header
    udp.o(i.udp_sendto_if) refers to pbuf.o(i.pbuf_alloc) for pbuf_alloc
    udp.o(i.udp_sendto_if) refers to pbuf.o(i.pbuf_chain) for pbuf_chain
    udp.o(i.udp_sendto_if) refers to def.o(i.lwip_htons) for lwip_htons
    udp.o(i.udp_sendto_if) refers to pbuf.o(i.pbuf_free) for pbuf_free
    udp.o(i.udp_sendto_if) refers to ip.o(i.ip_output_if) for ip_output_if
    mem.o(i.mem_calloc) refers to mem.o(i.mem_malloc) for mem_malloc
    mem.o(i.mem_calloc) refers to memseta.o(.text) for __aeabi_memclr
    mem.o(i.mem_free) refers to mem.o(i.plug_holes) for plug_holes
    mem.o(i.mem_free) refers to mem.o(.data) for .data
    mem.o(i.mem_init) refers to mem.o(.bss) for .bss
    mem.o(i.mem_init) refers to mem.o(.data) for .data
    mem.o(i.mem_malloc) refers to mem.o(.data) for .data
    mem.o(i.mem_trim) refers to mem.o(.data) for .data
    mem.o(i.plug_holes) refers to mem.o(.data) for .data
    netif.o(i.netif_add) refers to netif.o(i.netif_set_addr) for netif_set_addr
    netif.o(i.netif_add) refers to netif.o(.data) for .data
    netif.o(i.netif_find) refers to netif.o(.data) for .data
    netif.o(i.netif_remove) refers to netif.o(i.netif_set_down) for netif_set_down
    netif.o(i.netif_remove) refers to netif.o(.data) for .data
    netif.o(i.netif_set_addr) refers to netif.o(i.netif_set_ipaddr) for netif_set_ipaddr
    netif.o(i.netif_set_addr) refers to netif.o(i.netif_set_netmask) for netif_set_netmask
    netif.o(i.netif_set_addr) refers to netif.o(i.netif_set_gw) for netif_set_gw
    netif.o(i.netif_set_default) refers to netif.o(.data) for .data
    netif.o(i.netif_set_down) refers to etharp.o(i.etharp_cleanup_netif) for etharp_cleanup_netif
    netif.o(i.netif_set_ipaddr) refers to tcp.o(i.tcp_abort) for tcp_abort
    netif.o(i.netif_set_ipaddr) refers to tcp.o(.data) for tcp_active_pcbs
    netif.o(i.netif_set_link_up) refers to dhcp.o(i.dhcp_network_changed) for dhcp_network_changed
    netif.o(i.netif_set_link_up) refers to etharp.o(i.etharp_request) for etharp_request
    netif.o(i.netif_set_up) refers to etharp.o(i.etharp_request) for etharp_request
    tcp.o(i.tcp_abandon) refers to tcp.o(i.tcp_pcb_remove) for tcp_pcb_remove
    tcp.o(i.tcp_abandon) refers to tcp.o(i.tcp_segs_free) for tcp_segs_free
    tcp.o(i.tcp_abandon) refers to tcp_out.o(i.tcp_rst) for tcp_rst
    tcp.o(i.tcp_abandon) refers to memp.o(i.memp_free) for memp_free
    tcp.o(i.tcp_abandon) refers to tcp.o(.data) for .data
    tcp.o(i.tcp_abort) refers to tcp.o(i.tcp_abandon) for tcp_abandon
    tcp.o(i.tcp_alloc) refers to memp.o(i.memp_malloc) for memp_malloc
    tcp.o(i.tcp_alloc) refers to tcp.o(i.tcp_abort) for tcp_abort
    tcp.o(i.tcp_alloc) refers to memseta.o(.text) for __aeabi_memclr4
    tcp.o(i.tcp_alloc) refers to tcp.o(i.tcp_next_iss) for tcp_next_iss
    tcp.o(i.tcp_alloc) refers to tcp.o(.data) for .data
    tcp.o(i.tcp_alloc) refers to tcp.o(i.tcp_recv_null) for tcp_recv_null
    tcp.o(i.tcp_bind) refers to tcp.o(i.tcp_new_port) for tcp_new_port
    tcp.o(i.tcp_bind) refers to lwip_timers.o(i.tcp_timer_needed) for tcp_timer_needed
    tcp.o(i.tcp_bind) refers to tcp.o(.constdata) for .constdata
    tcp.o(i.tcp_bind) refers to tcp.o(.data) for .data
    tcp.o(i.tcp_close) refers to tcp.o(i.tcp_close_shutdown) for tcp_close_shutdown
    tcp.o(i.tcp_close_shutdown) refers to tcp_out.o(i.tcp_rst) for tcp_rst
    tcp.o(i.tcp_close_shutdown) refers to tcp.o(i.tcp_pcb_purge) for tcp_pcb_purge
    tcp.o(i.tcp_close_shutdown) refers to memp.o(i.memp_free) for memp_free
    tcp.o(i.tcp_close_shutdown) refers to lwip_timers.o(i.tcp_timer_needed) for tcp_timer_needed
    tcp.o(i.tcp_close_shutdown) refers to tcp.o(i.tcp_pcb_remove) for tcp_pcb_remove
    tcp.o(i.tcp_close_shutdown) refers to tcp_out.o(i.tcp_send_fin) for tcp_send_fin
    tcp.o(i.tcp_close_shutdown) refers to tcp_out.o(i.tcp_output) for tcp_output
    tcp.o(i.tcp_close_shutdown) refers to tcp.o(.data) for .data
    tcp.o(i.tcp_connect) refers to ip.o(i.ip_route) for ip_route
    tcp.o(i.tcp_connect) refers to tcp.o(i.tcp_new_port) for tcp_new_port
    tcp.o(i.tcp_connect) refers to tcp.o(i.tcp_next_iss) for tcp_next_iss
    tcp.o(i.tcp_connect) refers to tcp.o(i.tcp_eff_send_mss) for tcp_eff_send_mss
    tcp.o(i.tcp_connect) refers to tcp_out.o(i.tcp_enqueue_flags) for tcp_enqueue_flags
    tcp.o(i.tcp_connect) refers to lwip_timers.o(i.tcp_timer_needed) for tcp_timer_needed
    tcp.o(i.tcp_connect) refers to tcp_out.o(i.tcp_output) for tcp_output
    tcp.o(i.tcp_connect) refers to tcp.o(.data) for .data
    tcp.o(i.tcp_debug_state_str) refers to tcp.o(.constdata) for .constdata
    tcp.o(i.tcp_eff_send_mss) refers to ip.o(i.ip_route) for ip_route
    tcp.o(i.tcp_fasttmr) refers to tcp_out.o(i.tcp_output) for tcp_output
    tcp.o(i.tcp_fasttmr) refers to tcp.o(i.tcp_process_refused_data) for tcp_process_refused_data
    tcp.o(i.tcp_fasttmr) refers to tcp.o(.data) for .data
    tcp.o(i.tcp_listen_with_backlog) refers to memp.o(i.memp_malloc) for memp_malloc
    tcp.o(i.tcp_listen_with_backlog) refers to memp.o(i.memp_free) for memp_free
    tcp.o(i.tcp_listen_with_backlog) refers to lwip_timers.o(i.tcp_timer_needed) for tcp_timer_needed
    tcp.o(i.tcp_listen_with_backlog) refers to tcp.o(.data) for .data
    tcp.o(i.tcp_listen_with_backlog) refers to tcp.o(i.tcp_accept_null) for tcp_accept_null
    tcp.o(i.tcp_new) refers to tcp.o(i.tcp_alloc) for tcp_alloc
    tcp.o(i.tcp_new_port) refers to tcp.o(.constdata) for .constdata
    tcp.o(i.tcp_new_port) refers to tcp.o(.data) for .data
    tcp.o(i.tcp_next_iss) refers to tcp.o(.data) for .data
    tcp.o(i.tcp_pcb_purge) refers to pbuf.o(i.pbuf_free) for pbuf_free
    tcp.o(i.tcp_pcb_purge) refers to tcp.o(i.tcp_segs_free) for tcp_segs_free
    tcp.o(i.tcp_pcb_remove) refers to tcp.o(i.tcp_pcb_purge) for tcp_pcb_purge
    tcp.o(i.tcp_pcb_remove) refers to tcp_out.o(i.tcp_output) for tcp_output
    tcp.o(i.tcp_pcb_remove) refers to tcp.o(.data) for .data
    tcp.o(i.tcp_process_refused_data) refers to tcp.o(i.tcp_recv_null) for tcp_recv_null
    tcp.o(i.tcp_recv_null) refers to tcp.o(i.tcp_recved) for tcp_recved
    tcp.o(i.tcp_recv_null) refers to pbuf.o(i.pbuf_free) for pbuf_free
    tcp.o(i.tcp_recv_null) refers to tcp.o(i.tcp_close) for tcp_close
    tcp.o(i.tcp_recved) refers to tcp.o(i.tcp_update_rcv_ann_wnd) for tcp_update_rcv_ann_wnd
    tcp.o(i.tcp_recved) refers to tcp_out.o(i.tcp_output) for tcp_output
    tcp.o(i.tcp_seg_free) refers to pbuf.o(i.pbuf_free) for pbuf_free
    tcp.o(i.tcp_seg_free) refers to memp.o(i.memp_free) for memp_free
    tcp.o(i.tcp_segs_free) refers to tcp.o(i.tcp_seg_free) for tcp_seg_free
    tcp.o(i.tcp_shutdown) refers to pbuf.o(i.pbuf_free) for pbuf_free
    tcp.o(i.tcp_shutdown) refers to tcp.o(i.tcp_close_shutdown) for tcp_close_shutdown
    tcp.o(i.tcp_slowtmr) refers to tcp_out.o(i.tcp_zero_window_probe) for tcp_zero_window_probe
    tcp.o(i.tcp_slowtmr) refers to tcp_out.o(i.tcp_rexmit_rto) for tcp_rexmit_rto
    tcp.o(i.tcp_slowtmr) refers to tcp_out.o(i.tcp_keepalive) for tcp_keepalive
    tcp.o(i.tcp_slowtmr) refers to tcp.o(i.tcp_pcb_purge) for tcp_pcb_purge
    tcp.o(i.tcp_slowtmr) refers to tcp_out.o(i.tcp_rst) for tcp_rst
    tcp.o(i.tcp_slowtmr) refers to memp.o(i.memp_free) for memp_free
    tcp.o(i.tcp_slowtmr) refers to tcp_out.o(i.tcp_output) for tcp_output
    tcp.o(i.tcp_slowtmr) refers to tcp.o(.data) for .data
    tcp.o(i.tcp_slowtmr) refers to tcp.o(.constdata) for .constdata
    tcp.o(i.tcp_tmr) refers to tcp.o(i.tcp_fasttmr) for tcp_fasttmr
    tcp.o(i.tcp_tmr) refers to tcp.o(i.tcp_slowtmr) for tcp_slowtmr
    tcp.o(i.tcp_tmr) refers to tcp.o(.data) for .data
    tcp.o(.constdata) refers to tcp.o(.conststring) for .conststring
    tcp.o(.constdata) refers to tcp.o(.data) for tcp_listen_pcbs
    tcp_out.o(i.tcp_create_segment) refers to memp.o(i.memp_malloc) for memp_malloc
    tcp_out.o(i.tcp_create_segment) refers to pbuf.o(i.pbuf_header) for pbuf_header
    tcp_out.o(i.tcp_create_segment) refers to tcp.o(i.tcp_seg_free) for tcp_seg_free
    tcp_out.o(i.tcp_create_segment) refers to pbuf.o(i.pbuf_free) for pbuf_free
    tcp_out.o(i.tcp_create_segment) refers to def.o(i.lwip_htons) for lwip_htons
    tcp_out.o(i.tcp_create_segment) refers to def.o(i.lwip_htonl) for lwip_htonl
    tcp_out.o(i.tcp_enqueue_flags) refers to pbuf.o(i.pbuf_alloc) for pbuf_alloc
    tcp_out.o(i.tcp_enqueue_flags) refers to tcp_out.o(i.tcp_create_segment) for tcp_create_segment
    tcp_out.o(i.tcp_enqueue_flags) refers to pbuf.o(i.pbuf_clen) for pbuf_clen
    tcp_out.o(i.tcp_keepalive) refers to def.o(i.lwip_htonl) for lwip_htonl
    tcp_out.o(i.tcp_keepalive) refers to tcp_out.o(i.tcp_output_alloc_header) for tcp_output_alloc_header
    tcp_out.o(i.tcp_keepalive) refers to ip.o(i.ip_output) for ip_output
    tcp_out.o(i.tcp_keepalive) refers to pbuf.o(i.pbuf_free) for pbuf_free
    tcp_out.o(i.tcp_output) refers to def.o(i.lwip_ntohl) for lwip_ntohl
    tcp_out.o(i.tcp_output) refers to tcp_out.o(i.tcp_send_empty_ack) for tcp_send_empty_ack
    tcp_out.o(i.tcp_output) refers to def.o(i.lwip_ntohs) for lwip_ntohs
    tcp_out.o(i.tcp_output) refers to def.o(i.lwip_htons) for lwip_htons
    tcp_out.o(i.tcp_output) refers to tcp_out.o(i.tcp_output_segment) for tcp_output_segment
    tcp_out.o(i.tcp_output) refers to tcp.o(i.tcp_seg_free) for tcp_seg_free
    tcp_out.o(i.tcp_output) refers to tcp_in.o(.data) for tcp_input_pcb
    tcp_out.o(i.tcp_output_alloc_header) refers to pbuf.o(i.pbuf_alloc) for pbuf_alloc
    tcp_out.o(i.tcp_output_alloc_header) refers to def.o(i.lwip_htons) for lwip_htons
    tcp_out.o(i.tcp_output_alloc_header) refers to def.o(i.lwip_htonl) for lwip_htonl
    tcp_out.o(i.tcp_output_segment) refers to def.o(i.lwip_htonl) for lwip_htonl
    tcp_out.o(i.tcp_output_segment) refers to def.o(i.lwip_htons) for lwip_htons
    tcp_out.o(i.tcp_output_segment) refers to tcp.o(i.tcp_eff_send_mss) for tcp_eff_send_mss
    tcp_out.o(i.tcp_output_segment) refers to ip.o(i.ip_route) for ip_route
    tcp_out.o(i.tcp_output_segment) refers to def.o(i.lwip_ntohl) for lwip_ntohl
    tcp_out.o(i.tcp_output_segment) refers to ip.o(i.ip_output) for ip_output
    tcp_out.o(i.tcp_output_segment) refers to tcp.o(.data) for tcp_ticks
    tcp_out.o(i.tcp_pbuf_prealloc) refers to pbuf.o(i.pbuf_alloc) for pbuf_alloc
    tcp_out.o(i.tcp_rexmit) refers to def.o(i.lwip_ntohl) for lwip_ntohl
    tcp_out.o(i.tcp_rexmit_fast) refers to tcp_out.o(i.tcp_rexmit) for tcp_rexmit
    tcp_out.o(i.tcp_rexmit_rto) refers to tcp_out.o(i.tcp_output) for tcp_output
    tcp_out.o(i.tcp_rst) refers to pbuf.o(i.pbuf_alloc) for pbuf_alloc
    tcp_out.o(i.tcp_rst) refers to def.o(i.lwip_htons) for lwip_htons
    tcp_out.o(i.tcp_rst) refers to def.o(i.lwip_htonl) for lwip_htonl
    tcp_out.o(i.tcp_rst) refers to ip.o(i.ip_output) for ip_output
    tcp_out.o(i.tcp_rst) refers to pbuf.o(i.pbuf_free) for pbuf_free
    tcp_out.o(i.tcp_send_empty_ack) refers to def.o(i.lwip_htonl) for lwip_htonl
    tcp_out.o(i.tcp_send_empty_ack) refers to tcp_out.o(i.tcp_output_alloc_header) for tcp_output_alloc_header
    tcp_out.o(i.tcp_send_empty_ack) refers to ip.o(i.ip_output) for ip_output
    tcp_out.o(i.tcp_send_empty_ack) refers to pbuf.o(i.pbuf_free) for pbuf_free
    tcp_out.o(i.tcp_send_fin) refers to def.o(i.lwip_ntohs) for lwip_ntohs
    tcp_out.o(i.tcp_send_fin) refers to tcp_out.o(i.tcp_enqueue_flags) for tcp_enqueue_flags
    tcp_out.o(i.tcp_send_fin) refers to def.o(i.lwip_htons) for lwip_htons
    tcp_out.o(i.tcp_write) refers to tcp_out.o(i.tcp_pbuf_prealloc) for tcp_pbuf_prealloc
    tcp_out.o(i.tcp_write) refers to memcpya.o(.text) for __aeabi_memcpy
    tcp_out.o(i.tcp_write) refers to pbuf.o(i.pbuf_alloc) for pbuf_alloc
    tcp_out.o(i.tcp_write) refers to pbuf.o(i.pbuf_clen) for pbuf_clen
    tcp_out.o(i.tcp_write) refers to pbuf.o(i.pbuf_cat) for pbuf_cat
    tcp_out.o(i.tcp_write) refers to pbuf.o(i.pbuf_free) for pbuf_free
    tcp_out.o(i.tcp_write) refers to tcp_out.o(i.tcp_create_segment) for tcp_create_segment
    tcp_out.o(i.tcp_write) refers to def.o(i.lwip_htons) for lwip_htons
    tcp_out.o(i.tcp_write) refers to tcp.o(i.tcp_segs_free) for tcp_segs_free
    tcp_out.o(i.tcp_zero_window_probe) refers to def.o(i.lwip_ntohs) for lwip_ntohs
    tcp_out.o(i.tcp_zero_window_probe) refers to tcp_out.o(i.tcp_output_alloc_header) for tcp_output_alloc_header
    tcp_out.o(i.tcp_zero_window_probe) refers to def.o(i.lwip_htons) for lwip_htons
    tcp_out.o(i.tcp_zero_window_probe) refers to pbuf.o(i.pbuf_copy_partial) for pbuf_copy_partial
    tcp_out.o(i.tcp_zero_window_probe) refers to ip.o(i.ip_output) for ip_output
    tcp_out.o(i.tcp_zero_window_probe) refers to pbuf.o(i.pbuf_free) for pbuf_free
    raw.o(i.raw_input) refers to raw.o(.data) for .data
    raw.o(i.raw_input) refers to ip.o(.data) for current_iphdr_dest
    raw.o(i.raw_new) refers to memp.o(i.memp_malloc) for memp_malloc
    raw.o(i.raw_new) refers to memseta.o(.text) for __aeabi_memclr4
    raw.o(i.raw_new) refers to raw.o(.data) for .data
    raw.o(i.raw_remove) refers to memp.o(i.memp_free) for memp_free
    raw.o(i.raw_remove) refers to raw.o(.data) for .data
    raw.o(i.raw_send) refers to raw.o(i.raw_sendto) for raw_sendto
    raw.o(i.raw_sendto) refers to pbuf.o(i.pbuf_header) for pbuf_header
    raw.o(i.raw_sendto) refers to pbuf.o(i.pbuf_alloc) for pbuf_alloc
    raw.o(i.raw_sendto) refers to pbuf.o(i.pbuf_chain) for pbuf_chain
    raw.o(i.raw_sendto) refers to ip.o(i.ip_route) for ip_route
    raw.o(i.raw_sendto) refers to ip.o(i.ip_output_if) for ip_output_if
    raw.o(i.raw_sendto) refers to pbuf.o(i.pbuf_free) for pbuf_free
    init.o(i.lwip_init) refers to mem.o(i.mem_init) for mem_init
    init.o(i.lwip_init) refers to memp.o(i.memp_init) for memp_init
    init.o(i.lwip_init) refers to netif.o(i.netif_init) for netif_init
    init.o(i.lwip_init) refers to udp.o(i.udp_init) for udp_init
    init.o(i.lwip_init) refers to tcp.o(i.tcp_init) for tcp_init
    init.o(i.lwip_init) refers to lwip_timers.o(i.sys_timeouts_init) for sys_timeouts_init
    pbuf.o(i.pbuf_alloc) refers to memp.o(i.memp_malloc) for memp_malloc
    pbuf.o(i.pbuf_alloc) refers to pbuf.o(i.pbuf_free) for pbuf_free
    pbuf.o(i.pbuf_alloc) refers to mem.o(i.mem_malloc) for mem_malloc
    pbuf.o(i.pbuf_chain) refers to pbuf.o(i.pbuf_cat) for pbuf_cat
    pbuf.o(i.pbuf_chain) refers to pbuf.o(i.pbuf_ref) for pbuf_ref
    pbuf.o(i.pbuf_coalesce) refers to pbuf.o(i.pbuf_alloc) for pbuf_alloc
    pbuf.o(i.pbuf_coalesce) refers to pbuf.o(i.pbuf_copy) for pbuf_copy
    pbuf.o(i.pbuf_coalesce) refers to pbuf.o(i.pbuf_free) for pbuf_free
    pbuf.o(i.pbuf_copy) refers to memcpya.o(.text) for __aeabi_memcpy
    pbuf.o(i.pbuf_copy_partial) refers to memcpya.o(.text) for __aeabi_memcpy
    pbuf.o(i.pbuf_dechain) refers to pbuf.o(i.pbuf_free) for pbuf_free
    pbuf.o(i.pbuf_free) refers to mem.o(i.mem_free) for mem_free
    pbuf.o(i.pbuf_free) refers to memp.o(i.memp_free) for memp_free
    pbuf.o(i.pbuf_memcmp) refers to pbuf.o(i.pbuf_get_at) for pbuf_get_at
    pbuf.o(i.pbuf_memfind) refers to pbuf.o(i.pbuf_memcmp) for pbuf_memcmp
    pbuf.o(i.pbuf_realloc) refers to mem.o(i.mem_trim) for mem_trim
    pbuf.o(i.pbuf_realloc) refers to pbuf.o(i.pbuf_free) for pbuf_free
    pbuf.o(i.pbuf_strstr) refers to strlen.o(.text) for strlen
    pbuf.o(i.pbuf_strstr) refers to pbuf.o(i.pbuf_memfind) for pbuf_memfind
    pbuf.o(i.pbuf_take) refers to memcpya.o(.text) for __aeabi_memcpy
    ip_addr.o(i.ip4_addr_netmask_valid) refers to def.o(i.lwip_htonl) for lwip_htonl
    ip_addr.o(i.ipaddr_addr) refers to ip_addr.o(i.ipaddr_aton) for ipaddr_aton
    ip_addr.o(i.ipaddr_aton) refers to def.o(i.lwip_htonl) for lwip_htonl
    ip_addr.o(i.ipaddr_ntoa) refers to ip_addr.o(i.ipaddr_ntoa_r) for ipaddr_ntoa_r
    ip_addr.o(i.ipaddr_ntoa) refers to ip_addr.o(.bss) for .bss
    inet_chksum.o(i.inet_chksum) refers to inet_chksum.o(i.lwip_standard_chksum) for lwip_standard_chksum
    inet_chksum.o(i.inet_chksum_pbuf) refers to inet_chksum.o(i.lwip_standard_chksum) for lwip_standard_chksum
    inet_chksum.o(i.inet_chksum_pseudo) refers to inet_chksum.o(i.lwip_standard_chksum) for lwip_standard_chksum
    inet_chksum.o(i.inet_chksum_pseudo) refers to def.o(i.lwip_htons) for lwip_htons
    inet_chksum.o(i.inet_chksum_pseudo_partial) refers to inet_chksum.o(i.lwip_standard_chksum) for lwip_standard_chksum
    inet_chksum.o(i.inet_chksum_pseudo_partial) refers to def.o(i.lwip_htons) for lwip_htons
    ip_frag.o(i.ip_frag) refers to def.o(i.lwip_ntohs) for lwip_ntohs
    ip_frag.o(i.ip_frag) refers to pbuf.o(i.pbuf_alloc) for pbuf_alloc
    ip_frag.o(i.ip_frag) refers to memcpya.o(.text) for __aeabi_memcpy
    ip_frag.o(i.ip_frag) refers to memp.o(i.memp_malloc) for memp_malloc
    ip_frag.o(i.ip_frag) refers to pbuf.o(i.pbuf_alloced_custom) for pbuf_alloced_custom
    ip_frag.o(i.ip_frag) refers to pbuf.o(i.pbuf_ref) for pbuf_ref
    ip_frag.o(i.ip_frag) refers to pbuf.o(i.pbuf_cat) for pbuf_cat
    ip_frag.o(i.ip_frag) refers to def.o(i.lwip_htons) for lwip_htons
    ip_frag.o(i.ip_frag) refers to inet_chksum.o(i.inet_chksum) for inet_chksum
    ip_frag.o(i.ip_frag) refers to pbuf.o(i.pbuf_free) for pbuf_free
    ip_frag.o(i.ip_frag) refers to ip_frag.o(i.ip_frag_free_pbuf_custom_ref) for ip_frag_free_pbuf_custom_ref
    ip_frag.o(i.ip_frag) refers to ip_frag.o(i.ipfrag_free_pbuf_custom) for ipfrag_free_pbuf_custom
    ip_frag.o(i.ip_frag_free_pbuf_custom_ref) refers to memp.o(i.memp_free) for memp_free
    ip_frag.o(i.ip_reass) refers to def.o(i.lwip_ntohs) for lwip_ntohs
    ip_frag.o(i.ip_reass) refers to pbuf.o(i.pbuf_clen) for pbuf_clen
    ip_frag.o(i.ip_reass) refers to ip_frag.o(i.ip_reass_remove_oldest_datagram) for ip_reass_remove_oldest_datagram
    ip_frag.o(i.ip_reass) refers to memp.o(i.memp_malloc) for memp_malloc
    ip_frag.o(i.ip_reass) refers to memseta.o(.text) for __aeabi_memclr4
    ip_frag.o(i.ip_reass) refers to memcpya.o(.text) for __aeabi_memcpy
    ip_frag.o(i.ip_reass) refers to ip_frag.o(i.ip_reass_chain_frag_into_datagram_and_validate) for ip_reass_chain_frag_into_datagram_and_validate
    ip_frag.o(i.ip_reass) refers to def.o(i.lwip_htons) for lwip_htons
    ip_frag.o(i.ip_reass) refers to inet_chksum.o(i.inet_chksum) for inet_chksum
    ip_frag.o(i.ip_reass) refers to pbuf.o(i.pbuf_header) for pbuf_header
    ip_frag.o(i.ip_reass) refers to pbuf.o(i.pbuf_cat) for pbuf_cat
    ip_frag.o(i.ip_reass) refers to ip_frag.o(i.ip_reass_dequeue_datagram) for ip_reass_dequeue_datagram
    ip_frag.o(i.ip_reass) refers to pbuf.o(i.pbuf_free) for pbuf_free
    ip_frag.o(i.ip_reass) refers to ip_frag.o(.data) for .data
    ip_frag.o(i.ip_reass_chain_frag_into_datagram_and_validate) refers to def.o(i.lwip_ntohs) for lwip_ntohs
    ip_frag.o(i.ip_reass_chain_frag_into_datagram_and_validate) refers to pbuf.o(i.pbuf_clen) for pbuf_clen
    ip_frag.o(i.ip_reass_chain_frag_into_datagram_and_validate) refers to pbuf.o(i.pbuf_free) for pbuf_free
    ip_frag.o(i.ip_reass_chain_frag_into_datagram_and_validate) refers to ip_frag.o(.data) for .data
    ip_frag.o(i.ip_reass_dequeue_datagram) refers to memp.o(i.memp_free) for memp_free
    ip_frag.o(i.ip_reass_dequeue_datagram) refers to ip_frag.o(.data) for .data
    ip_frag.o(i.ip_reass_free_complete_datagram) refers to memcpya.o(.text) for __aeabi_memcpy
    ip_frag.o(i.ip_reass_free_complete_datagram) refers to icmp.o(i.icmp_time_exceeded) for icmp_time_exceeded
    ip_frag.o(i.ip_reass_free_complete_datagram) refers to pbuf.o(i.pbuf_clen) for pbuf_clen
    ip_frag.o(i.ip_reass_free_complete_datagram) refers to pbuf.o(i.pbuf_free) for pbuf_free
    ip_frag.o(i.ip_reass_free_complete_datagram) refers to ip_frag.o(i.ip_reass_dequeue_datagram) for ip_reass_dequeue_datagram
    ip_frag.o(i.ip_reass_free_complete_datagram) refers to ip_frag.o(.data) for .data
    ip_frag.o(i.ip_reass_remove_oldest_datagram) refers to ip_frag.o(i.ip_reass_free_complete_datagram) for ip_reass_free_complete_datagram
    ip_frag.o(i.ip_reass_remove_oldest_datagram) refers to ip_frag.o(.data) for .data
    ip_frag.o(i.ip_reass_tmr) refers to ip_frag.o(i.ip_reass_free_complete_datagram) for ip_reass_free_complete_datagram
    ip_frag.o(i.ip_reass_tmr) refers to ip_frag.o(.data) for .data
    ip_frag.o(i.ipfrag_free_pbuf_custom) refers to pbuf.o(i.pbuf_free) for pbuf_free
    ip_frag.o(i.ipfrag_free_pbuf_custom) refers to ip_frag.o(i.ip_frag_free_pbuf_custom_ref) for ip_frag_free_pbuf_custom_ref
    ip.o(i.ip_input) refers to def.o(i.lwip_ntohs) for lwip_ntohs
    ip.o(i.ip_input) refers to pbuf.o(i.pbuf_free) for pbuf_free
    ip.o(i.ip_input) refers to pbuf.o(i.pbuf_realloc) for pbuf_realloc
    ip.o(i.ip_input) refers to ip_addr.o(i.ip4_addr_isbroadcast) for ip4_addr_isbroadcast
    ip.o(i.ip_input) refers to ip_frag.o(i.ip_reass) for ip_reass
    ip.o(i.ip_input) refers to raw.o(i.raw_input) for raw_input
    ip.o(i.ip_input) refers to udp.o(i.udp_input) for udp_input
    ip.o(i.ip_input) refers to tcp_in.o(i.tcp_input) for tcp_input
    ip.o(i.ip_input) refers to icmp.o(i.icmp_input) for icmp_input
    ip.o(i.ip_input) refers to icmp.o(i.icmp_dest_unreach) for icmp_dest_unreach
    ip.o(i.ip_input) refers to ip.o(.data) for .data
    ip.o(i.ip_input) refers to netif.o(.data) for netif_list
    ip.o(i.ip_output) refers to ip.o(i.ip_route) for ip_route
    ip.o(i.ip_output) refers to ip.o(i.ip_output_if) for ip_output_if
    ip.o(i.ip_output_if) refers to pbuf.o(i.pbuf_header) for pbuf_header
    ip.o(i.ip_output_if) refers to def.o(i.lwip_htons) for lwip_htons
    ip.o(i.ip_output_if) refers to ip_frag.o(i.ip_frag) for ip_frag
    ip.o(i.ip_output_if) refers to ip.o(.data) for .data
    ip.o(i.ip_route) refers to netif.o(.data) for netif_list
    icmp.o(i.icmp_dest_unreach) refers to icmp.o(i.icmp_send_response) for icmp_send_response
    icmp.o(i.icmp_input) refers to pbuf.o(i.pbuf_header) for pbuf_header
    icmp.o(i.icmp_input) refers to ip_addr.o(i.ip4_addr_isbroadcast) for ip4_addr_isbroadcast
    icmp.o(i.icmp_input) refers to inet_chksum.o(i.inet_chksum_pbuf) for inet_chksum_pbuf
    icmp.o(i.icmp_input) refers to pbuf.o(i.pbuf_alloc) for pbuf_alloc
    icmp.o(i.icmp_input) refers to pbuf.o(i.pbuf_copy) for pbuf_copy
    icmp.o(i.icmp_input) refers to pbuf.o(i.pbuf_free) for pbuf_free
    icmp.o(i.icmp_input) refers to ip.o(i.ip_output_if) for ip_output_if
    icmp.o(i.icmp_input) refers to ip.o(.data) for current_iphdr_dest
    icmp.o(i.icmp_send_response) refers to pbuf.o(i.pbuf_alloc) for pbuf_alloc
    icmp.o(i.icmp_send_response) refers to memcpya.o(.text) for __aeabi_memcpy
    icmp.o(i.icmp_send_response) refers to inet_chksum.o(i.inet_chksum) for inet_chksum
    icmp.o(i.icmp_send_response) refers to ip.o(i.ip_output) for ip_output
    icmp.o(i.icmp_send_response) refers to pbuf.o(i.pbuf_free) for pbuf_free
    icmp.o(i.icmp_time_exceeded) refers to icmp.o(i.icmp_send_response) for icmp_send_response
    err.o(i.lwip_strerr) refers to err.o(.data) for .data
    err.o(.data) refers to err.o(.conststring) for .conststring
    etharp.o(i.etharp_arp_input) refers to etharp.o(i.etharp_update_arp_entry) for etharp_update_arp_entry
    etharp.o(i.etharp_arp_input) refers to def.o(i.lwip_htons) for lwip_htons
    etharp.o(i.etharp_arp_input) refers to dhcp.o(i.dhcp_arp_reply) for dhcp_arp_reply
    etharp.o(i.etharp_arp_input) refers to pbuf.o(i.pbuf_free) for pbuf_free
    etharp.o(i.etharp_cleanup_netif) refers to etharp.o(i.etharp_free_entry) for etharp_free_entry
    etharp.o(i.etharp_cleanup_netif) refers to etharp.o(.bss) for .bss
    etharp.o(i.etharp_find_addr) refers to etharp.o(i.etharp_find_entry) for etharp_find_entry
    etharp.o(i.etharp_find_addr) refers to etharp.o(.bss) for .bss
    etharp.o(i.etharp_find_entry) refers to etharp.o(i.etharp_free_entry) for etharp_free_entry
    etharp.o(i.etharp_find_entry) refers to etharp.o(.bss) for .bss
    etharp.o(i.etharp_free_entry) refers to pbuf.o(i.pbuf_free) for pbuf_free
    etharp.o(i.etharp_free_entry) refers to etharp.o(.bss) for .bss
    etharp.o(i.etharp_free_entry) refers to etharp.o(.constdata) for .constdata
    etharp.o(i.etharp_output) refers to pbuf.o(i.pbuf_header) for pbuf_header
    etharp.o(i.etharp_output) refers to ip_addr.o(i.ip4_addr_isbroadcast) for ip4_addr_isbroadcast
    etharp.o(i.etharp_output) refers to etharp.o(i.etharp_send_ip) for etharp_send_ip
    etharp.o(i.etharp_output) refers to etharp.o(i.etharp_output_to_arp_index) for etharp_output_to_arp_index
    etharp.o(i.etharp_output) refers to etharp.o(i.etharp_query) for etharp_query
    etharp.o(i.etharp_output) refers to etharp.o(.constdata) for .constdata
    etharp.o(i.etharp_output) refers to etharp.o(.data) for .data
    etharp.o(i.etharp_output) refers to etharp.o(.bss) for .bss
    etharp.o(i.etharp_output_to_arp_index) refers to etharp.o(i.etharp_request) for etharp_request
    etharp.o(i.etharp_output_to_arp_index) refers to etharp.o(i.etharp_send_ip) for etharp_send_ip
    etharp.o(i.etharp_output_to_arp_index) refers to etharp.o(.bss) for .bss
    etharp.o(i.etharp_query) refers to ip_addr.o(i.ip4_addr_isbroadcast) for ip4_addr_isbroadcast
    etharp.o(i.etharp_query) refers to etharp.o(i.etharp_find_entry) for etharp_find_entry
    etharp.o(i.etharp_query) refers to etharp.o(i.etharp_request) for etharp_request
    etharp.o(i.etharp_query) refers to etharp.o(i.etharp_send_ip) for etharp_send_ip
    etharp.o(i.etharp_query) refers to pbuf.o(i.pbuf_alloc) for pbuf_alloc
    etharp.o(i.etharp_query) refers to pbuf.o(i.pbuf_copy) for pbuf_copy
    etharp.o(i.etharp_query) refers to pbuf.o(i.pbuf_free) for pbuf_free
    etharp.o(i.etharp_query) refers to pbuf.o(i.pbuf_ref) for pbuf_ref
    etharp.o(i.etharp_query) refers to etharp.o(.bss) for .bss
    etharp.o(i.etharp_query) refers to etharp.o(.data) for .data
    etharp.o(i.etharp_raw) refers to pbuf.o(i.pbuf_alloc) for pbuf_alloc
    etharp.o(i.etharp_raw) refers to def.o(i.lwip_htons) for lwip_htons
    etharp.o(i.etharp_raw) refers to pbuf.o(i.pbuf_free) for pbuf_free
    etharp.o(i.etharp_request) refers to etharp.o(i.etharp_raw) for etharp_raw
    etharp.o(i.etharp_request) refers to etharp.o(.constdata) for .constdata
    etharp.o(i.etharp_tmr) refers to etharp.o(i.etharp_free_entry) for etharp_free_entry
    etharp.o(i.etharp_tmr) refers to etharp.o(.bss) for .bss
    etharp.o(i.etharp_update_arp_entry) refers to ip_addr.o(i.ip4_addr_isbroadcast) for ip4_addr_isbroadcast
    etharp.o(i.etharp_update_arp_entry) refers to etharp.o(i.etharp_find_entry) for etharp_find_entry
    etharp.o(i.etharp_update_arp_entry) refers to etharp.o(i.etharp_send_ip) for etharp_send_ip
    etharp.o(i.etharp_update_arp_entry) refers to pbuf.o(i.pbuf_free) for pbuf_free
    etharp.o(i.etharp_update_arp_entry) refers to etharp.o(.bss) for .bss
    etharp.o(i.ethernet_input) refers to memcmp.o(.text) for memcmp
    etharp.o(i.ethernet_input) refers to pbuf.o(i.pbuf_header) for pbuf_header
    etharp.o(i.ethernet_input) refers to ip.o(i.ip_input) for ip_input
    etharp.o(i.ethernet_input) refers to etharp.o(i.etharp_arp_input) for etharp_arp_input
    etharp.o(i.ethernet_input) refers to pbuf.o(i.pbuf_free) for pbuf_free
    etharp.o(i.ethernet_input) refers to etharp.o(.constdata) for .constdata
    stm32f4xx_hal_flash_ex.o(i.HAL_FLASHEx_Erase) refers to stm32f4xx_hal_flash.o(i.FLASH_WaitForLastOperation) for FLASH_WaitForLastOperation
    stm32f4xx_hal_flash_ex.o(i.HAL_FLASHEx_Erase) refers to stm32f4xx_hal_flash_ex.o(i.FLASH_MassErase) for FLASH_MassErase
    stm32f4xx_hal_flash_ex.o(i.HAL_FLASHEx_Erase) refers to stm32f4xx_hal_flash_ex.o(i.FLASH_Erase_Sector) for FLASH_Erase_Sector
    stm32f4xx_hal_flash_ex.o(i.HAL_FLASHEx_Erase) refers to stm32f4xx_hal_flash_ex.o(i.FLASH_FlushCaches) for FLASH_FlushCaches
    stm32f4xx_hal_flash_ex.o(i.HAL_FLASHEx_Erase) refers to stm32f4xx_hal_flash.o(.bss) for pFlash
    stm32f4xx_hal_flash_ex.o(i.HAL_FLASHEx_Erase_IT) refers to stm32f4xx_hal_flash_ex.o(i.FLASH_Erase_Sector) for FLASH_Erase_Sector
    stm32f4xx_hal_flash_ex.o(i.HAL_FLASHEx_Erase_IT) refers to stm32f4xx_hal_flash_ex.o(i.FLASH_MassErase) for FLASH_MassErase
    stm32f4xx_hal_flash_ex.o(i.HAL_FLASHEx_Erase_IT) refers to stm32f4xx_hal_flash.o(.bss) for pFlash
    stm32f4xx_hal_flash_ex.o(i.HAL_FLASHEx_OBProgram) refers to stm32f4xx_hal_flash.o(i.FLASH_WaitForLastOperation) for FLASH_WaitForLastOperation
    stm32f4xx_hal_flash_ex.o(i.HAL_FLASHEx_OBProgram) refers to stm32f4xx_hal_flash.o(.bss) for pFlash
    stm32f4xx_hal_rcc.o(i.HAL_RCC_ClockConfig) refers to stm32f4xx_hal.o(i.HAL_GetTick) for HAL_GetTick
    stm32f4xx_hal_rcc.o(i.HAL_RCC_ClockConfig) refers to stm32f4xx_hal.o(i.HAL_InitTick) for HAL_InitTick
    stm32f4xx_hal_rcc.o(i.HAL_RCC_GetHCLKFreq) refers to stm32f4xx_hal_rcc.o(i.HAL_RCC_GetSysClockFreq) for HAL_RCC_GetSysClockFreq
    stm32f4xx_hal_rcc.o(i.HAL_RCC_GetHCLKFreq) refers to stm32f4xx_hal_rcc.o(.constdata) for .constdata
    stm32f4xx_hal_rcc.o(i.HAL_RCC_GetHCLKFreq) refers to system_stm32f4xx.o(.data) for SystemCoreClock
    stm32f4xx_hal_rcc.o(i.HAL_RCC_GetPCLK1Freq) refers to stm32f4xx_hal_rcc.o(i.HAL_RCC_GetHCLKFreq) for HAL_RCC_GetHCLKFreq
    stm32f4xx_hal_rcc.o(i.HAL_RCC_GetPCLK1Freq) refers to stm32f4xx_hal_rcc.o(.constdata) for .constdata
    stm32f4xx_hal_rcc.o(i.HAL_RCC_GetPCLK2Freq) refers to stm32f4xx_hal_rcc.o(i.HAL_RCC_GetHCLKFreq) for HAL_RCC_GetHCLKFreq
    stm32f4xx_hal_rcc.o(i.HAL_RCC_GetPCLK2Freq) refers to stm32f4xx_hal_rcc.o(.constdata) for .constdata
    stm32f4xx_hal_rcc.o(i.HAL_RCC_MCOConfig) refers to stm32f4xx_hal_gpio.o(i.HAL_GPIO_Init) for HAL_GPIO_Init
    stm32f4xx_hal_rcc.o(i.HAL_RCC_NMI_IRQHandler) refers to stm32f4xx_hal_rcc.o(i.HAL_RCC_CSSCallback) for HAL_RCC_CSSCallback
    stm32f4xx_hal_rcc.o(i.HAL_RCC_OscConfig) refers to stm32f4xx_hal.o(i.HAL_GetTick) for HAL_GetTick
    stm32f4xx_hal_flash.o(i.FLASH_SetErrorCode) refers to stm32f4xx_hal_flash.o(.bss) for .bss
    stm32f4xx_hal_flash.o(i.FLASH_WaitForLastOperation) refers to stm32f4xx_hal.o(i.HAL_GetTick) for HAL_GetTick
    stm32f4xx_hal_flash.o(i.FLASH_WaitForLastOperation) refers to stm32f4xx_hal_flash.o(i.FLASH_SetErrorCode) for FLASH_SetErrorCode
    stm32f4xx_hal_flash.o(i.FLASH_WaitForLastOperation) refers to stm32f4xx_hal_flash.o(.bss) for .bss
    stm32f4xx_hal_flash.o(i.HAL_FLASH_GetError) refers to stm32f4xx_hal_flash.o(.bss) for .bss
    stm32f4xx_hal_flash.o(i.HAL_FLASH_IRQHandler) refers to stm32f4xx_hal_flash.o(i.FLASH_SetErrorCode) for FLASH_SetErrorCode
    stm32f4xx_hal_flash.o(i.HAL_FLASH_IRQHandler) refers to stm32f4xx_hal_flash.o(i.HAL_FLASH_OperationErrorCallback) for HAL_FLASH_OperationErrorCallback
    stm32f4xx_hal_flash.o(i.HAL_FLASH_IRQHandler) refers to stm32f4xx_hal_flash.o(i.HAL_FLASH_EndOfOperationCallback) for HAL_FLASH_EndOfOperationCallback
    stm32f4xx_hal_flash.o(i.HAL_FLASH_IRQHandler) refers to stm32f4xx_hal_flash_ex.o(i.FLASH_Erase_Sector) for FLASH_Erase_Sector
    stm32f4xx_hal_flash.o(i.HAL_FLASH_IRQHandler) refers to stm32f4xx_hal_flash_ex.o(i.FLASH_FlushCaches) for FLASH_FlushCaches
    stm32f4xx_hal_flash.o(i.HAL_FLASH_IRQHandler) refers to stm32f4xx_hal_flash.o(.bss) for .bss
    stm32f4xx_hal_flash.o(i.HAL_FLASH_OB_Launch) refers to stm32f4xx_hal_flash.o(i.FLASH_WaitForLastOperation) for FLASH_WaitForLastOperation
    stm32f4xx_hal_flash.o(i.HAL_FLASH_Program) refers to stm32f4xx_hal_flash.o(i.FLASH_WaitForLastOperation) for FLASH_WaitForLastOperation
    stm32f4xx_hal_flash.o(i.HAL_FLASH_Program) refers to stm32f4xx_hal_flash.o(i.FLASH_Program_DoubleWord) for FLASH_Program_DoubleWord
    stm32f4xx_hal_flash.o(i.HAL_FLASH_Program) refers to stm32f4xx_hal_flash.o(i.FLASH_Program_Byte) for FLASH_Program_Byte
    stm32f4xx_hal_flash.o(i.HAL_FLASH_Program) refers to stm32f4xx_hal_flash.o(i.FLASH_Program_HalfWord) for FLASH_Program_HalfWord
    stm32f4xx_hal_flash.o(i.HAL_FLASH_Program) refers to stm32f4xx_hal_flash.o(i.FLASH_Program_Word) for FLASH_Program_Word
    stm32f4xx_hal_flash.o(i.HAL_FLASH_Program) refers to stm32f4xx_hal_flash.o(.bss) for .bss
    stm32f4xx_hal_flash.o(i.HAL_FLASH_Program_IT) refers to stm32f4xx_hal_flash.o(i.FLASH_Program_DoubleWord) for FLASH_Program_DoubleWord
    stm32f4xx_hal_flash.o(i.HAL_FLASH_Program_IT) refers to stm32f4xx_hal_flash.o(i.FLASH_Program_Byte) for FLASH_Program_Byte
    stm32f4xx_hal_flash.o(i.HAL_FLASH_Program_IT) refers to stm32f4xx_hal_flash.o(i.FLASH_Program_HalfWord) for FLASH_Program_HalfWord
    stm32f4xx_hal_flash.o(i.HAL_FLASH_Program_IT) refers to stm32f4xx_hal_flash.o(i.FLASH_Program_Word) for FLASH_Program_Word
    stm32f4xx_hal_flash.o(i.HAL_FLASH_Program_IT) refers to stm32f4xx_hal_flash.o(.bss) for .bss
    stm32f4xx_hal.o(i.HAL_DeInit) refers to stm32f4xx_hal.o(i.HAL_MspDeInit) for HAL_MspDeInit
    stm32f4xx_hal.o(i.HAL_Delay) refers to stm32f4xx_hal.o(i.HAL_GetTick) for HAL_GetTick
    stm32f4xx_hal.o(i.HAL_GetTick) refers to stm32f4xx_hal.o(.data) for .data
    stm32f4xx_hal.o(i.HAL_IncTick) refers to stm32f4xx_hal.o(.data) for .data
    stm32f4xx_hal.o(i.HAL_Init) refers to stm32f4xx_hal_cortex.o(i.HAL_NVIC_SetPriorityGrouping) for HAL_NVIC_SetPriorityGrouping
    stm32f4xx_hal.o(i.HAL_Init) refers to stm32f4xx_hal.o(i.HAL_InitTick) for HAL_InitTick
    stm32f4xx_hal.o(i.HAL_Init) refers to stm32f4xx_hal.o(i.HAL_MspInit) for HAL_MspInit
    stm32f4xx_hal.o(i.HAL_InitTick) refers to stm32f4xx_hal_rcc.o(i.HAL_RCC_GetHCLKFreq) for HAL_RCC_GetHCLKFreq
    stm32f4xx_hal.o(i.HAL_InitTick) refers to stm32f4xx_hal_cortex.o(i.HAL_SYSTICK_Config) for HAL_SYSTICK_Config
    stm32f4xx_hal.o(i.HAL_InitTick) refers to stm32f4xx_hal_cortex.o(i.HAL_NVIC_SetPriority) for HAL_NVIC_SetPriority
    stm32f4xx_hal_gpio.o(i.HAL_GPIO_EXTI_IRQHandler) refers to stm32f4xx_hal_gpio.o(i.HAL_GPIO_EXTI_Callback) for HAL_GPIO_EXTI_Callback
    stm32f4xx_hal_pwr.o(i.HAL_PWR_PVD_IRQHandler) refers to stm32f4xx_hal_pwr.o(i.HAL_PWR_PVDCallback) for HAL_PWR_PVDCallback
    stm32f4xx_hal_sram.o(i.HAL_SRAM_DeInit) refers to stm32f4xx_hal_sram.o(i.HAL_SRAM_MspDeInit) for HAL_SRAM_MspDeInit
    stm32f4xx_hal_sram.o(i.HAL_SRAM_DeInit) refers to stm32f4xx_ll_fsmc.o(i.FSMC_NORSRAM_DeInit) for FSMC_NORSRAM_DeInit
    stm32f4xx_hal_sram.o(i.HAL_SRAM_Init) refers to stm32f4xx_hal_sram.o(i.HAL_SRAM_MspInit) for HAL_SRAM_MspInit
    stm32f4xx_hal_sram.o(i.HAL_SRAM_Init) refers to stm32f4xx_ll_fsmc.o(i.FSMC_NORSRAM_Init) for FSMC_NORSRAM_Init
    stm32f4xx_hal_sram.o(i.HAL_SRAM_Init) refers to stm32f4xx_ll_fsmc.o(i.FSMC_NORSRAM_Timing_Init) for FSMC_NORSRAM_Timing_Init
    stm32f4xx_hal_sram.o(i.HAL_SRAM_Init) refers to stm32f4xx_ll_fsmc.o(i.FSMC_NORSRAM_Extended_Timing_Init) for FSMC_NORSRAM_Extended_Timing_Init
    stm32f4xx_hal_sram.o(i.HAL_SRAM_Read_DMA) refers to stm32f4xx_hal_dma.o(i.HAL_DMA_Start_IT) for HAL_DMA_Start_IT
    stm32f4xx_hal_sram.o(i.HAL_SRAM_Read_DMA) refers to stm32f4xx_hal_sram.o(i.HAL_SRAM_DMA_XferCpltCallback) for HAL_SRAM_DMA_XferCpltCallback
    stm32f4xx_hal_sram.o(i.HAL_SRAM_Read_DMA) refers to stm32f4xx_hal_sram.o(i.HAL_SRAM_DMA_XferErrorCallback) for HAL_SRAM_DMA_XferErrorCallback
    stm32f4xx_hal_sram.o(i.HAL_SRAM_WriteOperation_Disable) refers to stm32f4xx_ll_fsmc.o(i.FSMC_NORSRAM_WriteOperation_Disable) for FSMC_NORSRAM_WriteOperation_Disable
    stm32f4xx_hal_sram.o(i.HAL_SRAM_WriteOperation_Enable) refers to stm32f4xx_ll_fsmc.o(i.FSMC_NORSRAM_WriteOperation_Enable) for FSMC_NORSRAM_WriteOperation_Enable
    stm32f4xx_hal_sram.o(i.HAL_SRAM_Write_DMA) refers to stm32f4xx_hal_dma.o(i.HAL_DMA_Start_IT) for HAL_DMA_Start_IT
    stm32f4xx_hal_sram.o(i.HAL_SRAM_Write_DMA) refers to stm32f4xx_hal_sram.o(i.HAL_SRAM_DMA_XferCpltCallback) for HAL_SRAM_DMA_XferCpltCallback
    stm32f4xx_hal_sram.o(i.HAL_SRAM_Write_DMA) refers to stm32f4xx_hal_sram.o(i.HAL_SRAM_DMA_XferErrorCallback) for HAL_SRAM_DMA_XferErrorCallback
    stm32f4xx_ll_fsmc.o(i.FSMC_NAND_GetECC) refers to stm32f4xx_hal.o(i.HAL_GetTick) for HAL_GetTick
    stm32f4xx_hal_cortex.o(i.HAL_NVIC_SetPriority) refers to stm32f4xx_hal_cortex.o(i.NVIC_SetPriority) for NVIC_SetPriority
    stm32f4xx_hal_cortex.o(i.HAL_SYSTICK_Config) refers to stm32f4xx_hal_cortex.o(i.NVIC_SetPriority) for NVIC_SetPriority
    stm32f4xx_hal_cortex.o(i.HAL_SYSTICK_IRQHandler) refers to stm32f4xx_hal_cortex.o(i.HAL_SYSTICK_Callback) for HAL_SYSTICK_Callback
    stm32f4xx_hal_uart.o(i.HAL_HalfDuplex_Init) refers to stm32f4xx_hal_uart.o(i.HAL_UART_MspInit) for HAL_UART_MspInit
    stm32f4xx_hal_uart.o(i.HAL_HalfDuplex_Init) refers to stm32f4xx_hal_uart.o(i.UART_SetConfig) for UART_SetConfig
    stm32f4xx_hal_uart.o(i.HAL_LIN_Init) refers to stm32f4xx_hal_uart.o(i.HAL_UART_MspInit) for HAL_UART_MspInit
    stm32f4xx_hal_uart.o(i.HAL_LIN_Init) refers to stm32f4xx_hal_uart.o(i.UART_SetConfig) for UART_SetConfig
    stm32f4xx_hal_uart.o(i.HAL_MultiProcessor_Init) refers to stm32f4xx_hal_uart.o(i.HAL_UART_MspInit) for HAL_UART_MspInit
    stm32f4xx_hal_uart.o(i.HAL_MultiProcessor_Init) refers to stm32f4xx_hal_uart.o(i.UART_SetConfig) for UART_SetConfig
    stm32f4xx_hal_uart.o(i.HAL_UART_DMAStop) refers to stm32f4xx_hal_dma.o(i.HAL_DMA_Abort) for HAL_DMA_Abort
    stm32f4xx_hal_uart.o(i.HAL_UART_DeInit) refers to stm32f4xx_hal_uart.o(i.HAL_UART_MspDeInit) for HAL_UART_MspDeInit
    stm32f4xx_hal_uart.o(i.HAL_UART_IRQHandler) refers to stm32f4xx_hal_uart.o(i.UART_Receive_IT) for UART_Receive_IT
    stm32f4xx_hal_uart.o(i.HAL_UART_IRQHandler) refers to stm32f4xx_hal_uart.o(i.UART_Transmit_IT) for UART_Transmit_IT
    stm32f4xx_hal_uart.o(i.HAL_UART_IRQHandler) refers to stm32f4xx_hal_uart.o(i.HAL_UART_TxCpltCallback) for HAL_UART_TxCpltCallback
    stm32f4xx_hal_uart.o(i.HAL_UART_IRQHandler) refers to stm32f4xx_hal_uart.o(i.HAL_UART_ErrorCallback) for HAL_UART_ErrorCallback
    stm32f4xx_hal_uart.o(i.HAL_UART_Init) refers to stm32f4xx_hal_uart.o(i.HAL_UART_MspInit) for HAL_UART_MspInit
    stm32f4xx_hal_uart.o(i.HAL_UART_Init) refers to stm32f4xx_hal_uart.o(i.UART_SetConfig) for UART_SetConfig
    stm32f4xx_hal_uart.o(i.HAL_UART_Receive) refers to stm32f4xx_hal_uart.o(i.UART_WaitOnFlagUntilTimeout) for UART_WaitOnFlagUntilTimeout
    stm32f4xx_hal_uart.o(i.HAL_UART_Receive_DMA) refers to stm32f4xx_hal_dma.o(i.HAL_DMA_Start_IT) for HAL_DMA_Start_IT
    stm32f4xx_hal_uart.o(i.HAL_UART_Receive_DMA) refers to stm32f4xx_hal_uart.o(i.UART_DMAReceiveCplt) for UART_DMAReceiveCplt
    stm32f4xx_hal_uart.o(i.HAL_UART_Receive_DMA) refers to stm32f4xx_hal_uart.o(i.UART_DMARxHalfCplt) for UART_DMARxHalfCplt
    stm32f4xx_hal_uart.o(i.HAL_UART_Receive_DMA) refers to stm32f4xx_hal_uart.o(i.UART_DMAError) for UART_DMAError
    stm32f4xx_hal_uart.o(i.HAL_UART_Transmit) refers to stm32f4xx_hal_uart.o(i.UART_WaitOnFlagUntilTimeout) for UART_WaitOnFlagUntilTimeout
    stm32f4xx_hal_uart.o(i.HAL_UART_Transmit_DMA) refers to stm32f4xx_hal_dma.o(i.HAL_DMA_Start_IT) for HAL_DMA_Start_IT
    stm32f4xx_hal_uart.o(i.HAL_UART_Transmit_DMA) refers to stm32f4xx_hal_uart.o(i.UART_DMATransmitCplt) for UART_DMATransmitCplt
    stm32f4xx_hal_uart.o(i.HAL_UART_Transmit_DMA) refers to stm32f4xx_hal_uart.o(i.UART_DMATxHalfCplt) for UART_DMATxHalfCplt
    stm32f4xx_hal_uart.o(i.HAL_UART_Transmit_DMA) refers to stm32f4xx_hal_uart.o(i.UART_DMAError) for UART_DMAError
    stm32f4xx_hal_uart.o(i.UART_DMAError) refers to stm32f4xx_hal_uart.o(i.HAL_UART_ErrorCallback) for HAL_UART_ErrorCallback
    stm32f4xx_hal_uart.o(i.UART_DMAReceiveCplt) refers to stm32f4xx_hal_uart.o(i.HAL_UART_RxCpltCallback) for HAL_UART_RxCpltCallback
    stm32f4xx_hal_uart.o(i.UART_DMARxHalfCplt) refers to stm32f4xx_hal_uart.o(i.HAL_UART_RxHalfCpltCallback) for HAL_UART_RxHalfCpltCallback
    stm32f4xx_hal_uart.o(i.UART_DMATransmitCplt) refers to stm32f4xx_hal_uart.o(i.HAL_UART_TxCpltCallback) for HAL_UART_TxCpltCallback
    stm32f4xx_hal_uart.o(i.UART_DMATxHalfCplt) refers to stm32f4xx_hal_uart.o(i.HAL_UART_TxHalfCpltCallback) for HAL_UART_TxHalfCpltCallback
    stm32f4xx_hal_uart.o(i.UART_Receive_IT) refers to stm32f4xx_hal_uart.o(i.HAL_UART_RxCpltCallback) for HAL_UART_RxCpltCallback
    stm32f4xx_hal_uart.o(i.UART_SetConfig) refers to stm32f4xx_hal_rcc.o(i.HAL_RCC_GetPCLK2Freq) for HAL_RCC_GetPCLK2Freq
    stm32f4xx_hal_uart.o(i.UART_SetConfig) refers to stm32f4xx_hal_rcc.o(i.HAL_RCC_GetPCLK1Freq) for HAL_RCC_GetPCLK1Freq
    stm32f4xx_hal_uart.o(i.UART_WaitOnFlagUntilTimeout) refers to stm32f4xx_hal.o(i.HAL_GetTick) for HAL_GetTick
    stm32f4xx_hal_i2c.o(i.HAL_I2C_DeInit) refers to stm32f4xx_hal_i2c.o(i.HAL_I2C_MspDeInit) for HAL_I2C_MspDeInit
    stm32f4xx_hal_i2c.o(i.HAL_I2C_ER_IRQHandler) refers to stm32f4xx_hal_i2c.o(i.HAL_I2C_ErrorCallback) for HAL_I2C_ErrorCallback
    stm32f4xx_hal_i2c.o(i.HAL_I2C_ER_IRQHandler) refers to stm32f4xx_hal_i2c.o(i.HAL_I2C_ListenCpltCallback) for HAL_I2C_ListenCpltCallback
    stm32f4xx_hal_i2c.o(i.HAL_I2C_ER_IRQHandler) refers to stm32f4xx_hal_i2c.o(i.I2C_Slave_AF) for I2C_Slave_AF
    stm32f4xx_hal_i2c.o(i.HAL_I2C_EV_IRQHandler) refers to stm32f4xx_hal_i2c.o(i.I2C_MasterTransmit_BTF) for I2C_MasterTransmit_BTF
    stm32f4xx_hal_i2c.o(i.HAL_I2C_EV_IRQHandler) refers to stm32f4xx_hal_i2c.o(i.I2C_MasterReceive_BTF) for I2C_MasterReceive_BTF
    stm32f4xx_hal_i2c.o(i.HAL_I2C_EV_IRQHandler) refers to stm32f4xx_hal_i2c.o(i.I2C_MasterReceive_RXNE) for I2C_MasterReceive_RXNE
    stm32f4xx_hal_i2c.o(i.HAL_I2C_EV_IRQHandler) refers to stm32f4xx_hal_i2c.o(i.HAL_I2C_AddrCallback) for HAL_I2C_AddrCallback
    stm32f4xx_hal_i2c.o(i.HAL_I2C_EV_IRQHandler) refers to stm32f4xx_hal_i2c.o(i.I2C_Slave_STOPF) for I2C_Slave_STOPF
    stm32f4xx_hal_i2c.o(i.HAL_I2C_EV_IRQHandler) refers to stm32f4xx_hal_i2c.o(i.HAL_I2C_SlaveTxCpltCallback) for HAL_I2C_SlaveTxCpltCallback
    stm32f4xx_hal_i2c.o(i.HAL_I2C_EV_IRQHandler) refers to stm32f4xx_hal_i2c.o(i.HAL_I2C_SlaveRxCpltCallback) for HAL_I2C_SlaveRxCpltCallback
    stm32f4xx_hal_i2c.o(i.HAL_I2C_Init) refers to stm32f4xx_hal_i2c.o(i.HAL_I2C_MspInit) for HAL_I2C_MspInit
    stm32f4xx_hal_i2c.o(i.HAL_I2C_Init) refers to stm32f4xx_hal_rcc.o(i.HAL_RCC_GetPCLK1Freq) for HAL_RCC_GetPCLK1Freq
    stm32f4xx_hal_i2c.o(i.HAL_I2C_IsDeviceReady) refers to stm32f4xx_hal_i2c.o(i.I2C_WaitOnFlagUntilTimeout) for I2C_WaitOnFlagUntilTimeout
    stm32f4xx_hal_i2c.o(i.HAL_I2C_IsDeviceReady) refers to stm32f4xx_hal.o(i.HAL_GetTick) for HAL_GetTick
    stm32f4xx_hal_i2c.o(i.HAL_I2C_Master_Receive) refers to stm32f4xx_hal_i2c.o(i.I2C_WaitOnFlagUntilTimeout) for I2C_WaitOnFlagUntilTimeout
    stm32f4xx_hal_i2c.o(i.HAL_I2C_Master_Receive) refers to stm32f4xx_hal_i2c.o(i.I2C_MasterRequestRead) for I2C_MasterRequestRead
    stm32f4xx_hal_i2c.o(i.HAL_I2C_Master_Receive) refers to stm32f4xx_hal_i2c.o(i.I2C_WaitOnRXNEFlagUntilTimeout) for I2C_WaitOnRXNEFlagUntilTimeout
    stm32f4xx_hal_i2c.o(i.HAL_I2C_Master_Receive_DMA) refers to stm32f4xx_hal_i2c.o(i.I2C_WaitOnFlagUntilTimeout) for I2C_WaitOnFlagUntilTimeout
    stm32f4xx_hal_i2c.o(i.HAL_I2C_Master_Receive_DMA) refers to stm32f4xx_hal_dma.o(i.HAL_DMA_Start_IT) for HAL_DMA_Start_IT
    stm32f4xx_hal_i2c.o(i.HAL_I2C_Master_Receive_DMA) refers to stm32f4xx_hal_i2c.o(i.I2C_MasterRequestRead) for I2C_MasterRequestRead
    stm32f4xx_hal_i2c.o(i.HAL_I2C_Master_Receive_DMA) refers to stm32f4xx_hal_i2c.o(i.I2C_DMAMasterReceiveCplt) for I2C_DMAMasterReceiveCplt
    stm32f4xx_hal_i2c.o(i.HAL_I2C_Master_Receive_DMA) refers to stm32f4xx_hal_i2c.o(i.I2C_DMAError) for I2C_DMAError
    stm32f4xx_hal_i2c.o(i.HAL_I2C_Master_Receive_IT) refers to stm32f4xx_hal_i2c.o(i.I2C_WaitOnFlagUntilTimeout) for I2C_WaitOnFlagUntilTimeout
    stm32f4xx_hal_i2c.o(i.HAL_I2C_Master_Receive_IT) refers to stm32f4xx_hal_i2c.o(i.I2C_MasterRequestRead) for I2C_MasterRequestRead
    stm32f4xx_hal_i2c.o(i.HAL_I2C_Master_Sequential_Receive_IT) refers to stm32f4xx_hal_i2c.o(i.I2C_WaitOnFlagUntilTimeout) for I2C_WaitOnFlagUntilTimeout
    stm32f4xx_hal_i2c.o(i.HAL_I2C_Master_Sequential_Receive_IT) refers to stm32f4xx_hal_i2c.o(i.I2C_MasterRequestRead) for I2C_MasterRequestRead
    stm32f4xx_hal_i2c.o(i.HAL_I2C_Master_Sequential_Transmit_IT) refers to stm32f4xx_hal_i2c.o(i.I2C_WaitOnFlagUntilTimeout) for I2C_WaitOnFlagUntilTimeout
    stm32f4xx_hal_i2c.o(i.HAL_I2C_Master_Sequential_Transmit_IT) refers to stm32f4xx_hal_i2c.o(i.I2C_MasterRequestWrite) for I2C_MasterRequestWrite
    stm32f4xx_hal_i2c.o(i.HAL_I2C_Master_Transmit) refers to stm32f4xx_hal_i2c.o(i.I2C_WaitOnFlagUntilTimeout) for I2C_WaitOnFlagUntilTimeout
    stm32f4xx_hal_i2c.o(i.HAL_I2C_Master_Transmit) refers to stm32f4xx_hal_i2c.o(i.I2C_MasterRequestWrite) for I2C_MasterRequestWrite
    stm32f4xx_hal_i2c.o(i.HAL_I2C_Master_Transmit) refers to stm32f4xx_hal_i2c.o(i.I2C_WaitOnTXEFlagUntilTimeout) for I2C_WaitOnTXEFlagUntilTimeout
    stm32f4xx_hal_i2c.o(i.HAL_I2C_Master_Transmit) refers to stm32f4xx_hal.o(i.HAL_GetTick) for HAL_GetTick
    stm32f4xx_hal_i2c.o(i.HAL_I2C_Master_Transmit) refers to stm32f4xx_hal_i2c.o(i.I2C_IsAcknowledgeFailed) for I2C_IsAcknowledgeFailed
    stm32f4xx_hal_i2c.o(i.HAL_I2C_Master_Transmit_DMA) refers to stm32f4xx_hal_i2c.o(i.I2C_WaitOnFlagUntilTimeout) for I2C_WaitOnFlagUntilTimeout
    stm32f4xx_hal_i2c.o(i.HAL_I2C_Master_Transmit_DMA) refers to stm32f4xx_hal_dma.o(i.HAL_DMA_Start_IT) for HAL_DMA_Start_IT
    stm32f4xx_hal_i2c.o(i.HAL_I2C_Master_Transmit_DMA) refers to stm32f4xx_hal_i2c.o(i.I2C_MasterRequestWrite) for I2C_MasterRequestWrite
    stm32f4xx_hal_i2c.o(i.HAL_I2C_Master_Transmit_DMA) refers to stm32f4xx_hal_i2c.o(i.I2C_DMAMasterTransmitCplt) for I2C_DMAMasterTransmitCplt
    stm32f4xx_hal_i2c.o(i.HAL_I2C_Master_Transmit_DMA) refers to stm32f4xx_hal_i2c.o(i.I2C_DMAError) for I2C_DMAError
    stm32f4xx_hal_i2c.o(i.HAL_I2C_Master_Transmit_IT) refers to stm32f4xx_hal_i2c.o(i.I2C_WaitOnFlagUntilTimeout) for I2C_WaitOnFlagUntilTimeout
    stm32f4xx_hal_i2c.o(i.HAL_I2C_Master_Transmit_IT) refers to stm32f4xx_hal_i2c.o(i.I2C_MasterRequestWrite) for I2C_MasterRequestWrite
    stm32f4xx_hal_i2c.o(i.HAL_I2C_Mem_Read) refers to stm32f4xx_hal_i2c.o(i.I2C_WaitOnFlagUntilTimeout) for I2C_WaitOnFlagUntilTimeout
    stm32f4xx_hal_i2c.o(i.HAL_I2C_Mem_Read) refers to stm32f4xx_hal_i2c.o(i.I2C_RequestMemoryRead) for I2C_RequestMemoryRead
    stm32f4xx_hal_i2c.o(i.HAL_I2C_Mem_Read) refers to stm32f4xx_hal_i2c.o(i.I2C_WaitOnRXNEFlagUntilTimeout) for I2C_WaitOnRXNEFlagUntilTimeout
    stm32f4xx_hal_i2c.o(i.HAL_I2C_Mem_Read_DMA) refers to stm32f4xx_hal_i2c.o(i.I2C_WaitOnFlagUntilTimeout) for I2C_WaitOnFlagUntilTimeout
    stm32f4xx_hal_i2c.o(i.HAL_I2C_Mem_Read_DMA) refers to stm32f4xx_hal_dma.o(i.HAL_DMA_Start_IT) for HAL_DMA_Start_IT
    stm32f4xx_hal_i2c.o(i.HAL_I2C_Mem_Read_DMA) refers to stm32f4xx_hal_i2c.o(i.I2C_RequestMemoryRead) for I2C_RequestMemoryRead
    stm32f4xx_hal_i2c.o(i.HAL_I2C_Mem_Read_DMA) refers to stm32f4xx_hal_i2c.o(i.I2C_DMAMemReceiveCplt) for I2C_DMAMemReceiveCplt
    stm32f4xx_hal_i2c.o(i.HAL_I2C_Mem_Read_DMA) refers to stm32f4xx_hal_i2c.o(i.I2C_DMAError) for I2C_DMAError
    stm32f4xx_hal_i2c.o(i.HAL_I2C_Mem_Read_IT) refers to stm32f4xx_hal_i2c.o(i.I2C_WaitOnFlagUntilTimeout) for I2C_WaitOnFlagUntilTimeout
    stm32f4xx_hal_i2c.o(i.HAL_I2C_Mem_Read_IT) refers to stm32f4xx_hal_i2c.o(i.I2C_RequestMemoryRead) for I2C_RequestMemoryRead
    stm32f4xx_hal_i2c.o(i.HAL_I2C_Mem_Write) refers to stm32f4xx_hal_i2c.o(i.I2C_WaitOnFlagUntilTimeout) for I2C_WaitOnFlagUntilTimeout
    stm32f4xx_hal_i2c.o(i.HAL_I2C_Mem_Write) refers to stm32f4xx_hal_i2c.o(i.I2C_RequestMemoryWrite) for I2C_RequestMemoryWrite
    stm32f4xx_hal_i2c.o(i.HAL_I2C_Mem_Write) refers to stm32f4xx_hal_i2c.o(i.I2C_WaitOnTXEFlagUntilTimeout) for I2C_WaitOnTXEFlagUntilTimeout
    stm32f4xx_hal_i2c.o(i.HAL_I2C_Mem_Write_DMA) refers to stm32f4xx_hal_i2c.o(i.I2C_WaitOnFlagUntilTimeout) for I2C_WaitOnFlagUntilTimeout
    stm32f4xx_hal_i2c.o(i.HAL_I2C_Mem_Write_DMA) refers to stm32f4xx_hal_dma.o(i.HAL_DMA_Start_IT) for HAL_DMA_Start_IT
    stm32f4xx_hal_i2c.o(i.HAL_I2C_Mem_Write_DMA) refers to stm32f4xx_hal_i2c.o(i.I2C_RequestMemoryWrite) for I2C_RequestMemoryWrite
    stm32f4xx_hal_i2c.o(i.HAL_I2C_Mem_Write_DMA) refers to stm32f4xx_hal_i2c.o(i.I2C_RequestMemoryRead) for I2C_RequestMemoryRead
    stm32f4xx_hal_i2c.o(i.HAL_I2C_Mem_Write_DMA) refers to stm32f4xx_hal_i2c.o(i.I2C_DMAMemTransmitCplt) for I2C_DMAMemTransmitCplt
    stm32f4xx_hal_i2c.o(i.HAL_I2C_Mem_Write_DMA) refers to stm32f4xx_hal_i2c.o(i.I2C_DMAError) for I2C_DMAError
    stm32f4xx_hal_i2c.o(i.HAL_I2C_Mem_Write_IT) refers to stm32f4xx_hal_i2c.o(i.I2C_WaitOnFlagUntilTimeout) for I2C_WaitOnFlagUntilTimeout
    stm32f4xx_hal_i2c.o(i.HAL_I2C_Mem_Write_IT) refers to stm32f4xx_hal_i2c.o(i.I2C_RequestMemoryWrite) for I2C_RequestMemoryWrite
    stm32f4xx_hal_i2c.o(i.HAL_I2C_Slave_Receive) refers to stm32f4xx_hal_i2c.o(i.I2C_WaitOnFlagUntilTimeout) for I2C_WaitOnFlagUntilTimeout
    stm32f4xx_hal_i2c.o(i.HAL_I2C_Slave_Receive) refers to stm32f4xx_hal_i2c.o(i.I2C_WaitOnRXNEFlagUntilTimeout) for I2C_WaitOnRXNEFlagUntilTimeout
    stm32f4xx_hal_i2c.o(i.HAL_I2C_Slave_Receive) refers to stm32f4xx_hal_i2c.o(i.I2C_WaitOnSTOPFlagUntilTimeout) for I2C_WaitOnSTOPFlagUntilTimeout
    stm32f4xx_hal_i2c.o(i.HAL_I2C_Slave_Receive_DMA) refers to stm32f4xx_hal_i2c.o(i.I2C_WaitOnFlagUntilTimeout) for I2C_WaitOnFlagUntilTimeout
    stm32f4xx_hal_i2c.o(i.HAL_I2C_Slave_Receive_DMA) refers to stm32f4xx_hal_dma.o(i.HAL_DMA_Start_IT) for HAL_DMA_Start_IT
    stm32f4xx_hal_i2c.o(i.HAL_I2C_Slave_Receive_DMA) refers to stm32f4xx_hal_i2c.o(i.I2C_DMASlaveReceiveCplt) for I2C_DMASlaveReceiveCplt
    stm32f4xx_hal_i2c.o(i.HAL_I2C_Slave_Receive_DMA) refers to stm32f4xx_hal_i2c.o(i.I2C_DMAError) for I2C_DMAError
    stm32f4xx_hal_i2c.o(i.HAL_I2C_Slave_Receive_IT) refers to stm32f4xx_hal_i2c.o(i.I2C_WaitOnFlagUntilTimeout) for I2C_WaitOnFlagUntilTimeout
    stm32f4xx_hal_i2c.o(i.HAL_I2C_Slave_Transmit) refers to stm32f4xx_hal_i2c.o(i.I2C_WaitOnFlagUntilTimeout) for I2C_WaitOnFlagUntilTimeout
    stm32f4xx_hal_i2c.o(i.HAL_I2C_Slave_Transmit) refers to stm32f4xx_hal_i2c.o(i.I2C_WaitOnTXEFlagUntilTimeout) for I2C_WaitOnTXEFlagUntilTimeout
    stm32f4xx_hal_i2c.o(i.HAL_I2C_Slave_Transmit_DMA) refers to stm32f4xx_hal_i2c.o(i.I2C_WaitOnFlagUntilTimeout) for I2C_WaitOnFlagUntilTimeout
    stm32f4xx_hal_i2c.o(i.HAL_I2C_Slave_Transmit_DMA) refers to stm32f4xx_hal_dma.o(i.HAL_DMA_Start_IT) for HAL_DMA_Start_IT
    stm32f4xx_hal_i2c.o(i.HAL_I2C_Slave_Transmit_DMA) refers to stm32f4xx_hal_i2c.o(i.I2C_DMASlaveTransmitCplt) for I2C_DMASlaveTransmitCplt
    stm32f4xx_hal_i2c.o(i.HAL_I2C_Slave_Transmit_DMA) refers to stm32f4xx_hal_i2c.o(i.I2C_DMAError) for I2C_DMAError
    stm32f4xx_hal_i2c.o(i.HAL_I2C_Slave_Transmit_IT) refers to stm32f4xx_hal_i2c.o(i.I2C_WaitOnFlagUntilTimeout) for I2C_WaitOnFlagUntilTimeout
    stm32f4xx_hal_i2c.o(i.I2C_DMAError) refers to stm32f4xx_hal_i2c.o(i.HAL_I2C_ErrorCallback) for HAL_I2C_ErrorCallback
    stm32f4xx_hal_i2c.o(i.I2C_DMAMasterReceiveCplt) refers to stm32f4xx_hal_i2c.o(i.HAL_I2C_ErrorCallback) for HAL_I2C_ErrorCallback
    stm32f4xx_hal_i2c.o(i.I2C_DMAMasterReceiveCplt) refers to stm32f4xx_hal_i2c.o(i.HAL_I2C_MasterRxCpltCallback) for HAL_I2C_MasterRxCpltCallback
    stm32f4xx_hal_i2c.o(i.I2C_DMAMasterTransmitCplt) refers to stm32f4xx_hal_i2c.o(i.I2C_WaitOnFlagUntilTimeout) for I2C_WaitOnFlagUntilTimeout
    stm32f4xx_hal_i2c.o(i.I2C_DMAMasterTransmitCplt) refers to stm32f4xx_hal_i2c.o(i.HAL_I2C_ErrorCallback) for HAL_I2C_ErrorCallback
    stm32f4xx_hal_i2c.o(i.I2C_DMAMasterTransmitCplt) refers to stm32f4xx_hal_i2c.o(i.HAL_I2C_MasterTxCpltCallback) for HAL_I2C_MasterTxCpltCallback
    stm32f4xx_hal_i2c.o(i.I2C_DMAMemReceiveCplt) refers to stm32f4xx_hal_i2c.o(i.HAL_I2C_ErrorCallback) for HAL_I2C_ErrorCallback
    stm32f4xx_hal_i2c.o(i.I2C_DMAMemReceiveCplt) refers to stm32f4xx_hal_i2c.o(i.HAL_I2C_MemRxCpltCallback) for HAL_I2C_MemRxCpltCallback
    stm32f4xx_hal_i2c.o(i.I2C_DMAMemTransmitCplt) refers to stm32f4xx_hal_i2c.o(i.I2C_WaitOnFlagUntilTimeout) for I2C_WaitOnFlagUntilTimeout
    stm32f4xx_hal_i2c.o(i.I2C_DMAMemTransmitCplt) refers to stm32f4xx_hal_i2c.o(i.HAL_I2C_ErrorCallback) for HAL_I2C_ErrorCallback
    stm32f4xx_hal_i2c.o(i.I2C_DMAMemTransmitCplt) refers to stm32f4xx_hal_i2c.o(i.HAL_I2C_MemTxCpltCallback) for HAL_I2C_MemTxCpltCallback
    stm32f4xx_hal_i2c.o(i.I2C_DMASlaveReceiveCplt) refers to stm32f4xx_hal_i2c.o(i.I2C_WaitOnSTOPFlagUntilTimeout) for I2C_WaitOnSTOPFlagUntilTimeout
    stm32f4xx_hal_i2c.o(i.I2C_DMASlaveReceiveCplt) refers to stm32f4xx_hal_i2c.o(i.HAL_I2C_ErrorCallback) for HAL_I2C_ErrorCallback
    stm32f4xx_hal_i2c.o(i.I2C_DMASlaveReceiveCplt) refers to stm32f4xx_hal_i2c.o(i.HAL_I2C_SlaveRxCpltCallback) for HAL_I2C_SlaveRxCpltCallback
    stm32f4xx_hal_i2c.o(i.I2C_DMASlaveTransmitCplt) refers to stm32f4xx_hal_i2c.o(i.I2C_WaitOnFlagUntilTimeout) for I2C_WaitOnFlagUntilTimeout
    stm32f4xx_hal_i2c.o(i.I2C_DMASlaveTransmitCplt) refers to stm32f4xx_hal_i2c.o(i.HAL_I2C_ErrorCallback) for HAL_I2C_ErrorCallback
    stm32f4xx_hal_i2c.o(i.I2C_DMASlaveTransmitCplt) refers to stm32f4xx_hal_i2c.o(i.HAL_I2C_SlaveTxCpltCallback) for HAL_I2C_SlaveTxCpltCallback
    stm32f4xx_hal_i2c.o(i.I2C_MasterReceive_BTF) refers to stm32f4xx_hal_i2c.o(i.HAL_I2C_MasterRxCpltCallback) for HAL_I2C_MasterRxCpltCallback
    stm32f4xx_hal_i2c.o(i.I2C_MasterReceive_BTF) refers to stm32f4xx_hal_i2c.o(i.HAL_I2C_MemRxCpltCallback) for HAL_I2C_MemRxCpltCallback
    stm32f4xx_hal_i2c.o(i.I2C_MasterReceive_RXNE) refers to stm32f4xx_hal_i2c.o(i.HAL_I2C_MasterRxCpltCallback) for HAL_I2C_MasterRxCpltCallback
    stm32f4xx_hal_i2c.o(i.I2C_MasterReceive_RXNE) refers to stm32f4xx_hal_i2c.o(i.HAL_I2C_MemRxCpltCallback) for HAL_I2C_MemRxCpltCallback
    stm32f4xx_hal_i2c.o(i.I2C_MasterRequestRead) refers to stm32f4xx_hal_i2c.o(i.I2C_WaitOnFlagUntilTimeout) for I2C_WaitOnFlagUntilTimeout
    stm32f4xx_hal_i2c.o(i.I2C_MasterRequestRead) refers to stm32f4xx_hal_i2c.o(i.I2C_WaitOnMasterAddressFlagUntilTimeout) for I2C_WaitOnMasterAddressFlagUntilTimeout
    stm32f4xx_hal_i2c.o(i.I2C_MasterRequestWrite) refers to stm32f4xx_hal_i2c.o(i.I2C_WaitOnFlagUntilTimeout) for I2C_WaitOnFlagUntilTimeout
    stm32f4xx_hal_i2c.o(i.I2C_MasterRequestWrite) refers to stm32f4xx_hal_i2c.o(i.I2C_WaitOnMasterAddressFlagUntilTimeout) for I2C_WaitOnMasterAddressFlagUntilTimeout
    stm32f4xx_hal_i2c.o(i.I2C_MasterTransmit_BTF) refers to stm32f4xx_hal_i2c.o(i.HAL_I2C_MasterTxCpltCallback) for HAL_I2C_MasterTxCpltCallback
    stm32f4xx_hal_i2c.o(i.I2C_MasterTransmit_BTF) refers to stm32f4xx_hal_i2c.o(i.HAL_I2C_MemTxCpltCallback) for HAL_I2C_MemTxCpltCallback
    stm32f4xx_hal_i2c.o(i.I2C_RequestMemoryRead) refers to stm32f4xx_hal_i2c.o(i.I2C_WaitOnFlagUntilTimeout) for I2C_WaitOnFlagUntilTimeout
    stm32f4xx_hal_i2c.o(i.I2C_RequestMemoryRead) refers to stm32f4xx_hal_i2c.o(i.I2C_WaitOnMasterAddressFlagUntilTimeout) for I2C_WaitOnMasterAddressFlagUntilTimeout
    stm32f4xx_hal_i2c.o(i.I2C_RequestMemoryRead) refers to stm32f4xx_hal_i2c.o(i.I2C_WaitOnTXEFlagUntilTimeout) for I2C_WaitOnTXEFlagUntilTimeout
    stm32f4xx_hal_i2c.o(i.I2C_RequestMemoryWrite) refers to stm32f4xx_hal_i2c.o(i.I2C_WaitOnFlagUntilTimeout) for I2C_WaitOnFlagUntilTimeout
    stm32f4xx_hal_i2c.o(i.I2C_RequestMemoryWrite) refers to stm32f4xx_hal_i2c.o(i.I2C_WaitOnMasterAddressFlagUntilTimeout) for I2C_WaitOnMasterAddressFlagUntilTimeout
    stm32f4xx_hal_i2c.o(i.I2C_RequestMemoryWrite) refers to stm32f4xx_hal_i2c.o(i.I2C_WaitOnTXEFlagUntilTimeout) for I2C_WaitOnTXEFlagUntilTimeout
    stm32f4xx_hal_i2c.o(i.I2C_Slave_AF) refers to stm32f4xx_hal_i2c.o(i.HAL_I2C_ListenCpltCallback) for HAL_I2C_ListenCpltCallback
    stm32f4xx_hal_i2c.o(i.I2C_Slave_AF) refers to stm32f4xx_hal_i2c.o(i.HAL_I2C_SlaveTxCpltCallback) for HAL_I2C_SlaveTxCpltCallback
    stm32f4xx_hal_i2c.o(i.I2C_Slave_STOPF) refers to stm32f4xx_hal_i2c.o(i.HAL_I2C_ListenCpltCallback) for HAL_I2C_ListenCpltCallback
    stm32f4xx_hal_i2c.o(i.I2C_Slave_STOPF) refers to stm32f4xx_hal_i2c.o(i.HAL_I2C_SlaveRxCpltCallback) for HAL_I2C_SlaveRxCpltCallback
    stm32f4xx_hal_i2c.o(i.I2C_WaitOnFlagUntilTimeout) refers to stm32f4xx_hal.o(i.HAL_GetTick) for HAL_GetTick
    stm32f4xx_hal_i2c.o(i.I2C_WaitOnMasterAddressFlagUntilTimeout) refers to stm32f4xx_hal.o(i.HAL_GetTick) for HAL_GetTick
    stm32f4xx_hal_i2c.o(i.I2C_WaitOnRXNEFlagUntilTimeout) refers to stm32f4xx_hal.o(i.HAL_GetTick) for HAL_GetTick
    stm32f4xx_hal_i2c.o(i.I2C_WaitOnSTOPFlagUntilTimeout) refers to stm32f4xx_hal.o(i.HAL_GetTick) for HAL_GetTick
    stm32f4xx_hal_i2c.o(i.I2C_WaitOnSTOPFlagUntilTimeout) refers to stm32f4xx_hal_i2c.o(i.I2C_IsAcknowledgeFailed) for I2C_IsAcknowledgeFailed
    stm32f4xx_hal_i2c.o(i.I2C_WaitOnTXEFlagUntilTimeout) refers to stm32f4xx_hal.o(i.HAL_GetTick) for HAL_GetTick
    stm32f4xx_hal_i2c.o(i.I2C_WaitOnTXEFlagUntilTimeout) refers to stm32f4xx_hal_i2c.o(i.I2C_IsAcknowledgeFailed) for I2C_IsAcknowledgeFailed
    stm32f4xx_hal_eth.o(i.ETH_FlushTransmitFIFO) refers to stm32f4xx_hal.o(i.HAL_Delay) for HAL_Delay
    stm32f4xx_hal_eth.o(i.ETH_MACDMAConfig) refers to stm32f4xx_hal.o(i.HAL_Delay) for HAL_Delay
    stm32f4xx_hal_eth.o(i.HAL_ETH_ConfigDMA) refers to stm32f4xx_hal.o(i.HAL_Delay) for HAL_Delay
    stm32f4xx_hal_eth.o(i.HAL_ETH_ConfigMAC) refers to stm32f4xx_hal.o(i.HAL_Delay) for HAL_Delay
    stm32f4xx_hal_eth.o(i.HAL_ETH_DeInit) refers to stm32f4xx_hal_eth.o(i.HAL_ETH_MspDeInit) for HAL_ETH_MspDeInit
    stm32f4xx_hal_eth.o(i.HAL_ETH_IRQHandler) refers to stm32f4xx_hal_eth.o(i.HAL_ETH_RxCpltCallback) for HAL_ETH_RxCpltCallback
    stm32f4xx_hal_eth.o(i.HAL_ETH_IRQHandler) refers to stm32f4xx_hal_eth.o(i.HAL_ETH_TxCpltCallback) for HAL_ETH_TxCpltCallback
    stm32f4xx_hal_eth.o(i.HAL_ETH_IRQHandler) refers to stm32f4xx_hal_eth.o(i.HAL_ETH_ErrorCallback) for HAL_ETH_ErrorCallback
    stm32f4xx_hal_eth.o(i.HAL_ETH_Init) refers to ethernetif.o(i.HAL_ETH_MspInit) for HAL_ETH_MspInit
    stm32f4xx_hal_eth.o(i.HAL_ETH_Init) refers to stm32f4xx_hal.o(i.HAL_GetTick) for HAL_GetTick
    stm32f4xx_hal_eth.o(i.HAL_ETH_Init) refers to stm32f4xx_hal_rcc.o(i.HAL_RCC_GetHCLKFreq) for HAL_RCC_GetHCLKFreq
    stm32f4xx_hal_eth.o(i.HAL_ETH_Init) refers to stm32f4xx_hal_eth.o(i.HAL_ETH_WritePHYRegister) for HAL_ETH_WritePHYRegister
    stm32f4xx_hal_eth.o(i.HAL_ETH_Init) refers to stm32f4xx_hal.o(i.HAL_Delay) for HAL_Delay
    stm32f4xx_hal_eth.o(i.HAL_ETH_Init) refers to stm32f4xx_hal_eth.o(i.HAL_ETH_ReadPHYRegister) for HAL_ETH_ReadPHYRegister
    stm32f4xx_hal_eth.o(i.HAL_ETH_Init) refers to stm32f4xx_hal_eth.o(i.ETH_MACDMAConfig) for ETH_MACDMAConfig
    stm32f4xx_hal_eth.o(i.HAL_ETH_ReadPHYRegister) refers to stm32f4xx_hal.o(i.HAL_GetTick) for HAL_GetTick
    stm32f4xx_hal_eth.o(i.HAL_ETH_Start) refers to stm32f4xx_hal.o(i.HAL_Delay) for HAL_Delay
    stm32f4xx_hal_eth.o(i.HAL_ETH_Start) refers to stm32f4xx_hal_eth.o(i.ETH_FlushTransmitFIFO) for ETH_FlushTransmitFIFO
    stm32f4xx_hal_eth.o(i.HAL_ETH_Stop) refers to stm32f4xx_hal.o(i.HAL_Delay) for HAL_Delay
    stm32f4xx_hal_eth.o(i.HAL_ETH_Stop) refers to stm32f4xx_hal_eth.o(i.ETH_FlushTransmitFIFO) for ETH_FlushTransmitFIFO
    stm32f4xx_hal_eth.o(i.HAL_ETH_WritePHYRegister) refers to stm32f4xx_hal.o(i.HAL_GetTick) for HAL_GetTick
    stm32f4xx_hal_dma.o(i.DMA_CalcBaseAndBitshift) refers to stm32f4xx_hal_dma.o(.constdata) for .constdata
    stm32f4xx_hal_dma.o(i.HAL_DMA_Abort) refers to stm32f4xx_hal.o(i.HAL_GetTick) for HAL_GetTick
    stm32f4xx_hal_dma.o(i.HAL_DMA_DeInit) refers to stm32f4xx_hal_dma.o(i.DMA_CalcBaseAndBitshift) for DMA_CalcBaseAndBitshift
    stm32f4xx_hal_dma.o(i.HAL_DMA_Init) refers to stm32f4xx_hal_dma.o(i.DMA_CalcBaseAndBitshift) for DMA_CalcBaseAndBitshift
    stm32f4xx_hal_dma.o(i.HAL_DMA_PollForTransfer) refers to stm32f4xx_hal.o(i.HAL_GetTick) for HAL_GetTick
    stm32f4xx_hal_dma.o(i.HAL_DMA_Start) refers to stm32f4xx_hal_dma.o(i.DMA_SetConfig) for DMA_SetConfig
    stm32f4xx_hal_dma.o(i.HAL_DMA_Start_IT) refers to stm32f4xx_hal_dma.o(i.DMA_SetConfig) for DMA_SetConfig
    startup_stm32f407xx.o(RESET) refers to startup_stm32f407xx.o(STACK) for __initial_sp
    startup_stm32f407xx.o(RESET) refers to startup_stm32f407xx.o(.text) for Reset_Handler
    startup_stm32f407xx.o(RESET) refers to stm32f4xx_it.o(i.NMI_Handler) for NMI_Handler
    startup_stm32f407xx.o(RESET) refers to stm32f4xx_it.o(i.HardFault_Handler) for HardFault_Handler
    startup_stm32f407xx.o(RESET) refers to stm32f4xx_it.o(i.MemManage_Handler) for MemManage_Handler
    startup_stm32f407xx.o(RESET) refers to stm32f4xx_it.o(i.BusFault_Handler) for BusFault_Handler
    startup_stm32f407xx.o(RESET) refers to stm32f4xx_it.o(i.UsageFault_Handler) for UsageFault_Handler
    startup_stm32f407xx.o(RESET) refers to stm32f4xx_it.o(i.DebugMon_Handler) for DebugMon_Handler
    startup_stm32f407xx.o(RESET) refers to stm32f4xx_it.o(i.SysTick_Handler) for SysTick_Handler
    startup_stm32f407xx.o(RESET) refers to stm32f4xx_it.o(i.EXTI15_10_IRQHandler) for EXTI15_10_IRQHandler
    startup_stm32f407xx.o(.text) refers to system_stm32f4xx.o(i.SystemInit) for SystemInit
    startup_stm32f407xx.o(.text) refers to entry.o(.ARM.Collect$$$$00000000) for __main
    httpserver.o(i.IAP_HTTP_writedata) refers to flash_if.o(i.FLASH_If_Write) for FLASH_If_Write
    httpserver.o(i.IAP_HTTP_writedata) refers to httpserver.o(.data) for .data
    httpserver.o(i.IAP_httpd_init) refers to tcp.o(i.tcp_new) for tcp_new
    httpserver.o(i.IAP_httpd_init) refers to tcp.o(i.tcp_bind) for tcp_bind
    httpserver.o(i.IAP_httpd_init) refers to tcp.o(i.tcp_listen_with_backlog) for tcp_listen_with_backlog
    httpserver.o(i.IAP_httpd_init) refers to tcp.o(i.tcp_accept) for tcp_accept
    httpserver.o(i.IAP_httpd_init) refers to ip_addr.o(.constdata) for ip_addr_any
    httpserver.o(i.IAP_httpd_init) refers to httpserver.o(i.http_accept) for http_accept
    httpserver.o(i.Parse_Content_Length) refers to strncmp.o(.text) for strncmp
    httpserver.o(i.Parse_Content_Length) refers to httpserver.o(.data) for .data
    httpserver.o(i.Parse_Content_Length) refers to httpserver.o(.constdata) for .constdata
    httpserver.o(i.close_conn) refers to tcp.o(i.tcp_arg) for tcp_arg
    httpserver.o(i.close_conn) refers to tcp.o(i.tcp_sent) for tcp_sent
    httpserver.o(i.close_conn) refers to tcp.o(i.tcp_recv) for tcp_recv
    httpserver.o(i.close_conn) refers to mem.o(i.mem_free) for mem_free
    httpserver.o(i.close_conn) refers to tcp.o(i.tcp_close) for tcp_close
    httpserver.o(i.conn_err) refers to mem.o(i.mem_free) for mem_free
    httpserver.o(i.fs_open) refers to strcmp.o(.text) for strcmp
    httpserver.o(i.fs_open) refers to httpserver.o(.constdata) for .constdata
    httpserver.o(i.http_accept) refers to mem.o(i.mem_malloc) for mem_malloc
    httpserver.o(i.http_accept) refers to tcp.o(i.tcp_arg) for tcp_arg
    httpserver.o(i.http_accept) refers to tcp.o(i.tcp_recv) for tcp_recv
    httpserver.o(i.http_accept) refers to tcp.o(i.tcp_err) for tcp_err
    httpserver.o(i.http_accept) refers to tcp.o(i.tcp_poll) for tcp_poll
    httpserver.o(i.http_accept) refers to httpserver.o(i.http_recv) for http_recv
    httpserver.o(i.http_accept) refers to httpserver.o(i.conn_err) for conn_err
    httpserver.o(i.http_accept) refers to httpserver.o(i.http_poll) for http_poll
    httpserver.o(i.http_poll) refers to httpserver.o(i.send_data) for send_data
    httpserver.o(i.http_poll) refers to tcp.o(i.tcp_close) for tcp_close
    httpserver.o(i.http_recv) refers to tcp.o(i.tcp_recved) for tcp_recved
    httpserver.o(i.http_recv) refers to pbuf.o(i.pbuf_free) for pbuf_free
    httpserver.o(i.http_recv) refers to strncmp.o(.text) for strncmp
    httpserver.o(i.http_recv) refers to httpserver.o(i.NVIC_SystemReset) for NVIC_SystemReset
    httpserver.o(i.http_recv) refers to httpserver.o(i.close_conn) for close_conn
    httpserver.o(i.http_recv) refers to printf2.o(i.__0sprintf$2) for __2sprintf
    httpserver.o(i.http_recv) refers to httpserver.o(i.fs_open) for fs_open
    httpserver.o(i.http_recv) refers to httpserver.o(i.send_data) for send_data
    httpserver.o(i.http_recv) refers to tcp.o(i.tcp_sent) for tcp_sent
    httpserver.o(i.http_recv) refers to httpserver.o(i.Parse_Content_Length) for Parse_Content_Length
    httpserver.o(i.http_recv) refers to flash_if.o(i.FLASH_If_Init) for FLASH_If_Init
    httpserver.o(i.http_recv) refers to flash_if.o(i.FLASH_If_Erase) for FLASH_If_Erase
    httpserver.o(i.http_recv) refers to httpserver.o(i.IAP_HTTP_writedata) for IAP_HTTP_writedata
    httpserver.o(i.http_recv) refers to stm32f4xx_hal_gpio.o(i.HAL_GPIO_WritePin) for HAL_GPIO_WritePin
    httpserver.o(i.http_recv) refers to stm32f4xx_hal.o(i.HAL_Delay) for HAL_Delay
    httpserver.o(i.http_recv) refers to stm324xg_eval_eeprom.o(i.BSP_EEPROM_WriteBuffer) for BSP_EEPROM_WriteBuffer
    httpserver.o(i.http_recv) refers to httpserver.o(.data) for .data
    httpserver.o(i.http_recv) refers to httpserver.o(i.http_sent) for http_sent
    httpserver.o(i.http_recv) refers to httpserver.o(.constdata) for .constdata
    httpserver.o(i.http_recv) refers to main.o(.data) for Update_EPPROM
    httpserver.o(i.http_sent) refers to httpserver.o(i.send_data) for send_data
    httpserver.o(i.http_sent) refers to httpserver.o(i.close_conn) for close_conn
    httpserver.o(i.http_sent) refers to stm32f4xx_hal_gpio.o(i.HAL_GPIO_WritePin) for HAL_GPIO_WritePin
    httpserver.o(i.http_sent) refers to stm32f4xx_hal.o(i.HAL_Delay) for HAL_Delay
    httpserver.o(i.http_sent) refers to stm324xg_eval_eeprom.o(i.BSP_EEPROM_WriteBuffer) for BSP_EEPROM_WriteBuffer
    httpserver.o(i.http_sent) refers to httpserver.o(i.NVIC_SystemReset) for NVIC_SystemReset
    httpserver.o(i.http_sent) refers to httpserver.o(.data) for .data
    httpserver.o(i.http_sent) refers to main.o(.data) for Update_EPPROM
    httpserver.o(i.send_data) refers to tcp_out.o(i.tcp_write) for tcp_write
    httpserver.o(.constdata) refers to httpserver.o(.constdata) for data_index_html
    httpserver.o(.constdata) refers to httpserver.o(.constdata) for file_index_html
    httpserver.o(.constdata) refers to httpserver.o(.constdata) for data_reset_html
    httpserver.o(.constdata) refers to httpserver.o(.constdata) for file_reset_html
    httpserver.o(.constdata) refers to httpserver.o(.constdata) for data_upload_html
    httpserver.o(.constdata) refers to httpserver.o(.constdata) for file_upload_html
    httpserver.o(.constdata) refers to httpserver.o(.constdata) for data_uploaddone_html
    ethernetif.o(i.ethernetif_init) refers to ethernetif.o(i.low_level_init) for low_level_init
    ethernetif.o(i.ethernetif_init) refers to etharp.o(i.etharp_output) for etharp_output
    ethernetif.o(i.ethernetif_init) refers to ethernetif.o(i.low_level_output) for low_level_output
    ethernetif.o(i.ethernetif_input) refers to ethernetif.o(i.low_level_input) for low_level_input
    ethernetif.o(i.ethernetif_input) refers to pbuf.o(i.pbuf_free) for pbuf_free
    ethernetif.o(i.ethernetif_set_link) refers to stm32f4xx_hal_eth.o(i.HAL_ETH_ReadPHYRegister) for HAL_ETH_ReadPHYRegister
    ethernetif.o(i.ethernetif_set_link) refers to netif.o(i.netif_set_link_up) for netif_set_link_up
    ethernetif.o(i.ethernetif_set_link) refers to netif.o(i.netif_set_link_down) for netif_set_link_down
    ethernetif.o(i.ethernetif_set_link) refers to ethernetif.o(.bss) for .bss
    ethernetif.o(i.ethernetif_update_config) refers to stm32f4xx_hal_eth.o(i.HAL_ETH_WritePHYRegister) for HAL_ETH_WritePHYRegister
    ethernetif.o(i.ethernetif_update_config) refers to stm32f4xx_hal.o(i.HAL_GetTick) for HAL_GetTick
    ethernetif.o(i.ethernetif_update_config) refers to stm32f4xx_hal_eth.o(i.HAL_ETH_ReadPHYRegister) for HAL_ETH_ReadPHYRegister
    ethernetif.o(i.ethernetif_update_config) refers to stm32f4xx_hal_eth.o(i.HAL_ETH_ConfigMAC) for HAL_ETH_ConfigMAC
    ethernetif.o(i.ethernetif_update_config) refers to stm32f4xx_hal_eth.o(i.HAL_ETH_Start) for HAL_ETH_Start
    ethernetif.o(i.ethernetif_update_config) refers to stm32f4xx_hal_eth.o(i.HAL_ETH_Stop) for HAL_ETH_Stop
    ethernetif.o(i.ethernetif_update_config) refers to app_ethernet.o(i.ethernetif_notify_conn_changed) for ethernetif_notify_conn_changed
    ethernetif.o(i.ethernetif_update_config) refers to ethernetif.o(.bss) for .bss
    ethernetif.o(i.low_level_init) refers to stm32f4xx_hal_eth.o(i.HAL_ETH_Init) for HAL_ETH_Init
    ethernetif.o(i.low_level_init) refers to stm32f4xx_hal_eth.o(i.HAL_ETH_DMATxDescListInit) for HAL_ETH_DMATxDescListInit
    ethernetif.o(i.low_level_init) refers to stm32f4xx_hal_eth.o(i.HAL_ETH_DMARxDescListInit) for HAL_ETH_DMARxDescListInit
    ethernetif.o(i.low_level_init) refers to stm32f4xx_hal_eth.o(i.HAL_ETH_Start) for HAL_ETH_Start
    ethernetif.o(i.low_level_init) refers to stm32f4xx_hal_eth.o(i.HAL_ETH_ReadPHYRegister) for HAL_ETH_ReadPHYRegister
    ethernetif.o(i.low_level_init) refers to stm32f4xx_hal_eth.o(i.HAL_ETH_WritePHYRegister) for HAL_ETH_WritePHYRegister
    ethernetif.o(i.low_level_init) refers to ethernetif.o(.bss) for .bss
    ethernetif.o(i.low_level_input) refers to stm32f4xx_hal_eth.o(i.HAL_ETH_GetReceivedFrame) for HAL_ETH_GetReceivedFrame
    ethernetif.o(i.low_level_input) refers to pbuf.o(i.pbuf_alloc) for pbuf_alloc
    ethernetif.o(i.low_level_input) refers to memcpya.o(.text) for __aeabi_memcpy
    ethernetif.o(i.low_level_input) refers to ethernetif.o(.bss) for .bss
    ethernetif.o(i.low_level_output) refers to memcpya.o(.text) for __aeabi_memcpy
    ethernetif.o(i.low_level_output) refers to stm32f4xx_hal_eth.o(i.HAL_ETH_TransmitFrame) for HAL_ETH_TransmitFrame
    ethernetif.o(i.low_level_output) refers to ethernetif.o(.bss) for .bss
    ethernetif.o(i.sys_now) refers to stm32f4xx_hal.o(i.HAL_GetTick) for HAL_GetTick
    flash_if.o(i.FLASH_If_Erase) refers to stm32f4xx_hal_flash_ex.o(i.HAL_FLASHEx_Erase) for HAL_FLASHEx_Erase
    flash_if.o(i.FLASH_If_Init) refers to stm32f4xx_hal_flash.o(i.HAL_FLASH_Unlock) for HAL_FLASH_Unlock
    flash_if.o(i.FLASH_If_Write) refers to stm32f4xx_hal_flash.o(i.HAL_FLASH_Program) for HAL_FLASH_Program
    main.o(i.I2C_Config) refers to stm32f4xx_hal_i2c.o(i.HAL_I2C_GetState) for HAL_I2C_GetState
    main.o(i.I2C_Config) refers to stm32f4xx_hal_i2c.o(i.HAL_I2C_Init) for HAL_I2C_Init
    main.o(i.I2C_Config) refers to stm324xg_eval_eeprom.o(i.BSP_EEPROM_WriteBuffer) for BSP_EEPROM_WriteBuffer
    main.o(i.I2C_Config) refers to main.o(.bss) for .bss
    main.o(i.I2C_Config) refers to main.o(.data) for .data
    main.o(i.Init_Config) refers to stm32f4xx_hal_gpio.o(i.HAL_GPIO_Init) for HAL_GPIO_Init
    main.o(i.Init_Config) refers to stm32f4xx_hal_gpio.o(i.HAL_GPIO_WritePin) for HAL_GPIO_WritePin
    main.o(i.Init_Config) refers to stm32f4xx_hal.o(i.HAL_Delay) for HAL_Delay
    main.o(i.Init_Config) refers to main.o(i.I2C_Config) for I2C_Config
    main.o(i.Init_Config) refers to stm32f4xx_hal_cortex.o(i.HAL_NVIC_SetPriority) for HAL_NVIC_SetPriority
    main.o(i.Init_Config) refers to stm32f4xx_hal_cortex.o(i.HAL_NVIC_EnableIRQ) for HAL_NVIC_EnableIRQ
    main.o(i.Netif_Config) refers to netif.o(i.netif_add) for netif_add
    main.o(i.Netif_Config) refers to netif.o(i.netif_set_default) for netif_set_default
    main.o(i.Netif_Config) refers to netif.o(i.netif_set_up) for netif_set_up
    main.o(i.Netif_Config) refers to netif.o(i.netif_set_down) for netif_set_down
    main.o(i.Netif_Config) refers to netif.o(i.netif_set_link_callback) for netif_set_link_callback
    main.o(i.Netif_Config) refers to etharp.o(i.ethernet_input) for ethernet_input
    main.o(i.Netif_Config) refers to ethernetif.o(i.ethernetif_init) for ethernetif_init
    main.o(i.Netif_Config) refers to main.o(.bss) for .bss
    main.o(i.Netif_Config) refers to ethernetif.o(i.ethernetif_update_config) for ethernetif_update_config
    main.o(i.SystemClock_Config) refers to stm32f4xx_hal_rcc.o(i.HAL_RCC_OscConfig) for HAL_RCC_OscConfig
    main.o(i.SystemClock_Config) refers to stm32f4xx_hal_rcc.o(i.HAL_RCC_ClockConfig) for HAL_RCC_ClockConfig
    main.o(i.SystemClock_Config) refers to stm32f4xx_hal.o(i.HAL_GetREVID) for HAL_GetREVID
    main.o(i.main) refers to stm32f4xx_hal.o(i.HAL_Init) for HAL_Init
    main.o(i.main) refers to main.o(i.SystemClock_Config) for SystemClock_Config
    main.o(i.main) refers to stm32f4xx_hal_gpio.o(i.HAL_GPIO_Init) for HAL_GPIO_Init
    main.o(i.main) refers to stm32f4xx_hal_gpio.o(i.HAL_GPIO_ReadPin) for HAL_GPIO_ReadPin
    main.o(i.main) refers to stm32f4xx_hal_gpio.o(i.HAL_GPIO_WritePin) for HAL_GPIO_WritePin
    main.o(i.main) refers to stm32f4xx_hal.o(i.HAL_Delay) for HAL_Delay
    main.o(i.main) refers to stm324xg_eval_eeprom.o(i.BSP_EEPROM_WriteBuffer) for BSP_EEPROM_WriteBuffer
    main.o(i.main) refers to main.o(i.Init_Config) for Init_Config
    main.o(i.main) refers to init.o(i.lwip_init) for lwip_init
    main.o(i.main) refers to main.o(i.Netif_Config) for Netif_Config
    main.o(i.main) refers to httpserver.o(i.IAP_httpd_init) for IAP_httpd_init
    main.o(i.main) refers to app_ethernet.o(i.User_notification) for User_notification
    main.o(i.main) refers to ethernetif.o(i.ethernetif_input) for ethernetif_input
    main.o(i.main) refers to lwip_timers.o(i.sys_check_timeouts) for sys_check_timeouts
    main.o(i.main) refers to main.o(.data) for .data
    main.o(i.main) refers to main.o(.bss) for .bss
    stm32f4xx_it.o(i.EXTI15_10_IRQHandler) refers to stm32f4xx_hal_gpio.o(i.HAL_GPIO_EXTI_IRQHandler) for HAL_GPIO_EXTI_IRQHandler
    stm32f4xx_it.o(i.SysTick_Handler) refers to stm32f4xx_hal.o(i.HAL_IncTick) for HAL_IncTick
    app_ethernet.o(i.ethernetif_notify_conn_changed) refers to netif.o(i.netif_set_addr) for netif_set_addr
    app_ethernet.o(i.ethernetif_notify_conn_changed) refers to netif.o(i.netif_set_up) for netif_set_up
    app_ethernet.o(i.ethernetif_notify_conn_changed) refers to netif.o(i.netif_set_down) for netif_set_down
    stm324xg_eval_eeprom.o(i.BSP_EEPROM_Init) refers to stm324xg_eval.o(i.EEPROM_IO_Init) for EEPROM_IO_Init
    stm324xg_eval_eeprom.o(i.BSP_EEPROM_Init) refers to stm324xg_eval.o(i.EEPROM_IO_IsDeviceReady) for EEPROM_IO_IsDeviceReady
    stm324xg_eval_eeprom.o(i.BSP_EEPROM_ReadBuffer) refers to stm324xg_eval.o(i.EEPROM_IO_ReadData) for EEPROM_IO_ReadData
    stm324xg_eval_eeprom.o(i.BSP_EEPROM_ReadBuffer) refers to stm324xg_eval_eeprom.o(i.BSP_EEPROM_TIMEOUT_UserCallback) for BSP_EEPROM_TIMEOUT_UserCallback
    stm324xg_eval_eeprom.o(i.BSP_EEPROM_WriteBuffer) refers to stm324xg_eval_eeprom.o(i.EEPROM_WritePage) for EEPROM_WritePage
    stm324xg_eval_eeprom.o(i.EEPROM_WritePage) refers to stm324xg_eval.o(i.EEPROM_IO_WriteData) for EEPROM_IO_WriteData
    stm324xg_eval_eeprom.o(i.EEPROM_WritePage) refers to stm324xg_eval_eeprom.o(i.BSP_EEPROM_TIMEOUT_UserCallback) for BSP_EEPROM_TIMEOUT_UserCallback
    stm324xg_eval_eeprom.o(i.EEPROM_WritePage) refers to stm324xg_eval.o(i.EEPROM_IO_IsDeviceReady) for EEPROM_IO_IsDeviceReady
    stm324xg_eval_eeprom.o(i.EEPROM_WritePage) refers to stm324xg_eval_eeprom.o(.data) for .data
    stm324xg_eval.o(i.EEPROM_IO_IsDeviceReady) refers to stm32f4xx_hal_i2c.o(i.HAL_I2C_IsDeviceReady) for HAL_I2C_IsDeviceReady
    stm324xg_eval.o(i.EEPROM_IO_IsDeviceReady) refers to main.o(.bss) for hi2c1
    stm324xg_eval.o(i.EEPROM_IO_ReadData) refers to stm32f4xx_hal_i2c.o(i.HAL_I2C_Mem_Read) for HAL_I2C_Mem_Read
    stm324xg_eval.o(i.EEPROM_IO_ReadData) refers to stm32f4xx_hal_i2c.o(i.HAL_I2C_DeInit) for HAL_I2C_DeInit
    stm324xg_eval.o(i.EEPROM_IO_ReadData) refers to main.o(.bss) for hi2c1
    stm324xg_eval.o(i.EEPROM_IO_WriteData) refers to stm32f4xx_hal_i2c.o(i.HAL_I2C_Mem_Write) for HAL_I2C_Mem_Write
    stm324xg_eval.o(i.EEPROM_IO_WriteData) refers to stm32f4xx_hal_i2c.o(i.HAL_I2C_DeInit) for HAL_I2C_DeInit
    stm324xg_eval.o(i.EEPROM_IO_WriteData) refers to main.o(.bss) for hi2c1
    entry.o(.ARM.Collect$$$$00000000) refers (Special) to entry10a.o(.ARM.Collect$$$$0000000D) for __rt_final_cpp
    entry.o(.ARM.Collect$$$$00000000) refers (Special) to entry11a.o(.ARM.Collect$$$$0000000F) for __rt_final_exit
    entry.o(.ARM.Collect$$$$00000000) refers (Special) to entry7b.o(.ARM.Collect$$$$00000008) for _main_clock
    entry.o(.ARM.Collect$$$$00000000) refers (Special) to entry8b.o(.ARM.Collect$$$$0000000A) for _main_cpp_init
    entry.o(.ARM.Collect$$$$00000000) refers (Special) to entry9a.o(.ARM.Collect$$$$0000000B) for _main_init
    entry.o(.ARM.Collect$$$$00000000) refers (Special) to entry5.o(.ARM.Collect$$$$00000004) for _main_scatterload
    entry.o(.ARM.Collect$$$$00000000) refers (Special) to entry2.o(.ARM.Collect$$$$00000001) for _main_stk
    printfb.o(i.__0fprintf$bare) refers to printfb.o(i._printf_core) for _printf_core
    printfb.o(i.__0fprintf$bare) refers to fputc.o(i.fputc) for fputc
    printfb.o(i.__0printf$bare) refers to printfb.o(i._printf_core) for _printf_core
    printfb.o(i.__0printf$bare) refers to fputc.o(i.fputc) for fputc
    printfb.o(i.__0printf$bare) refers to stdout.o(.data) for __stdout
    printfb.o(i.__0snprintf$bare) refers to printfb.o(i._printf_core) for _printf_core
    printfb.o(i.__0snprintf$bare) refers to printfb.o(i._snputc) for _snputc
    printfb.o(i.__0sprintf$bare) refers to printfb.o(i._printf_core) for _printf_core
    printfb.o(i.__0sprintf$bare) refers to printfb.o(i._sputc) for _sputc
    printfb.o(i.__0vfprintf$bare) refers to printfb.o(i._printf_core) for _printf_core
    printfb.o(i.__0vfprintf$bare) refers to fputc.o(i.fputc) for fputc
    printfb.o(i.__0vprintf$bare) refers to printfb.o(i._printf_core) for _printf_core
    printfb.o(i.__0vprintf$bare) refers to fputc.o(i.fputc) for fputc
    printfb.o(i.__0vprintf$bare) refers to stdout.o(.data) for __stdout
    printfb.o(i.__0vsnprintf$bare) refers to printfb.o(i._printf_core) for _printf_core
    printfb.o(i.__0vsnprintf$bare) refers to printfb.o(i._snputc) for _snputc
    printfb.o(i.__0vsprintf$bare) refers to printfb.o(i._printf_core) for _printf_core
    printfb.o(i.__0vsprintf$bare) refers to printfb.o(i._sputc) for _sputc
    printf0.o(i.__0fprintf$0) refers to printf0.o(i._printf_core) for _printf_core
    printf0.o(i.__0fprintf$0) refers to fputc.o(i.fputc) for fputc
    printf0.o(i.__0printf$0) refers to printf0.o(i._printf_core) for _printf_core
    printf0.o(i.__0printf$0) refers to fputc.o(i.fputc) for fputc
    printf0.o(i.__0printf$0) refers to stdout.o(.data) for __stdout
    printf0.o(i.__0snprintf$0) refers to printf0.o(i._printf_core) for _printf_core
    printf0.o(i.__0snprintf$0) refers to printf0.o(i._snputc) for _snputc
    printf0.o(i.__0sprintf$0) refers to printf0.o(i._printf_core) for _printf_core
    printf0.o(i.__0sprintf$0) refers to printf0.o(i._sputc) for _sputc
    printf0.o(i.__0vfprintf$0) refers to printf0.o(i._printf_core) for _printf_core
    printf0.o(i.__0vfprintf$0) refers to fputc.o(i.fputc) for fputc
    printf0.o(i.__0vprintf$0) refers to printf0.o(i._printf_core) for _printf_core
    printf0.o(i.__0vprintf$0) refers to fputc.o(i.fputc) for fputc
    printf0.o(i.__0vprintf$0) refers to stdout.o(.data) for __stdout
    printf0.o(i.__0vsnprintf$0) refers to printf0.o(i._printf_core) for _printf_core
    printf0.o(i.__0vsnprintf$0) refers to printf0.o(i._snputc) for _snputc
    printf0.o(i.__0vsprintf$0) refers to printf0.o(i._printf_core) for _printf_core
    printf0.o(i.__0vsprintf$0) refers to printf0.o(i._sputc) for _sputc
    printf1.o(i.__0fprintf$1) refers to printf1.o(i._printf_core) for _printf_core
    printf1.o(i.__0fprintf$1) refers to fputc.o(i.fputc) for fputc
    printf1.o(i.__0printf$1) refers to printf1.o(i._printf_core) for _printf_core
    printf1.o(i.__0printf$1) refers to fputc.o(i.fputc) for fputc
    printf1.o(i.__0printf$1) refers to stdout.o(.data) for __stdout
    printf1.o(i.__0snprintf$1) refers to printf1.o(i._printf_core) for _printf_core
    printf1.o(i.__0snprintf$1) refers to printf1.o(i._snputc) for _snputc
    printf1.o(i.__0sprintf$1) refers to printf1.o(i._printf_core) for _printf_core
    printf1.o(i.__0sprintf$1) refers to printf1.o(i._sputc) for _sputc
    printf1.o(i.__0vfprintf$1) refers to printf1.o(i._printf_core) for _printf_core
    printf1.o(i.__0vfprintf$1) refers to fputc.o(i.fputc) for fputc
    printf1.o(i.__0vprintf$1) refers to printf1.o(i._printf_core) for _printf_core
    printf1.o(i.__0vprintf$1) refers to fputc.o(i.fputc) for fputc
    printf1.o(i.__0vprintf$1) refers to stdout.o(.data) for __stdout
    printf1.o(i.__0vsnprintf$1) refers to printf1.o(i._printf_core) for _printf_core
    printf1.o(i.__0vsnprintf$1) refers to printf1.o(i._snputc) for _snputc
    printf1.o(i.__0vsprintf$1) refers to printf1.o(i._printf_core) for _printf_core
    printf1.o(i.__0vsprintf$1) refers to printf1.o(i._sputc) for _sputc
    printf1.o(i._printf_core) refers to uidiv.o(.text) for __aeabi_uidivmod
    printf2.o(i.__0fprintf$2) refers to printf2.o(i._printf_core) for _printf_core
    printf2.o(i.__0fprintf$2) refers to fputc.o(i.fputc) for fputc
    printf2.o(i.__0printf$2) refers to printf2.o(i._printf_core) for _printf_core
    printf2.o(i.__0printf$2) refers to fputc.o(i.fputc) for fputc
    printf2.o(i.__0printf$2) refers to stdout.o(.data) for __stdout
    printf2.o(i.__0snprintf$2) refers to printf2.o(i._printf_core) for _printf_core
    printf2.o(i.__0snprintf$2) refers to printf2.o(i._snputc) for _snputc
    printf2.o(i.__0sprintf$2) refers to printf2.o(i._printf_core) for _printf_core
    printf2.o(i.__0sprintf$2) refers to printf2.o(i._sputc) for _sputc
    printf2.o(i.__0vfprintf$2) refers to printf2.o(i._printf_core) for _printf_core
    printf2.o(i.__0vfprintf$2) refers to fputc.o(i.fputc) for fputc
    printf2.o(i.__0vprintf$2) refers to printf2.o(i._printf_core) for _printf_core
    printf2.o(i.__0vprintf$2) refers to fputc.o(i.fputc) for fputc
    printf2.o(i.__0vprintf$2) refers to stdout.o(.data) for __stdout
    printf2.o(i.__0vsnprintf$2) refers to printf2.o(i._printf_core) for _printf_core
    printf2.o(i.__0vsnprintf$2) refers to printf2.o(i._snputc) for _snputc
    printf2.o(i.__0vsprintf$2) refers to printf2.o(i._printf_core) for _printf_core
    printf2.o(i.__0vsprintf$2) refers to printf2.o(i._sputc) for _sputc
    printf3.o(i.__0fprintf$3) refers to printf3.o(i._printf_core) for _printf_core
    printf3.o(i.__0fprintf$3) refers to fputc.o(i.fputc) for fputc
    printf3.o(i.__0printf$3) refers to printf3.o(i._printf_core) for _printf_core
    printf3.o(i.__0printf$3) refers to fputc.o(i.fputc) for fputc
    printf3.o(i.__0printf$3) refers to stdout.o(.data) for __stdout
    printf3.o(i.__0snprintf$3) refers to printf3.o(i._printf_core) for _printf_core
    printf3.o(i.__0snprintf$3) refers to printf3.o(i._snputc) for _snputc
    printf3.o(i.__0sprintf$3) refers to printf3.o(i._printf_core) for _printf_core
    printf3.o(i.__0sprintf$3) refers to printf3.o(i._sputc) for _sputc
    printf3.o(i.__0vfprintf$3) refers to printf3.o(i._printf_core) for _printf_core
    printf3.o(i.__0vfprintf$3) refers to fputc.o(i.fputc) for fputc
    printf3.o(i.__0vprintf$3) refers to printf3.o(i._printf_core) for _printf_core
    printf3.o(i.__0vprintf$3) refers to fputc.o(i.fputc) for fputc
    printf3.o(i.__0vprintf$3) refers to stdout.o(.data) for __stdout
    printf3.o(i.__0vsnprintf$3) refers to printf3.o(i._printf_core) for _printf_core
    printf3.o(i.__0vsnprintf$3) refers to printf3.o(i._snputc) for _snputc
    printf3.o(i.__0vsprintf$3) refers to printf3.o(i._printf_core) for _printf_core
    printf3.o(i.__0vsprintf$3) refers to printf3.o(i._sputc) for _sputc
    printf3.o(i._printf_core) refers to uidiv.o(.text) for __aeabi_uidivmod
    printf4.o(i.__0fprintf$4) refers to printf4.o(i._printf_core) for _printf_core
    printf4.o(i.__0fprintf$4) refers to fputc.o(i.fputc) for fputc
    printf4.o(i.__0printf$4) refers to printf4.o(i._printf_core) for _printf_core
    printf4.o(i.__0printf$4) refers to fputc.o(i.fputc) for fputc
    printf4.o(i.__0printf$4) refers to stdout.o(.data) for __stdout
    printf4.o(i.__0snprintf$4) refers to printf4.o(i._printf_core) for _printf_core
    printf4.o(i.__0snprintf$4) refers to printf4.o(i._snputc) for _snputc
    printf4.o(i.__0sprintf$4) refers to printf4.o(i._printf_core) for _printf_core
    printf4.o(i.__0sprintf$4) refers to printf4.o(i._sputc) for _sputc
    printf4.o(i.__0vfprintf$4) refers to printf4.o(i._printf_core) for _printf_core
    printf4.o(i.__0vfprintf$4) refers to fputc.o(i.fputc) for fputc
    printf4.o(i.__0vprintf$4) refers to printf4.o(i._printf_core) for _printf_core
    printf4.o(i.__0vprintf$4) refers to fputc.o(i.fputc) for fputc
    printf4.o(i.__0vprintf$4) refers to stdout.o(.data) for __stdout
    printf4.o(i.__0vsnprintf$4) refers to printf4.o(i._printf_core) for _printf_core
    printf4.o(i.__0vsnprintf$4) refers to printf4.o(i._snputc) for _snputc
    printf4.o(i.__0vsprintf$4) refers to printf4.o(i._printf_core) for _printf_core
    printf4.o(i.__0vsprintf$4) refers to printf4.o(i._sputc) for _sputc
    printf4.o(i._printf_core) refers to uldiv.o(.text) for __aeabi_uldivmod
    printf5.o(i.__0fprintf$5) refers to printf5.o(i._printf_core) for _printf_core
    printf5.o(i.__0fprintf$5) refers to fputc.o(i.fputc) for fputc
    printf5.o(i.__0printf$5) refers to printf5.o(i._printf_core) for _printf_core
    printf5.o(i.__0printf$5) refers to fputc.o(i.fputc) for fputc
    printf5.o(i.__0printf$5) refers to stdout.o(.data) for __stdout
    printf5.o(i.__0snprintf$5) refers to printf5.o(i._printf_core) for _printf_core
    printf5.o(i.__0snprintf$5) refers to printf5.o(i._snputc) for _snputc
    printf5.o(i.__0sprintf$5) refers to printf5.o(i._printf_core) for _printf_core
    printf5.o(i.__0sprintf$5) refers to printf5.o(i._sputc) for _sputc
    printf5.o(i.__0vfprintf$5) refers to printf5.o(i._printf_core) for _printf_core
    printf5.o(i.__0vfprintf$5) refers to fputc.o(i.fputc) for fputc
    printf5.o(i.__0vprintf$5) refers to printf5.o(i._printf_core) for _printf_core
    printf5.o(i.__0vprintf$5) refers to fputc.o(i.fputc) for fputc
    printf5.o(i.__0vprintf$5) refers to stdout.o(.data) for __stdout
    printf5.o(i.__0vsnprintf$5) refers to printf5.o(i._printf_core) for _printf_core
    printf5.o(i.__0vsnprintf$5) refers to printf5.o(i._snputc) for _snputc
    printf5.o(i.__0vsprintf$5) refers to printf5.o(i._printf_core) for _printf_core
    printf5.o(i.__0vsprintf$5) refers to printf5.o(i._sputc) for _sputc
    printf5.o(i._printf_core) refers to uldiv.o(.text) for __aeabi_uldivmod
    printf6.o(i.__0fprintf$6) refers to printf6.o(i._printf_core) for _printf_core
    printf6.o(i.__0fprintf$6) refers to fputc.o(i.fputc) for fputc
    printf6.o(i.__0printf$6) refers to printf6.o(i._printf_core) for _printf_core
    printf6.o(i.__0printf$6) refers to fputc.o(i.fputc) for fputc
    printf6.o(i.__0printf$6) refers to stdout.o(.data) for __stdout
    printf6.o(i.__0snprintf$6) refers to printf6.o(i._printf_core) for _printf_core
    printf6.o(i.__0snprintf$6) refers to printf6.o(i._snputc) for _snputc
    printf6.o(i.__0sprintf$6) refers to printf6.o(i._printf_core) for _printf_core
    printf6.o(i.__0sprintf$6) refers to printf6.o(i._sputc) for _sputc
    printf6.o(i.__0vfprintf$6) refers to printf6.o(i._printf_core) for _printf_core
    printf6.o(i.__0vfprintf$6) refers to fputc.o(i.fputc) for fputc
    printf6.o(i.__0vprintf$6) refers to printf6.o(i._printf_core) for _printf_core
    printf6.o(i.__0vprintf$6) refers to fputc.o(i.fputc) for fputc
    printf6.o(i.__0vprintf$6) refers to stdout.o(.data) for __stdout
    printf6.o(i.__0vsnprintf$6) refers to printf6.o(i._printf_core) for _printf_core
    printf6.o(i.__0vsnprintf$6) refers to printf6.o(i._snputc) for _snputc
    printf6.o(i.__0vsprintf$6) refers to printf6.o(i._printf_core) for _printf_core
    printf6.o(i.__0vsprintf$6) refers to printf6.o(i._sputc) for _sputc
    printf6.o(i._printf_core) refers to printf6.o(i._printf_pre_padding) for _printf_pre_padding
    printf6.o(i._printf_core) refers to uidiv.o(.text) for __aeabi_uidivmod
    printf6.o(i._printf_core) refers to printf6.o(i._printf_post_padding) for _printf_post_padding
    printf7.o(i.__0fprintf$7) refers to printf7.o(i._printf_core) for _printf_core
    printf7.o(i.__0fprintf$7) refers to fputc.o(i.fputc) for fputc
    printf7.o(i.__0printf$7) refers to printf7.o(i._printf_core) for _printf_core
    printf7.o(i.__0printf$7) refers to fputc.o(i.fputc) for fputc
    printf7.o(i.__0printf$7) refers to stdout.o(.data) for __stdout
    printf7.o(i.__0snprintf$7) refers to printf7.o(i._printf_core) for _printf_core
    printf7.o(i.__0snprintf$7) refers to printf7.o(i._snputc) for _snputc
    printf7.o(i.__0sprintf$7) refers to printf7.o(i._printf_core) for _printf_core
    printf7.o(i.__0sprintf$7) refers to printf7.o(i._sputc) for _sputc
    printf7.o(i.__0vfprintf$7) refers to printf7.o(i._printf_core) for _printf_core
    printf7.o(i.__0vfprintf$7) refers to fputc.o(i.fputc) for fputc
    printf7.o(i.__0vprintf$7) refers to printf7.o(i._printf_core) for _printf_core
    printf7.o(i.__0vprintf$7) refers to fputc.o(i.fputc) for fputc
    printf7.o(i.__0vprintf$7) refers to stdout.o(.data) for __stdout
    printf7.o(i.__0vsnprintf$7) refers to printf7.o(i._printf_core) for _printf_core
    printf7.o(i.__0vsnprintf$7) refers to printf7.o(i._snputc) for _snputc
    printf7.o(i.__0vsprintf$7) refers to printf7.o(i._printf_core) for _printf_core
    printf7.o(i.__0vsprintf$7) refers to printf7.o(i._sputc) for _sputc
    printf7.o(i._printf_core) refers to printf7.o(i._printf_pre_padding) for _printf_pre_padding
    printf7.o(i._printf_core) refers to uldiv.o(.text) for __aeabi_uldivmod
    printf7.o(i._printf_core) refers to printf7.o(i._printf_post_padding) for _printf_post_padding
    printf8.o(i.__0fprintf$8) refers to printf8.o(i._printf_core) for _printf_core
    printf8.o(i.__0fprintf$8) refers to fputc.o(i.fputc) for fputc
    printf8.o(i.__0printf$8) refers to printf8.o(i._printf_core) for _printf_core
    printf8.o(i.__0printf$8) refers to fputc.o(i.fputc) for fputc
    printf8.o(i.__0printf$8) refers to stdout.o(.data) for __stdout
    printf8.o(i.__0snprintf$8) refers to printf8.o(i._printf_core) for _printf_core
    printf8.o(i.__0snprintf$8) refers to printf8.o(i._snputc) for _snputc
    printf8.o(i.__0sprintf$8) refers to printf8.o(i._printf_core) for _printf_core
    printf8.o(i.__0sprintf$8) refers to printf8.o(i._sputc) for _sputc
    printf8.o(i.__0vfprintf$8) refers to printf8.o(i._printf_core) for _printf_core
    printf8.o(i.__0vfprintf$8) refers to fputc.o(i.fputc) for fputc
    printf8.o(i.__0vprintf$8) refers to printf8.o(i._printf_core) for _printf_core
    printf8.o(i.__0vprintf$8) refers to fputc.o(i.fputc) for fputc
    printf8.o(i.__0vprintf$8) refers to stdout.o(.data) for __stdout
    printf8.o(i.__0vsnprintf$8) refers to printf8.o(i._printf_core) for _printf_core
    printf8.o(i.__0vsnprintf$8) refers to printf8.o(i._snputc) for _snputc
    printf8.o(i.__0vsprintf$8) refers to printf8.o(i._printf_core) for _printf_core
    printf8.o(i.__0vsprintf$8) refers to printf8.o(i._sputc) for _sputc
    printf8.o(i._printf_core) refers to printf8.o(i._printf_pre_padding) for _printf_pre_padding
    printf8.o(i._printf_core) refers to uldiv.o(.text) for __aeabi_uldivmod
    printf8.o(i._printf_core) refers to printf8.o(i._printf_post_padding) for _printf_post_padding
    printfa.o(i.__0fprintf) refers (Special) to iusefp.o(.text) for __I$use$fp
    printfa.o(i.__0fprintf) refers to printfa.o(i._printf_core) for _printf_core
    printfa.o(i.__0fprintf) refers to fputc.o(i.fputc) for fputc
    printfa.o(i.__0printf) refers (Special) to iusefp.o(.text) for __I$use$fp
    printfa.o(i.__0printf) refers to printfa.o(i._printf_core) for _printf_core
    printfa.o(i.__0printf) refers to fputc.o(i.fputc) for fputc
    printfa.o(i.__0printf) refers to stdout.o(.data) for __stdout
    printfa.o(i.__0snprintf) refers (Special) to iusefp.o(.text) for __I$use$fp
    printfa.o(i.__0snprintf) refers to printfa.o(i._printf_core) for _printf_core
    printfa.o(i.__0snprintf) refers to printfa.o(i._snputc) for _snputc
    printfa.o(i.__0sprintf) refers (Special) to iusefp.o(.text) for __I$use$fp
    printfa.o(i.__0sprintf) refers to printfa.o(i._printf_core) for _printf_core
    printfa.o(i.__0sprintf) refers to printfa.o(i._sputc) for _sputc
    printfa.o(i.__0vfprintf) refers (Special) to iusefp.o(.text) for __I$use$fp
    printfa.o(i.__0vfprintf) refers to printfa.o(i._printf_core) for _printf_core
    printfa.o(i.__0vfprintf) refers to fputc.o(i.fputc) for fputc
    printfa.o(i.__0vprintf) refers (Special) to iusefp.o(.text) for __I$use$fp
    printfa.o(i.__0vprintf) refers to printfa.o(i._printf_core) for _printf_core
    printfa.o(i.__0vprintf) refers to fputc.o(i.fputc) for fputc
    printfa.o(i.__0vprintf) refers to stdout.o(.data) for __stdout
    printfa.o(i.__0vsnprintf) refers (Special) to iusefp.o(.text) for __I$use$fp
    printfa.o(i.__0vsnprintf) refers to printfa.o(i._printf_core) for _printf_core
    printfa.o(i.__0vsnprintf) refers to printfa.o(i._snputc) for _snputc
    printfa.o(i.__0vsprintf) refers (Special) to iusefp.o(.text) for __I$use$fp
    printfa.o(i.__0vsprintf) refers to printfa.o(i._printf_core) for _printf_core
    printfa.o(i.__0vsprintf) refers to printfa.o(i._sputc) for _sputc
    printfa.o(i._fp_digits) refers (Special) to iusefp.o(.text) for __I$use$fp
    printfa.o(i._fp_digits) refers to dmul.o(.text) for __aeabi_dmul
    printfa.o(i._fp_digits) refers to ddiv.o(.text) for __aeabi_ddiv
    printfa.o(i._fp_digits) refers to cdrcmple.o(.text) for __aeabi_cdrcmple
    printfa.o(i._fp_digits) refers to dadd.o(.text) for __aeabi_dadd
    printfa.o(i._fp_digits) refers to dfixul.o(.text) for __aeabi_d2ulz
    printfa.o(i._fp_digits) refers to uldiv.o(.text) for __aeabi_uldivmod
    printfa.o(i._printf_core) refers (Special) to iusefp.o(.text) for __I$use$fp
    printfa.o(i._printf_core) refers to printfa.o(i._printf_pre_padding) for _printf_pre_padding
    printfa.o(i._printf_core) refers to uldiv.o(.text) for __aeabi_uldivmod
    printfa.o(i._printf_core) refers to printfa.o(i._printf_post_padding) for _printf_post_padding
    printfa.o(i._printf_core) refers to printfa.o(i._fp_digits) for _fp_digits
    printfa.o(i._printf_core) refers to uidiv.o(.text) for __aeabi_uidivmod
    printfa.o(i._printf_post_padding) refers (Special) to iusefp.o(.text) for __I$use$fp
    printfa.o(i._printf_pre_padding) refers (Special) to iusefp.o(.text) for __I$use$fp
    printfa.o(i._snputc) refers (Special) to iusefp.o(.text) for __I$use$fp
    printfa.o(i._sputc) refers (Special) to iusefp.o(.text) for __I$use$fp
    entry2.o(.ARM.Collect$$$$00000001) refers to entry2.o(.ARM.Collect$$$$00002712) for __lit__00000000
    entry2.o(.ARM.Collect$$$$00002712) refers to startup_stm32f407xx.o(STACK) for __initial_sp
    entry2.o(__vectab_stack_and_reset_area) refers to startup_stm32f407xx.o(STACK) for __initial_sp
    entry2.o(__vectab_stack_and_reset_area) refers to entry.o(.ARM.Collect$$$$00000000) for __main
    entry5.o(.ARM.Collect$$$$00000004) refers to init.o(.text) for __scatterload
    entry9a.o(.ARM.Collect$$$$0000000B) refers to main.o(i.main) for main
    entry9b.o(.ARM.Collect$$$$0000000C) refers to main.o(i.main) for main
    fputc.o(i.fputc) refers (Special) to iusesemip.o(.text) for __I$use$semihosting$fputc
    fputc.o(i.fputc) refers (Special) to semi.o(.text) for __semihosting_library_function
    uldiv.o(.text) refers to llushr.o(.text) for __aeabi_llsr
    uldiv.o(.text) refers to llshl.o(.text) for __aeabi_llsl
    dadd.o(.text) refers to llshl.o(.text) for __aeabi_llsl
    dadd.o(.text) refers to llsshr.o(.text) for __aeabi_lasr
    dadd.o(.text) refers to depilogue.o(.text) for _double_epilogue
    dmul.o(.text) refers to depilogue.o(.text) for _double_epilogue
    ddiv.o(.text) refers to depilogue.o(.text) for _double_round
    dfixul.o(.text) refers to llushr.o(.text) for __aeabi_llsr
    dfixul.o(.text) refers to llshl.o(.text) for __aeabi_llsl
    init.o(.text) refers to entry5.o(.ARM.Collect$$$$00000004) for __main_after_scatterload
    depilogue.o(.text) refers to llshl.o(.text) for __aeabi_llsl
    depilogue.o(.text) refers to llushr.o(.text) for __aeabi_llsr


==============================================================================

Removing Unused input sections from the image.

    Removing system_stm32f4xx.o(.rev16_text), (4 bytes).
    Removing system_stm32f4xx.o(.revsh_text), (4 bytes).
    Removing system_stm32f4xx.o(.rrx_text), (6 bytes).
    Removing system_stm32f4xx.o(i.SystemCoreClockUpdate), (124 bytes).
    Removing lwip_timers.o(i.sys_restart_timeouts), (16 bytes).
    Removing lwip_timers.o(i.sys_untimeout), (72 bytes).
    Removing memp.o(.conststring), (110 bytes).
    Removing memp.o(.data), (40 bytes).
    Removing dhcp.o(i.dhcp_cleanup), (20 bytes).
    Removing dhcp.o(i.dhcp_handle_ack), (92 bytes).
    Removing dhcp.o(i.dhcp_inform), (152 bytes).
    Removing dhcp.o(i.dhcp_network_changed), (70 bytes).
    Removing dhcp.o(i.dhcp_parse_reply), (504 bytes).
    Removing dhcp.o(i.dhcp_recv), (276 bytes).
    Removing dhcp.o(i.dhcp_set_struct), (18 bytes).
    Removing dhcp.o(i.dhcp_start), (164 bytes).
    Removing dhcp.o(i.dhcp_stop), (48 bytes).
    Removing dhcp.o(.bss), (50 bytes).
    Removing udp.o(i.udp_connect), (76 bytes).
    Removing udp.o(i.udp_disconnect), (16 bytes).
    Removing udp.o(i.udp_new), (26 bytes).
    Removing udp.o(i.udp_recv), (6 bytes).
    Removing udp.o(i.udp_remove), (44 bytes).
    Removing udp.o(i.udp_send), (8 bytes).
    Removing udp.o(i.udp_sendto), (40 bytes).
    Removing mem.o(i.mem_calloc), (26 bytes).
    Removing netif.o(i.netif_find), (64 bytes).
    Removing netif.o(i.netif_remove), (72 bytes).
    Removing netif.o(i.netif_set_link_down), (26 bytes).
    Removing netif.o(i.netif_set_link_up), (66 bytes).
    Removing tcp.o(i.tcp_connect), (244 bytes).
    Removing tcp.o(i.tcp_debug_state_str), (12 bytes).
    Removing tcp.o(i.tcp_setprio), (4 bytes).
    Removing tcp.o(i.tcp_shutdown), (78 bytes).
    Removing raw.o(i.raw_bind), (10 bytes).
    Removing raw.o(i.raw_connect), (10 bytes).
    Removing raw.o(i.raw_new), (44 bytes).
    Removing raw.o(i.raw_recv), (6 bytes).
    Removing raw.o(i.raw_remove), (44 bytes).
    Removing raw.o(i.raw_send), (6 bytes).
    Removing raw.o(i.raw_sendto), (144 bytes).
    Removing pbuf.o(i.pbuf_coalesce), (44 bytes).
    Removing pbuf.o(i.pbuf_dechain), (38 bytes).
    Removing pbuf.o(i.pbuf_get_at), (24 bytes).
    Removing pbuf.o(i.pbuf_memcmp), (68 bytes).
    Removing pbuf.o(i.pbuf_memfind), (60 bytes).
    Removing pbuf.o(i.pbuf_strstr), (56 bytes).
    Removing pbuf.o(i.pbuf_take), (78 bytes).
    Removing ip_addr.o(i.ip4_addr_netmask_valid), (38 bytes).
    Removing ip_addr.o(i.ipaddr_addr), (20 bytes).
    Removing ip_addr.o(i.ipaddr_aton), (248 bytes).
    Removing ip_addr.o(i.ipaddr_ntoa), (12 bytes).
    Removing ip_addr.o(i.ipaddr_ntoa_r), (120 bytes).
    Removing ip_addr.o(.bss), (16 bytes).
    Removing inet_chksum.o(i.inet_chksum_pseudo), (136 bytes).
    Removing inet_chksum.o(i.inet_chksum_pseudo_partial), (154 bytes).
    Removing err.o(i.lwip_strerr), (16 bytes).
    Removing err.o(.conststring), (295 bytes).
    Removing err.o(.data), (64 bytes).
    Removing etharp.o(i.etharp_find_addr), (56 bytes).
    Removing stm32f4xx_hal_flash_ex.o(.rev16_text), (4 bytes).
    Removing stm32f4xx_hal_flash_ex.o(.revsh_text), (4 bytes).
    Removing stm32f4xx_hal_flash_ex.o(.rrx_text), (6 bytes).
    Removing stm32f4xx_hal_flash_ex.o(i.HAL_FLASHEx_Erase_IT), (104 bytes).
    Removing stm32f4xx_hal_flash_ex.o(i.HAL_FLASHEx_OBGetConfig), (64 bytes).
    Removing stm32f4xx_hal_flash_ex.o(i.HAL_FLASHEx_OBProgram), (204 bytes).
    Removing stm32f4xx_hal_rcc.o(.rev16_text), (4 bytes).
    Removing stm32f4xx_hal_rcc.o(.revsh_text), (4 bytes).
    Removing stm32f4xx_hal_rcc.o(.rrx_text), (6 bytes).
    Removing stm32f4xx_hal_rcc.o(i.HAL_RCC_CSSCallback), (2 bytes).
    Removing stm32f4xx_hal_rcc.o(i.HAL_RCC_DeInit), (2 bytes).
    Removing stm32f4xx_hal_rcc.o(i.HAL_RCC_DisableCSS), (12 bytes).
    Removing stm32f4xx_hal_rcc.o(i.HAL_RCC_EnableCSS), (12 bytes).
    Removing stm32f4xx_hal_rcc.o(i.HAL_RCC_GetClockConfig), (64 bytes).
    Removing stm32f4xx_hal_rcc.o(i.HAL_RCC_GetOscConfig), (224 bytes).
    Removing stm32f4xx_hal_rcc.o(i.HAL_RCC_GetPCLK2Freq), (44 bytes).
    Removing stm32f4xx_hal_rcc.o(i.HAL_RCC_MCOConfig), (140 bytes).
    Removing stm32f4xx_hal_rcc.o(i.HAL_RCC_NMI_IRQHandler), (28 bytes).
    Removing stm32f4xx_hal_flash.o(.rev16_text), (4 bytes).
    Removing stm32f4xx_hal_flash.o(.revsh_text), (4 bytes).
    Removing stm32f4xx_hal_flash.o(.rrx_text), (6 bytes).
    Removing stm32f4xx_hal_flash.o(i.HAL_FLASH_EndOfOperationCallback), (2 bytes).
    Removing stm32f4xx_hal_flash.o(i.HAL_FLASH_GetError), (12 bytes).
    Removing stm32f4xx_hal_flash.o(i.HAL_FLASH_IRQHandler), (208 bytes).
    Removing stm32f4xx_hal_flash.o(i.HAL_FLASH_Lock), (20 bytes).
    Removing stm32f4xx_hal_flash.o(i.HAL_FLASH_OB_Launch), (24 bytes).
    Removing stm32f4xx_hal_flash.o(i.HAL_FLASH_OB_Lock), (20 bytes).
    Removing stm32f4xx_hal_flash.o(i.HAL_FLASH_OB_Unlock), (40 bytes).
    Removing stm32f4xx_hal_flash.o(i.HAL_FLASH_OperationErrorCallback), (2 bytes).
    Removing stm32f4xx_hal_flash.o(i.HAL_FLASH_Program_IT), (108 bytes).
    Removing stm32f4xx_hal.o(.rev16_text), (4 bytes).
    Removing stm32f4xx_hal.o(.revsh_text), (4 bytes).
    Removing stm32f4xx_hal.o(.rrx_text), (6 bytes).
    Removing stm32f4xx_hal.o(i.HAL_DBGMCU_DisableDBGSleepMode), (16 bytes).
    Removing stm32f4xx_hal.o(i.HAL_DBGMCU_DisableDBGStandbyMode), (16 bytes).
    Removing stm32f4xx_hal.o(i.HAL_DBGMCU_DisableDBGStopMode), (16 bytes).
    Removing stm32f4xx_hal.o(i.HAL_DBGMCU_EnableDBGSleepMode), (16 bytes).
    Removing stm32f4xx_hal.o(i.HAL_DBGMCU_EnableDBGStandbyMode), (16 bytes).
    Removing stm32f4xx_hal.o(i.HAL_DBGMCU_EnableDBGStopMode), (16 bytes).
    Removing stm32f4xx_hal.o(i.HAL_DeInit), (52 bytes).
    Removing stm32f4xx_hal.o(i.HAL_DisableCompensationCell), (28 bytes).
    Removing stm32f4xx_hal.o(i.HAL_EnableCompensationCell), (28 bytes).
    Removing stm32f4xx_hal.o(i.HAL_GetDEVID), (16 bytes).
    Removing stm32f4xx_hal.o(i.HAL_GetHalVersion), (8 bytes).
    Removing stm32f4xx_hal.o(i.HAL_MspDeInit), (2 bytes).
    Removing stm32f4xx_hal.o(i.HAL_ResumeTick), (14 bytes).
    Removing stm32f4xx_hal.o(i.HAL_SuspendTick), (14 bytes).
    Removing stm32f4xx_hal_gpio.o(.rev16_text), (4 bytes).
    Removing stm32f4xx_hal_gpio.o(.revsh_text), (4 bytes).
    Removing stm32f4xx_hal_gpio.o(.rrx_text), (6 bytes).
    Removing stm32f4xx_hal_gpio.o(i.HAL_GPIO_DeInit), (352 bytes).
    Removing stm32f4xx_hal_gpio.o(i.HAL_GPIO_LockPin), (34 bytes).
    Removing stm32f4xx_hal_gpio.o(i.HAL_GPIO_TogglePin), (8 bytes).
    Removing stm32f4xx_hal_i2s.o(.rev16_text), (4 bytes).
    Removing stm32f4xx_hal_i2s.o(.revsh_text), (4 bytes).
    Removing stm32f4xx_hal_i2s.o(.rrx_text), (6 bytes).
    Removing stm32f4xx_hal_i2s_ex.o(.rev16_text), (4 bytes).
    Removing stm32f4xx_hal_i2s_ex.o(.revsh_text), (4 bytes).
    Removing stm32f4xx_hal_i2s_ex.o(.rrx_text), (6 bytes).
    Removing stm32f4xx_hal_pwr.o(.rev16_text), (4 bytes).
    Removing stm32f4xx_hal_pwr.o(.revsh_text), (4 bytes).
    Removing stm32f4xx_hal_pwr.o(.rrx_text), (6 bytes).
    Removing stm32f4xx_hal_pwr.o(i.HAL_PWR_ConfigPVD), (124 bytes).
    Removing stm32f4xx_hal_pwr.o(i.HAL_PWR_DeInit), (24 bytes).
    Removing stm32f4xx_hal_pwr.o(i.HAL_PWR_DisableBkUpAccess), (28 bytes).
    Removing stm32f4xx_hal_pwr.o(i.HAL_PWR_DisablePVD), (24 bytes).
    Removing stm32f4xx_hal_pwr.o(i.HAL_PWR_DisableSEVOnPend), (16 bytes).
    Removing stm32f4xx_hal_pwr.o(i.HAL_PWR_DisableSleepOnExit), (16 bytes).
    Removing stm32f4xx_hal_pwr.o(i.HAL_PWR_DisableWakeUpPin), (16 bytes).
    Removing stm32f4xx_hal_pwr.o(i.HAL_PWR_EnableBkUpAccess), (24 bytes).
    Removing stm32f4xx_hal_pwr.o(i.HAL_PWR_EnablePVD), (24 bytes).
    Removing stm32f4xx_hal_pwr.o(i.HAL_PWR_EnableSEVOnPend), (16 bytes).
    Removing stm32f4xx_hal_pwr.o(i.HAL_PWR_EnableSleepOnExit), (16 bytes).
    Removing stm32f4xx_hal_pwr.o(i.HAL_PWR_EnableWakeUpPin), (16 bytes).
    Removing stm32f4xx_hal_pwr.o(i.HAL_PWR_EnterSLEEPMode), (32 bytes).
    Removing stm32f4xx_hal_pwr.o(i.HAL_PWR_EnterSTANDBYMode), (32 bytes).
    Removing stm32f4xx_hal_pwr.o(i.HAL_PWR_EnterSTOPMode), (56 bytes).
    Removing stm32f4xx_hal_pwr.o(i.HAL_PWR_PVDCallback), (2 bytes).
    Removing stm32f4xx_hal_pwr.o(i.HAL_PWR_PVD_IRQHandler), (28 bytes).
    Removing stm32f4xx_hal_sram.o(.rev16_text), (4 bytes).
    Removing stm32f4xx_hal_sram.o(.revsh_text), (4 bytes).
    Removing stm32f4xx_hal_sram.o(.rrx_text), (6 bytes).
    Removing stm32f4xx_hal_sram.o(i.HAL_SRAM_DMA_XferCpltCallback), (2 bytes).
    Removing stm32f4xx_hal_sram.o(i.HAL_SRAM_DMA_XferErrorCallback), (2 bytes).
    Removing stm32f4xx_hal_sram.o(i.HAL_SRAM_DeInit), (28 bytes).
    Removing stm32f4xx_hal_sram.o(i.HAL_SRAM_GetState), (6 bytes).
    Removing stm32f4xx_hal_sram.o(i.HAL_SRAM_Init), (86 bytes).
    Removing stm32f4xx_hal_sram.o(i.HAL_SRAM_MspDeInit), (2 bytes).
    Removing stm32f4xx_hal_sram.o(i.HAL_SRAM_MspInit), (2 bytes).
    Removing stm32f4xx_hal_sram.o(i.HAL_SRAM_Read_16b), (54 bytes).
    Removing stm32f4xx_hal_sram.o(i.HAL_SRAM_Read_32b), (50 bytes).
    Removing stm32f4xx_hal_sram.o(i.HAL_SRAM_Read_8b), (54 bytes).
    Removing stm32f4xx_hal_sram.o(i.HAL_SRAM_Read_DMA), (60 bytes).
    Removing stm32f4xx_hal_sram.o(i.HAL_SRAM_WriteOperation_Disable), (48 bytes).
    Removing stm32f4xx_hal_sram.o(i.HAL_SRAM_WriteOperation_Enable), (42 bytes).
    Removing stm32f4xx_hal_sram.o(i.HAL_SRAM_Write_16b), (66 bytes).
    Removing stm32f4xx_hal_sram.o(i.HAL_SRAM_Write_32b), (62 bytes).
    Removing stm32f4xx_hal_sram.o(i.HAL_SRAM_Write_8b), (66 bytes).
    Removing stm32f4xx_hal_sram.o(i.HAL_SRAM_Write_DMA), (80 bytes).
    Removing stm32f4xx_ll_fsmc.o(.rev16_text), (4 bytes).
    Removing stm32f4xx_ll_fsmc.o(.revsh_text), (4 bytes).
    Removing stm32f4xx_ll_fsmc.o(.rrx_text), (6 bytes).
    Removing stm32f4xx_ll_fsmc.o(i.FSMC_NAND_AttributeSpace_Timing_Init), (50 bytes).
    Removing stm32f4xx_ll_fsmc.o(i.FSMC_NAND_CommonSpace_Timing_Init), (50 bytes).
    Removing stm32f4xx_ll_fsmc.o(i.FSMC_NAND_DeInit), (52 bytes).
    Removing stm32f4xx_ll_fsmc.o(i.FSMC_NAND_ECC_Disable), (26 bytes).
    Removing stm32f4xx_ll_fsmc.o(i.FSMC_NAND_ECC_Enable), (26 bytes).
    Removing stm32f4xx_ll_fsmc.o(i.FSMC_NAND_GetECC), (80 bytes).
    Removing stm32f4xx_ll_fsmc.o(i.FSMC_NAND_Init), (80 bytes).
    Removing stm32f4xx_ll_fsmc.o(i.FSMC_NORSRAM_DeInit), (50 bytes).
    Removing stm32f4xx_ll_fsmc.o(i.FSMC_NORSRAM_Extended_Timing_Init), (64 bytes).
    Removing stm32f4xx_ll_fsmc.o(i.FSMC_NORSRAM_Init), (84 bytes).
    Removing stm32f4xx_ll_fsmc.o(i.FSMC_NORSRAM_Timing_Init), (68 bytes).
    Removing stm32f4xx_ll_fsmc.o(i.FSMC_NORSRAM_WriteOperation_Disable), (16 bytes).
    Removing stm32f4xx_ll_fsmc.o(i.FSMC_NORSRAM_WriteOperation_Enable), (16 bytes).
    Removing stm32f4xx_ll_fsmc.o(i.FSMC_PCCARD_AttributeSpace_Timing_Init), (28 bytes).
    Removing stm32f4xx_ll_fsmc.o(i.FSMC_PCCARD_CommonSpace_Timing_Init), (28 bytes).
    Removing stm32f4xx_ll_fsmc.o(i.FSMC_PCCARD_DeInit), (30 bytes).
    Removing stm32f4xx_ll_fsmc.o(i.FSMC_PCCARD_IOSpace_Timing_Init), (28 bytes).
    Removing stm32f4xx_ll_fsmc.o(i.FSMC_PCCARD_Init), (40 bytes).
    Removing stm32f4xx_hal_cortex.o(.rev16_text), (4 bytes).
    Removing stm32f4xx_hal_cortex.o(.revsh_text), (4 bytes).
    Removing stm32f4xx_hal_cortex.o(.rrx_text), (6 bytes).
    Removing stm32f4xx_hal_cortex.o(i.HAL_MPU_ConfigRegion), (84 bytes).
    Removing stm32f4xx_hal_cortex.o(i.HAL_NVIC_ClearPendingIRQ), (22 bytes).
    Removing stm32f4xx_hal_cortex.o(i.HAL_NVIC_DisableIRQ), (22 bytes).
    Removing stm32f4xx_hal_cortex.o(i.HAL_NVIC_GetActive), (32 bytes).
    Removing stm32f4xx_hal_cortex.o(i.HAL_NVIC_GetPendingIRQ), (32 bytes).
    Removing stm32f4xx_hal_cortex.o(i.HAL_NVIC_GetPriority), (82 bytes).
    Removing stm32f4xx_hal_cortex.o(i.HAL_NVIC_GetPriorityGrouping), (16 bytes).
    Removing stm32f4xx_hal_cortex.o(i.HAL_NVIC_SetPendingIRQ), (22 bytes).
    Removing stm32f4xx_hal_cortex.o(i.HAL_NVIC_SystemReset), (36 bytes).
    Removing stm32f4xx_hal_cortex.o(i.HAL_SYSTICK_CLKSourceConfig), (24 bytes).
    Removing stm32f4xx_hal_cortex.o(i.HAL_SYSTICK_Callback), (2 bytes).
    Removing stm32f4xx_hal_cortex.o(i.HAL_SYSTICK_IRQHandler), (8 bytes).
    Removing stm32f4xx_hal_uart.o(.rev16_text), (4 bytes).
    Removing stm32f4xx_hal_uart.o(.revsh_text), (4 bytes).
    Removing stm32f4xx_hal_uart.o(.rrx_text), (6 bytes).
    Removing stm32f4xx_hal_uart.o(i.HAL_HalfDuplex_EnableReceiver), (50 bytes).
    Removing stm32f4xx_hal_uart.o(i.HAL_HalfDuplex_EnableTransmitter), (50 bytes).
    Removing stm32f4xx_hal_uart.o(i.HAL_HalfDuplex_Init), (108 bytes).
    Removing stm32f4xx_hal_uart.o(i.HAL_LIN_Init), (128 bytes).
    Removing stm32f4xx_hal_uart.o(i.HAL_LIN_SendBreak), (46 bytes).
    Removing stm32f4xx_hal_uart.o(i.HAL_MultiProcessor_EnterMuteMode), (46 bytes).
    Removing stm32f4xx_hal_uart.o(i.HAL_MultiProcessor_ExitMuteMode), (46 bytes).
    Removing stm32f4xx_hal_uart.o(i.HAL_MultiProcessor_Init), (142 bytes).
    Removing stm32f4xx_hal_uart.o(i.HAL_UART_DMAPause), (66 bytes).
    Removing stm32f4xx_hal_uart.o(i.HAL_UART_DMAResume), (74 bytes).
    Removing stm32f4xx_hal_uart.o(i.HAL_UART_DMAStop), (52 bytes).
    Removing stm32f4xx_hal_uart.o(i.HAL_UART_DeInit), (40 bytes).
    Removing stm32f4xx_hal_uart.o(i.HAL_UART_ErrorCallback), (2 bytes).
    Removing stm32f4xx_hal_uart.o(i.HAL_UART_GetError), (4 bytes).
    Removing stm32f4xx_hal_uart.o(i.HAL_UART_GetState), (10 bytes).
    Removing stm32f4xx_hal_uart.o(i.HAL_UART_IRQHandler), (232 bytes).
    Removing stm32f4xx_hal_uart.o(i.HAL_UART_Init), (98 bytes).
    Removing stm32f4xx_hal_uart.o(i.HAL_UART_MspDeInit), (2 bytes).
    Removing stm32f4xx_hal_uart.o(i.HAL_UART_MspInit), (2 bytes).
    Removing stm32f4xx_hal_uart.o(i.HAL_UART_Receive), (172 bytes).
    Removing stm32f4xx_hal_uart.o(i.HAL_UART_Receive_DMA), (120 bytes).
    Removing stm32f4xx_hal_uart.o(i.HAL_UART_Receive_IT), (88 bytes).
    Removing stm32f4xx_hal_uart.o(i.HAL_UART_RxCpltCallback), (2 bytes).
    Removing stm32f4xx_hal_uart.o(i.HAL_UART_RxHalfCpltCallback), (2 bytes).
    Removing stm32f4xx_hal_uart.o(i.HAL_UART_Transmit), (170 bytes).
    Removing stm32f4xx_hal_uart.o(i.HAL_UART_Transmit_DMA), (124 bytes).
    Removing stm32f4xx_hal_uart.o(i.HAL_UART_Transmit_IT), (62 bytes).
    Removing stm32f4xx_hal_uart.o(i.HAL_UART_TxCpltCallback), (2 bytes).
    Removing stm32f4xx_hal_uart.o(i.HAL_UART_TxHalfCpltCallback), (2 bytes).
    Removing stm32f4xx_hal_uart.o(i.UART_DMAError), (34 bytes).
    Removing stm32f4xx_hal_uart.o(i.UART_DMAReceiveCplt), (40 bytes).
    Removing stm32f4xx_hal_uart.o(i.UART_DMARxHalfCplt), (10 bytes).
    Removing stm32f4xx_hal_uart.o(i.UART_DMATransmitCplt), (46 bytes).
    Removing stm32f4xx_hal_uart.o(i.UART_DMATxHalfCplt), (10 bytes).
    Removing stm32f4xx_hal_uart.o(i.UART_Receive_IT), (150 bytes).
    Removing stm32f4xx_hal_uart.o(i.UART_SetConfig), (684 bytes).
    Removing stm32f4xx_hal_uart.o(i.UART_Transmit_IT), (98 bytes).
    Removing stm32f4xx_hal_uart.o(i.UART_WaitOnFlagUntilTimeout), (150 bytes).
    Removing stm32f4xx_hal_i2c.o(.rev16_text), (4 bytes).
    Removing stm32f4xx_hal_i2c.o(.revsh_text), (4 bytes).
    Removing stm32f4xx_hal_i2c.o(.rrx_text), (6 bytes).
    Removing stm32f4xx_hal_i2c.o(i.HAL_I2C_AddrCallback), (2 bytes).
    Removing stm32f4xx_hal_i2c.o(i.HAL_I2C_DisableListen_IT), (68 bytes).
    Removing stm32f4xx_hal_i2c.o(i.HAL_I2C_ER_IRQHandler), (284 bytes).
    Removing stm32f4xx_hal_i2c.o(i.HAL_I2C_EV_IRQHandler), (488 bytes).
    Removing stm32f4xx_hal_i2c.o(i.HAL_I2C_EnableListen_IT), (42 bytes).
    Removing stm32f4xx_hal_i2c.o(i.HAL_I2C_ErrorCallback), (2 bytes).
    Removing stm32f4xx_hal_i2c.o(i.HAL_I2C_GetError), (4 bytes).
    Removing stm32f4xx_hal_i2c.o(i.HAL_I2C_GetMode), (6 bytes).
    Removing stm32f4xx_hal_i2c.o(i.HAL_I2C_ListenCpltCallback), (2 bytes).
    Removing stm32f4xx_hal_i2c.o(i.HAL_I2C_MasterRxCpltCallback), (2 bytes).
    Removing stm32f4xx_hal_i2c.o(i.HAL_I2C_MasterTxCpltCallback), (2 bytes).
    Removing stm32f4xx_hal_i2c.o(i.HAL_I2C_Master_Abort_IT), (92 bytes).
    Removing stm32f4xx_hal_i2c.o(i.HAL_I2C_Master_Receive), (468 bytes).
    Removing stm32f4xx_hal_i2c.o(i.HAL_I2C_Master_Receive_DMA), (260 bytes).
    Removing stm32f4xx_hal_i2c.o(i.HAL_I2C_Master_Receive_IT), (248 bytes).
    Removing stm32f4xx_hal_i2c.o(i.HAL_I2C_Master_Sequential_Receive_IT), (320 bytes).
    Removing stm32f4xx_hal_i2c.o(i.HAL_I2C_Master_Sequential_Transmit_IT), (220 bytes).
    Removing stm32f4xx_hal_i2c.o(i.HAL_I2C_Master_Transmit), (316 bytes).
    Removing stm32f4xx_hal_i2c.o(i.HAL_I2C_Master_Transmit_DMA), (252 bytes).
    Removing stm32f4xx_hal_i2c.o(i.HAL_I2C_Master_Transmit_IT), (200 bytes).
    Removing stm32f4xx_hal_i2c.o(i.HAL_I2C_MemRxCpltCallback), (2 bytes).
    Removing stm32f4xx_hal_i2c.o(i.HAL_I2C_MemTxCpltCallback), (2 bytes).
    Removing stm32f4xx_hal_i2c.o(i.HAL_I2C_Mem_Read), (468 bytes).
    Removing stm32f4xx_hal_i2c.o(i.HAL_I2C_Mem_Read_DMA), (276 bytes).
    Removing stm32f4xx_hal_i2c.o(i.HAL_I2C_Mem_Read_IT), (256 bytes).
    Removing stm32f4xx_hal_i2c.o(i.HAL_I2C_Mem_Write_DMA), (252 bytes).
    Removing stm32f4xx_hal_i2c.o(i.HAL_I2C_Mem_Write_IT), (204 bytes).
    Removing stm32f4xx_hal_i2c.o(i.HAL_I2C_SlaveRxCpltCallback), (2 bytes).
    Removing stm32f4xx_hal_i2c.o(i.HAL_I2C_SlaveTxCpltCallback), (2 bytes).
    Removing stm32f4xx_hal_i2c.o(i.HAL_I2C_Slave_Receive), (284 bytes).
    Removing stm32f4xx_hal_i2c.o(i.HAL_I2C_Slave_Receive_DMA), (204 bytes).
    Removing stm32f4xx_hal_i2c.o(i.HAL_I2C_Slave_Receive_IT), (132 bytes).
    Removing stm32f4xx_hal_i2c.o(i.HAL_I2C_Slave_Sequential_Receive_IT), (92 bytes).
    Removing stm32f4xx_hal_i2c.o(i.HAL_I2C_Slave_Sequential_Transmit_IT), (92 bytes).
    Removing stm32f4xx_hal_i2c.o(i.HAL_I2C_Slave_Transmit), (304 bytes).
    Removing stm32f4xx_hal_i2c.o(i.HAL_I2C_Slave_Transmit_DMA), (240 bytes).
    Removing stm32f4xx_hal_i2c.o(i.HAL_I2C_Slave_Transmit_IT), (132 bytes).
    Removing stm32f4xx_hal_i2c.o(i.I2C_DMAError), (42 bytes).
    Removing stm32f4xx_hal_i2c.o(i.I2C_DMAMasterReceiveCplt), (74 bytes).
    Removing stm32f4xx_hal_i2c.o(i.I2C_DMAMasterTransmitCplt), (84 bytes).
    Removing stm32f4xx_hal_i2c.o(i.I2C_DMAMemReceiveCplt), (74 bytes).
    Removing stm32f4xx_hal_i2c.o(i.I2C_DMAMemTransmitCplt), (84 bytes).
    Removing stm32f4xx_hal_i2c.o(i.I2C_DMASlaveReceiveCplt), (102 bytes).
    Removing stm32f4xx_hal_i2c.o(i.I2C_DMASlaveTransmitCplt), (90 bytes).
    Removing stm32f4xx_hal_i2c.o(i.I2C_MasterReceive_BTF), (232 bytes).
    Removing stm32f4xx_hal_i2c.o(i.I2C_MasterReceive_RXNE), (178 bytes).
    Removing stm32f4xx_hal_i2c.o(i.I2C_MasterRequestRead), (212 bytes).
    Removing stm32f4xx_hal_i2c.o(i.I2C_MasterRequestWrite), (144 bytes).
    Removing stm32f4xx_hal_i2c.o(i.I2C_MasterTransmit_BTF), (134 bytes).
    Removing stm32f4xx_hal_i2c.o(i.I2C_RequestMemoryRead), (226 bytes).
    Removing stm32f4xx_hal_i2c.o(i.I2C_Slave_AF), (148 bytes).
    Removing stm32f4xx_hal_i2c.o(i.I2C_Slave_STOPF), (112 bytes).
    Removing stm32f4xx_hal_i2c.o(i.I2C_WaitOnRXNEFlagUntilTimeout), (104 bytes).
    Removing stm32f4xx_hal_i2c.o(i.I2C_WaitOnSTOPFlagUntilTimeout), (78 bytes).
    Removing stm32f4xx_hal_eth.o(.rev16_text), (4 bytes).
    Removing stm32f4xx_hal_eth.o(.revsh_text), (4 bytes).
    Removing stm32f4xx_hal_eth.o(.rrx_text), (6 bytes).
    Removing stm32f4xx_hal_eth.o(i.HAL_ETH_ConfigDMA), (184 bytes).
    Removing stm32f4xx_hal_eth.o(i.HAL_ETH_DeInit), (26 bytes).
    Removing stm32f4xx_hal_eth.o(i.HAL_ETH_ErrorCallback), (2 bytes).
    Removing stm32f4xx_hal_eth.o(i.HAL_ETH_GetReceivedFrame_IT), (136 bytes).
    Removing stm32f4xx_hal_eth.o(i.HAL_ETH_GetState), (6 bytes).
    Removing stm32f4xx_hal_eth.o(i.HAL_ETH_IRQHandler), (122 bytes).
    Removing stm32f4xx_hal_eth.o(i.HAL_ETH_MspDeInit), (2 bytes).
    Removing stm32f4xx_hal_eth.o(i.HAL_ETH_MspInit), (2 bytes).
    Removing stm32f4xx_hal_eth.o(i.HAL_ETH_RxCpltCallback), (2 bytes).
    Removing stm32f4xx_hal_eth.o(i.HAL_ETH_TxCpltCallback), (2 bytes).
    Removing stm32f4xx_hal_dma.o(.rev16_text), (4 bytes).
    Removing stm32f4xx_hal_dma.o(.revsh_text), (4 bytes).
    Removing stm32f4xx_hal_dma.o(.rrx_text), (6 bytes).
    Removing stm32f4xx_hal_dma.o(i.DMA_CalcBaseAndBitshift), (40 bytes).
    Removing stm32f4xx_hal_dma.o(i.DMA_SetConfig), (40 bytes).
    Removing stm32f4xx_hal_dma.o(i.HAL_DMA_Abort), (84 bytes).
    Removing stm32f4xx_hal_dma.o(i.HAL_DMA_DeInit), (86 bytes).
    Removing stm32f4xx_hal_dma.o(i.HAL_DMA_GetError), (4 bytes).
    Removing stm32f4xx_hal_dma.o(i.HAL_DMA_GetState), (6 bytes).
    Removing stm32f4xx_hal_dma.o(i.HAL_DMA_IRQHandler), (416 bytes).
    Removing stm32f4xx_hal_dma.o(i.HAL_DMA_Init), (120 bytes).
    Removing stm32f4xx_hal_dma.o(i.HAL_DMA_PollForTransfer), (336 bytes).
    Removing stm32f4xx_hal_dma.o(i.HAL_DMA_Start), (58 bytes).
    Removing stm32f4xx_hal_dma.o(i.HAL_DMA_Start_IT), (78 bytes).
    Removing stm32f4xx_hal_dma.o(.constdata), (8 bytes).
    Removing startup_stm32f407xx.o(HEAP), (512 bytes).
    Removing httpserver.o(.rev16_text), (4 bytes).
    Removing httpserver.o(.revsh_text), (4 bytes).
    Removing httpserver.o(.rrx_text), (6 bytes).
    Removing ethernetif.o(.rev16_text), (4 bytes).
    Removing ethernetif.o(.revsh_text), (4 bytes).
    Removing ethernetif.o(.rrx_text), (6 bytes).
    Removing ethernetif.o(i.ethernetif_notify_conn_changed), (2 bytes).
    Removing ethernetif.o(i.ethernetif_set_link), (60 bytes).
    Removing flash_if.o(.rev16_text), (4 bytes).
    Removing flash_if.o(.revsh_text), (4 bytes).
    Removing flash_if.o(.rrx_text), (6 bytes).
    Removing main.o(.rev16_text), (4 bytes).
    Removing main.o(.revsh_text), (4 bytes).
    Removing main.o(.rrx_text), (6 bytes).
    Removing main.o(.data), (1 bytes).
    Removing main.o(.data), (1 bytes).
    Removing main.o(.data), (4 bytes).
    Removing stm32f4xx_it.o(.rev16_text), (4 bytes).
    Removing stm32f4xx_it.o(.revsh_text), (4 bytes).
    Removing stm32f4xx_it.o(.rrx_text), (6 bytes).
    Removing app_ethernet.o(.rev16_text), (4 bytes).
    Removing app_ethernet.o(.revsh_text), (4 bytes).
    Removing app_ethernet.o(.rrx_text), (6 bytes).
    Removing tftpserver.o(.rev16_text), (4 bytes).
    Removing tftpserver.o(.revsh_text), (4 bytes).
    Removing tftpserver.o(.rrx_text), (6 bytes).
    Removing stm324xg_eval_eeprom.o(.rev16_text), (4 bytes).
    Removing stm324xg_eval_eeprom.o(.revsh_text), (4 bytes).
    Removing stm324xg_eval_eeprom.o(.rrx_text), (6 bytes).
    Removing stm324xg_eval_eeprom.o(i.BSP_EEPROM_Init), (24 bytes).
    Removing stm324xg_eval_eeprom.o(i.BSP_EEPROM_ReadBuffer), (24 bytes).
    Removing stm324xg_eval_eeprom.o(.data), (4 bytes).
    Removing stm324xg_eval_eeprom.o(.data), (2 bytes).
    Removing stm324xg_eval.o(.rev16_text), (4 bytes).
    Removing stm324xg_eval.o(.revsh_text), (4 bytes).
    Removing stm324xg_eval.o(.rrx_text), (6 bytes).
    Removing stm324xg_eval.o(i.EEPROM_IO_Init), (2 bytes).
    Removing stm324xg_eval.o(i.EEPROM_IO_ReadData), (44 bytes).
    Removing dadd.o(.text), (334 bytes).
    Removing dmul.o(.text), (228 bytes).
    Removing ddiv.o(.text), (222 bytes).
    Removing dfixul.o(.text), (48 bytes).
    Removing cdrcmple.o(.text), (48 bytes).
    Removing depilogue.o(.text), (186 bytes).

366 unused section(s) (total 24121 bytes) removed from the image.

==============================================================================

Image Symbol Table

    Local Symbols

    Symbol Name                              Value     Ov Type        Size  Object(Section)

    ../clib/microlib/division.c              0x00000000   Number         0  uidiv.o ABSOLUTE
    ../clib/microlib/division.c              0x00000000   Number         0  uldiv.o ABSOLUTE
    ../clib/microlib/init/entry.s            0x00000000   Number         0  entry.o ABSOLUTE
    ../clib/microlib/init/entry.s            0x00000000   Number         0  entry10a.o ABSOLUTE
    ../clib/microlib/init/entry.s            0x00000000   Number         0  entry7a.o ABSOLUTE
    ../clib/microlib/init/entry.s            0x00000000   Number         0  entry11a.o ABSOLUTE
    ../clib/microlib/init/entry.s            0x00000000   Number         0  entry7b.o ABSOLUTE
    ../clib/microlib/init/entry.s            0x00000000   Number         0  entry8a.o ABSOLUTE
    ../clib/microlib/init/entry.s            0x00000000   Number         0  entry8b.o ABSOLUTE
    ../clib/microlib/init/entry.s            0x00000000   Number         0  entry11b.o ABSOLUTE
    ../clib/microlib/init/entry.s            0x00000000   Number         0  entry9a.o ABSOLUTE
    ../clib/microlib/init/entry.s            0x00000000   Number         0  entry2.o ABSOLUTE
    ../clib/microlib/init/entry.s            0x00000000   Number         0  entry10b.o ABSOLUTE
    ../clib/microlib/init/entry.s            0x00000000   Number         0  entry9b.o ABSOLUTE
    ../clib/microlib/init/entry.s            0x00000000   Number         0  entry5.o ABSOLUTE
    ../clib/microlib/longlong.c              0x00000000   Number         0  llshl.o ABSOLUTE
    ../clib/microlib/longlong.c              0x00000000   Number         0  llushr.o ABSOLUTE
    ../clib/microlib/longlong.c              0x00000000   Number         0  llsshr.o ABSOLUTE
    ../clib/microlib/printf/printf.c         0x00000000   Number         0  printf5.o ABSOLUTE
    ../clib/microlib/printf/printf.c         0x00000000   Number         0  printf6.o ABSOLUTE
    ../clib/microlib/printf/printf.c         0x00000000   Number         0  printf7.o ABSOLUTE
    ../clib/microlib/printf/printf.c         0x00000000   Number         0  printf8.o ABSOLUTE
    ../clib/microlib/printf/printf.c         0x00000000   Number         0  printfa.o ABSOLUTE
    ../clib/microlib/printf/printf.c         0x00000000   Number         0  printf0.o ABSOLUTE
    ../clib/microlib/printf/printf.c         0x00000000   Number         0  printf4.o ABSOLUTE
    ../clib/microlib/printf/printf.c         0x00000000   Number         0  printfb.o ABSOLUTE
    ../clib/microlib/printf/printf.c         0x00000000   Number         0  printf1.o ABSOLUTE
    ../clib/microlib/printf/printf.c         0x00000000   Number         0  printf2.o ABSOLUTE
    ../clib/microlib/printf/printf.c         0x00000000   Number         0  printf3.o ABSOLUTE
    ../clib/microlib/printf/stubs.s          0x00000000   Number         0  stubs.o ABSOLUTE
    ../clib/microlib/stdio/fputc.c           0x00000000   Number         0  fputc.o ABSOLUTE
    ../clib/microlib/stdio/semi.s            0x00000000   Number         0  semi.o ABSOLUTE
    ../clib/microlib/stdio/streams.c         0x00000000   Number         0  stdout.o ABSOLUTE
    ../clib/microlib/string/memcmp.c         0x00000000   Number         0  memcmp.o ABSOLUTE
    ../clib/microlib/string/memcpy.c         0x00000000   Number         0  memcpyb.o ABSOLUTE
    ../clib/microlib/string/memcpy.c         0x00000000   Number         0  memcpya.o ABSOLUTE
    ../clib/microlib/string/memset.c         0x00000000   Number         0  memseta.o ABSOLUTE
    ../clib/microlib/string/strcmp.c         0x00000000   Number         0  strcmp.o ABSOLUTE
    ../clib/microlib/string/strlen.c         0x00000000   Number         0  strlen.o ABSOLUTE
    ../clib/microlib/string/strncmp.c        0x00000000   Number         0  strncmp.o ABSOLUTE
    ../clib/microlib/stubs.s                 0x00000000   Number         0  iusefp.o ABSOLUTE
    ../clib/microlib/stubs.s                 0x00000000   Number         0  iusesemip.o ABSOLUTE
    ../fplib/microlib/fpadd.c                0x00000000   Number         0  dadd.o ABSOLUTE
    ../fplib/microlib/fpdiv.c                0x00000000   Number         0  ddiv.o ABSOLUTE
    ../fplib/microlib/fpepilogue.c           0x00000000   Number         0  depilogue.o ABSOLUTE
    ../fplib/microlib/fpfix.c                0x00000000   Number         0  dfixul.o ABSOLUTE
    ../fplib/microlib/fpmul.c                0x00000000   Number         0  dmul.o ABSOLUTE
    ..\..\..\..\..\..\Drivers\BSP\STM324xG_EVAL\stm324xg_eval.c 0x00000000   Number         0  stm324xg_eval.o ABSOLUTE
    ..\..\..\..\..\..\Drivers\BSP\STM324xG_EVAL\stm324xg_eval_eeprom.c 0x00000000   Number         0  stm324xg_eval_eeprom.o ABSOLUTE
    ..\..\..\..\..\..\Drivers\STM32F4xx_HAL_Driver\Src\stm32f4xx_hal.c 0x00000000   Number         0  stm32f4xx_hal.o ABSOLUTE
    ..\..\..\..\..\..\Drivers\STM32F4xx_HAL_Driver\Src\stm32f4xx_hal_cortex.c 0x00000000   Number         0  stm32f4xx_hal_cortex.o ABSOLUTE
    ..\..\..\..\..\..\Drivers\STM32F4xx_HAL_Driver\Src\stm32f4xx_hal_dma.c 0x00000000   Number         0  stm32f4xx_hal_dma.o ABSOLUTE
    ..\..\..\..\..\..\Drivers\STM32F4xx_HAL_Driver\Src\stm32f4xx_hal_eth.c 0x00000000   Number         0  stm32f4xx_hal_eth.o ABSOLUTE
    ..\..\..\..\..\..\Drivers\STM32F4xx_HAL_Driver\Src\stm32f4xx_hal_flash.c 0x00000000   Number         0  stm32f4xx_hal_flash.o ABSOLUTE
    ..\..\..\..\..\..\Drivers\STM32F4xx_HAL_Driver\Src\stm32f4xx_hal_flash_ex.c 0x00000000   Number         0  stm32f4xx_hal_flash_ex.o ABSOLUTE
    ..\..\..\..\..\..\Drivers\STM32F4xx_HAL_Driver\Src\stm32f4xx_hal_gpio.c 0x00000000   Number         0  stm32f4xx_hal_gpio.o ABSOLUTE
    ..\..\..\..\..\..\Drivers\STM32F4xx_HAL_Driver\Src\stm32f4xx_hal_i2c.c 0x00000000   Number         0  stm32f4xx_hal_i2c.o ABSOLUTE
    ..\..\..\..\..\..\Drivers\STM32F4xx_HAL_Driver\Src\stm32f4xx_hal_i2s.c 0x00000000   Number         0  stm32f4xx_hal_i2s.o ABSOLUTE
    ..\..\..\..\..\..\Drivers\STM32F4xx_HAL_Driver\Src\stm32f4xx_hal_i2s_ex.c 0x00000000   Number         0  stm32f4xx_hal_i2s_ex.o ABSOLUTE
    ..\..\..\..\..\..\Drivers\STM32F4xx_HAL_Driver\Src\stm32f4xx_hal_pwr.c 0x00000000   Number         0  stm32f4xx_hal_pwr.o ABSOLUTE
    ..\..\..\..\..\..\Drivers\STM32F4xx_HAL_Driver\Src\stm32f4xx_hal_rcc.c 0x00000000   Number         0  stm32f4xx_hal_rcc.o ABSOLUTE
    ..\..\..\..\..\..\Drivers\STM32F4xx_HAL_Driver\Src\stm32f4xx_hal_sram.c 0x00000000   Number         0  stm32f4xx_hal_sram.o ABSOLUTE
    ..\..\..\..\..\..\Drivers\STM32F4xx_HAL_Driver\Src\stm32f4xx_hal_uart.c 0x00000000   Number         0  stm32f4xx_hal_uart.o ABSOLUTE
    ..\..\..\..\..\..\Drivers\STM32F4xx_HAL_Driver\Src\stm32f4xx_ll_fsmc.c 0x00000000   Number         0  stm32f4xx_ll_fsmc.o ABSOLUTE
    ..\..\..\..\..\..\Middlewares\Third_Party\LwIP\src\api\api_lib.c 0x00000000   Number         0  api_lib.o ABSOLUTE
    ..\..\..\..\..\..\Middlewares\Third_Party\LwIP\src\api\api_msg.c 0x00000000   Number         0  api_msg.o ABSOLUTE
    ..\..\..\..\..\..\Middlewares\Third_Party\LwIP\src\api\err.c 0x00000000   Number         0  err.o ABSOLUTE
    ..\..\..\..\..\..\Middlewares\Third_Party\LwIP\src\api\netbuf.c 0x00000000   Number         0  netbuf.o ABSOLUTE
    ..\..\..\..\..\..\Middlewares\Third_Party\LwIP\src\api\netdb.c 0x00000000   Number         0  netdb.o ABSOLUTE
    ..\..\..\..\..\..\Middlewares\Third_Party\LwIP\src\api\netifapi.c 0x00000000   Number         0  netifapi.o ABSOLUTE
    ..\..\..\..\..\..\Middlewares\Third_Party\LwIP\src\api\sockets.c 0x00000000   Number         0  sockets.o ABSOLUTE
    ..\..\..\..\..\..\Middlewares\Third_Party\LwIP\src\api\tcpip.c 0x00000000   Number         0  tcpip.o ABSOLUTE
    ..\..\..\..\..\..\Middlewares\Third_Party\LwIP\src\core\def.c 0x00000000   Number         0  def.o ABSOLUTE
    ..\..\..\..\..\..\Middlewares\Third_Party\LwIP\src\core\dhcp.c 0x00000000   Number         0  dhcp.o ABSOLUTE
    ..\..\..\..\..\..\Middlewares\Third_Party\LwIP\src\core\dns.c 0x00000000   Number         0  dns.o ABSOLUTE
    ..\..\..\..\..\..\Middlewares\Third_Party\LwIP\src\core\init.c 0x00000000   Number         0  init.o ABSOLUTE
    ..\..\..\..\..\..\Middlewares\Third_Party\LwIP\src\core\ipv4\autoip.c 0x00000000   Number         0  autoip.o ABSOLUTE
    ..\..\..\..\..\..\Middlewares\Third_Party\LwIP\src\core\ipv4\icmp.c 0x00000000   Number         0  icmp.o ABSOLUTE
    ..\..\..\..\..\..\Middlewares\Third_Party\LwIP\src\core\ipv4\igmp.c 0x00000000   Number         0  igmp.o ABSOLUTE
    ..\..\..\..\..\..\Middlewares\Third_Party\LwIP\src\core\ipv4\inet.c 0x00000000   Number         0  inet.o ABSOLUTE
    ..\..\..\..\..\..\Middlewares\Third_Party\LwIP\src\core\ipv4\inet_chksum.c 0x00000000   Number         0  inet_chksum.o ABSOLUTE
    ..\..\..\..\..\..\Middlewares\Third_Party\LwIP\src\core\ipv4\ip.c 0x00000000   Number         0  ip.o ABSOLUTE
    ..\..\..\..\..\..\Middlewares\Third_Party\LwIP\src\core\ipv4\ip_addr.c 0x00000000   Number         0  ip_addr.o ABSOLUTE
    ..\..\..\..\..\..\Middlewares\Third_Party\LwIP\src\core\ipv4\ip_frag.c 0x00000000   Number         0  ip_frag.o ABSOLUTE
    ..\..\..\..\..\..\Middlewares\Third_Party\LwIP\src\core\lwip_timers.c 0x00000000   Number         0  lwip_timers.o ABSOLUTE
    ..\..\..\..\..\..\Middlewares\Third_Party\LwIP\src\core\mem.c 0x00000000   Number         0  mem.o ABSOLUTE
    ..\..\..\..\..\..\Middlewares\Third_Party\LwIP\src\core\memp.c 0x00000000   Number         0  memp.o ABSOLUTE
    ..\..\..\..\..\..\Middlewares\Third_Party\LwIP\src\core\netif.c 0x00000000   Number         0  netif.o ABSOLUTE
    ..\..\..\..\..\..\Middlewares\Third_Party\LwIP\src\core\pbuf.c 0x00000000   Number         0  pbuf.o ABSOLUTE
    ..\..\..\..\..\..\Middlewares\Third_Party\LwIP\src\core\raw.c 0x00000000   Number         0  raw.o ABSOLUTE
    ..\..\..\..\..\..\Middlewares\Third_Party\LwIP\src\core\stats.c 0x00000000   Number         0  stats.o ABSOLUTE
    ..\..\..\..\..\..\Middlewares\Third_Party\LwIP\src\core\sys.c 0x00000000   Number         0  sys.o ABSOLUTE
    ..\..\..\..\..\..\Middlewares\Third_Party\LwIP\src\core\tcp.c 0x00000000   Number         0  tcp.o ABSOLUTE
    ..\..\..\..\..\..\Middlewares\Third_Party\LwIP\src\core\tcp_in.c 0x00000000   Number         0  tcp_in.o ABSOLUTE
    ..\..\..\..\..\..\Middlewares\Third_Party\LwIP\src\core\tcp_out.c 0x00000000   Number         0  tcp_out.o ABSOLUTE
    ..\..\..\..\..\..\Middlewares\Third_Party\LwIP\src\core\udp.c 0x00000000   Number         0  udp.o ABSOLUTE
    ..\..\..\..\..\..\Middlewares\Third_Party\LwIP\src\netif\etharp.c 0x00000000   Number         0  etharp.o ABSOLUTE
    ..\Src\app_ethernet.c                    0x00000000   Number         0  app_ethernet.o ABSOLUTE
    ..\Src\ethernetif.c                      0x00000000   Number         0  ethernetif.o ABSOLUTE
    ..\Src\flash_if.c                        0x00000000   Number         0  flash_if.o ABSOLUTE
    ..\Src\httpserver.c                      0x00000000   Number         0  httpserver.o ABSOLUTE
    ..\Src\main.c                            0x00000000   Number         0  main.o ABSOLUTE
    ..\Src\stm32f4xx_it.c                    0x00000000   Number         0  stm32f4xx_it.o ABSOLUTE
    ..\Src\system_stm32f4xx.c                0x00000000   Number         0  system_stm32f4xx.o ABSOLUTE
    ..\Src\tftpserver.c                      0x00000000   Number         0  tftpserver.o ABSOLUTE
    ..\\..\\..\\..\\..\\..\\Drivers\\BSP\\STM324xG_EVAL\\stm324xg_eval.c 0x00000000   Number         0  stm324xg_eval.o ABSOLUTE
    ..\\..\\..\\..\\..\\..\\Drivers\\BSP\\STM324xG_EVAL\\stm324xg_eval_eeprom.c 0x00000000   Number         0  stm324xg_eval_eeprom.o ABSOLUTE
    ..\\..\\..\\..\\..\\..\\Drivers\\STM32F4xx_HAL_Driver\\Src\\stm32f4xx_hal.c 0x00000000   Number         0  stm32f4xx_hal.o ABSOLUTE
    ..\\..\\..\\..\\..\\..\\Drivers\\STM32F4xx_HAL_Driver\\Src\\stm32f4xx_hal_cortex.c 0x00000000   Number         0  stm32f4xx_hal_cortex.o ABSOLUTE
    ..\\..\\..\\..\\..\\..\\Drivers\\STM32F4xx_HAL_Driver\\Src\\stm32f4xx_hal_dma.c 0x00000000   Number         0  stm32f4xx_hal_dma.o ABSOLUTE
    ..\\..\\..\\..\\..\\..\\Drivers\\STM32F4xx_HAL_Driver\\Src\\stm32f4xx_hal_eth.c 0x00000000   Number         0  stm32f4xx_hal_eth.o ABSOLUTE
    ..\\..\\..\\..\\..\\..\\Drivers\\STM32F4xx_HAL_Driver\\Src\\stm32f4xx_hal_flash.c 0x00000000   Number         0  stm32f4xx_hal_flash.o ABSOLUTE
    ..\\..\\..\\..\\..\\..\\Drivers\\STM32F4xx_HAL_Driver\\Src\\stm32f4xx_hal_flash_ex.c 0x00000000   Number         0  stm32f4xx_hal_flash_ex.o ABSOLUTE
    ..\\..\\..\\..\\..\\..\\Drivers\\STM32F4xx_HAL_Driver\\Src\\stm32f4xx_hal_gpio.c 0x00000000   Number         0  stm32f4xx_hal_gpio.o ABSOLUTE
    ..\\..\\..\\..\\..\\..\\Drivers\\STM32F4xx_HAL_Driver\\Src\\stm32f4xx_hal_i2c.c 0x00000000   Number         0  stm32f4xx_hal_i2c.o ABSOLUTE
    ..\\..\\..\\..\\..\\..\\Drivers\\STM32F4xx_HAL_Driver\\Src\\stm32f4xx_hal_i2s.c 0x00000000   Number         0  stm32f4xx_hal_i2s.o ABSOLUTE
    ..\\..\\..\\..\\..\\..\\Drivers\\STM32F4xx_HAL_Driver\\Src\\stm32f4xx_hal_i2s_ex.c 0x00000000   Number         0  stm32f4xx_hal_i2s_ex.o ABSOLUTE
    ..\\..\\..\\..\\..\\..\\Drivers\\STM32F4xx_HAL_Driver\\Src\\stm32f4xx_hal_pwr.c 0x00000000   Number         0  stm32f4xx_hal_pwr.o ABSOLUTE
    ..\\..\\..\\..\\..\\..\\Drivers\\STM32F4xx_HAL_Driver\\Src\\stm32f4xx_hal_rcc.c 0x00000000   Number         0  stm32f4xx_hal_rcc.o ABSOLUTE
    ..\\..\\..\\..\\..\\..\\Drivers\\STM32F4xx_HAL_Driver\\Src\\stm32f4xx_hal_sram.c 0x00000000   Number         0  stm32f4xx_hal_sram.o ABSOLUTE
    ..\\..\\..\\..\\..\\..\\Drivers\\STM32F4xx_HAL_Driver\\Src\\stm32f4xx_hal_uart.c 0x00000000   Number         0  stm32f4xx_hal_uart.o ABSOLUTE
    ..\\..\\..\\..\\..\\..\\Drivers\\STM32F4xx_HAL_Driver\\Src\\stm32f4xx_ll_fsmc.c 0x00000000   Number         0  stm32f4xx_ll_fsmc.o ABSOLUTE
    ..\\Src\\app_ethernet.c                  0x00000000   Number         0  app_ethernet.o ABSOLUTE
    ..\\Src\\ethernetif.c                    0x00000000   Number         0  ethernetif.o ABSOLUTE
    ..\\Src\\flash_if.c                      0x00000000   Number         0  flash_if.o ABSOLUTE
    ..\\Src\\httpserver.c                    0x00000000   Number         0  httpserver.o ABSOLUTE
    ..\\Src\\main.c                          0x00000000   Number         0  main.o ABSOLUTE
    ..\\Src\\stm32f4xx_it.c                  0x00000000   Number         0  stm32f4xx_it.o ABSOLUTE
    ..\\Src\\system_stm32f4xx.c              0x00000000   Number         0  system_stm32f4xx.o ABSOLUTE
    ..\\Src\\tftpserver.c                    0x00000000   Number         0  tftpserver.o ABSOLUTE
    cdrcmple.s                               0x00000000   Number         0  cdrcmple.o ABSOLUTE
    dc.s                                     0x00000000   Number         0  dc.o ABSOLUTE
    handlers.s                               0x00000000   Number         0  handlers.o ABSOLUTE
    init.s                                   0x00000000   Number         0  init.o ABSOLUTE
    startup_stm32f407xx.s                    0x00000000   Number         0  startup_stm32f407xx.o ABSOLUTE
    RESET                                    0x08000000   Section      392  startup_stm32f407xx.o(RESET)
    .ARM.Collect$$$$00000000                 0x08000188   Section        0  entry.o(.ARM.Collect$$$$00000000)
    .ARM.Collect$$$$00000001                 0x08000188   Section        4  entry2.o(.ARM.Collect$$$$00000001)
    .ARM.Collect$$$$00000004                 0x0800018c   Section        4  entry5.o(.ARM.Collect$$$$00000004)
    .ARM.Collect$$$$00000008                 0x08000190   Section        0  entry7b.o(.ARM.Collect$$$$00000008)
    .ARM.Collect$$$$0000000A                 0x08000190   Section        0  entry8b.o(.ARM.Collect$$$$0000000A)
    .ARM.Collect$$$$0000000B                 0x08000190   Section        8  entry9a.o(.ARM.Collect$$$$0000000B)
    .ARM.Collect$$$$0000000D                 0x08000198   Section        0  entry10a.o(.ARM.Collect$$$$0000000D)
    .ARM.Collect$$$$0000000F                 0x08000198   Section        0  entry11a.o(.ARM.Collect$$$$0000000F)
    .ARM.Collect$$$$00002712                 0x08000198   Section        4  entry2.o(.ARM.Collect$$$$00002712)
    __lit__00000000                          0x08000198   Data           4  entry2.o(.ARM.Collect$$$$00002712)
    .text                                    0x0800019c   Section       36  startup_stm32f407xx.o(.text)
    $v0                                      0x0800019c   Number         0  startup_stm32f407xx.o(.text)
    .text                                    0x080001c0   Section        0  memcpya.o(.text)
    .text                                    0x080001e4   Section        0  memseta.o(.text)
    .text                                    0x08000208   Section        0  strcmp.o(.text)
    .text                                    0x08000224   Section        0  memcmp.o(.text)
    .text                                    0x0800023e   Section        0  strncmp.o(.text)
    .text                                    0x0800025c   Section       36  init.o(.text)
    i.BSP_EEPROM_TIMEOUT_UserCallback        0x08000280   Section        0  stm324xg_eval_eeprom.o(i.BSP_EEPROM_TIMEOUT_UserCallback)
    i.BSP_EEPROM_WriteBuffer                 0x08000282   Section        0  stm324xg_eval_eeprom.o(i.BSP_EEPROM_WriteBuffer)
    i.BusFault_Handler                       0x0800037a   Section        0  stm32f4xx_it.o(i.BusFault_Handler)
    i.DebugMon_Handler                       0x0800037c   Section        0  stm32f4xx_it.o(i.DebugMon_Handler)
    i.EEPROM_IO_IsDeviceReady                0x08000380   Section        0  stm324xg_eval.o(i.EEPROM_IO_IsDeviceReady)
    i.EEPROM_IO_WriteData                    0x08000390   Section        0  stm324xg_eval.o(i.EEPROM_IO_WriteData)
    i.EEPROM_WritePage                       0x080003bc   Section        0  stm324xg_eval_eeprom.o(i.EEPROM_WritePage)
    EEPROM_WritePage                         0x080003bd   Thumb Code    50  stm324xg_eval_eeprom.o(i.EEPROM_WritePage)
    i.ETH_FlushTransmitFIFO                  0x080003f4   Section        0  stm32f4xx_hal_eth.o(i.ETH_FlushTransmitFIFO)
    ETH_FlushTransmitFIFO                    0x080003f5   Thumb Code    46  stm32f4xx_hal_eth.o(i.ETH_FlushTransmitFIFO)
    i.ETH_MACDMAConfig                       0x08000424   Section        0  stm32f4xx_hal_eth.o(i.ETH_MACDMAConfig)
    ETH_MACDMAConfig                         0x08000425   Thumb Code   266  stm32f4xx_hal_eth.o(i.ETH_MACDMAConfig)
    i.EXTI15_10_IRQHandler                   0x08000548   Section        0  stm32f4xx_it.o(i.EXTI15_10_IRQHandler)
    i.FLASH_Erase_Sector                     0x08000550   Section        0  stm32f4xx_hal_flash_ex.o(i.FLASH_Erase_Sector)
    i.FLASH_FlushCaches                      0x080005a8   Section        0  stm32f4xx_hal_flash_ex.o(i.FLASH_FlushCaches)
    i.FLASH_If_Erase                         0x080005fc   Section        0  flash_if.o(i.FLASH_If_Erase)
    i.FLASH_If_Init                          0x08000630   Section        0  flash_if.o(i.FLASH_If_Init)
    i.FLASH_If_Write                         0x08000634   Section        0  flash_if.o(i.FLASH_If_Write)
    i.FLASH_MassErase                        0x08000684   Section        0  stm32f4xx_hal_flash_ex.o(i.FLASH_MassErase)
    FLASH_MassErase                          0x08000685   Thumb Code    34  stm32f4xx_hal_flash_ex.o(i.FLASH_MassErase)
    i.FLASH_Program_Byte                     0x080006ac   Section        0  stm32f4xx_hal_flash.o(i.FLASH_Program_Byte)
    FLASH_Program_Byte                       0x080006ad   Thumb Code    26  stm32f4xx_hal_flash.o(i.FLASH_Program_Byte)
    i.FLASH_Program_DoubleWord               0x080006cc   Section        0  stm32f4xx_hal_flash.o(i.FLASH_Program_DoubleWord)
    FLASH_Program_DoubleWord                 0x080006cd   Thumb Code    34  stm32f4xx_hal_flash.o(i.FLASH_Program_DoubleWord)
    i.FLASH_Program_HalfWord                 0x080006f4   Section        0  stm32f4xx_hal_flash.o(i.FLASH_Program_HalfWord)
    FLASH_Program_HalfWord                   0x080006f5   Thumb Code    30  stm32f4xx_hal_flash.o(i.FLASH_Program_HalfWord)
    i.FLASH_Program_Word                     0x08000718   Section        0  stm32f4xx_hal_flash.o(i.FLASH_Program_Word)
    FLASH_Program_Word                       0x08000719   Thumb Code    30  stm32f4xx_hal_flash.o(i.FLASH_Program_Word)
    i.FLASH_SetErrorCode                     0x0800073c   Section        0  stm32f4xx_hal_flash.o(i.FLASH_SetErrorCode)
    FLASH_SetErrorCode                       0x0800073d   Thumb Code   128  stm32f4xx_hal_flash.o(i.FLASH_SetErrorCode)
    i.FLASH_WaitForLastOperation             0x080007c4   Section        0  stm32f4xx_hal_flash.o(i.FLASH_WaitForLastOperation)
    i.HAL_Delay                              0x0800081c   Section        0  stm32f4xx_hal.o(i.HAL_Delay)
    i.HAL_ETH_ConfigMAC                      0x08000834   Section        0  stm32f4xx_hal_eth.o(i.HAL_ETH_ConfigMAC)
    i.HAL_ETH_DMARxDescListInit              0x08000964   Section        0  stm32f4xx_hal_eth.o(i.HAL_ETH_DMARxDescListInit)
    i.HAL_ETH_DMATxDescListInit              0x080009d8   Section        0  stm32f4xx_hal_eth.o(i.HAL_ETH_DMATxDescListInit)
    i.HAL_ETH_GetReceivedFrame               0x08000a50   Section        0  stm32f4xx_hal_eth.o(i.HAL_ETH_GetReceivedFrame)
    i.HAL_ETH_Init                           0x08000acc   Section        0  stm32f4xx_hal_eth.o(i.HAL_ETH_Init)
    i.HAL_ETH_MspInit                        0x08000cb8   Section        0  ethernetif.o(i.HAL_ETH_MspInit)
    i.HAL_ETH_ReadPHYRegister                0x08000cbc   Section        0  stm32f4xx_hal_eth.o(i.HAL_ETH_ReadPHYRegister)
    i.HAL_ETH_Start                          0x08000d40   Section        0  stm32f4xx_hal_eth.o(i.HAL_ETH_Start)
    i.HAL_ETH_Stop                           0x08000dc4   Section        0  stm32f4xx_hal_eth.o(i.HAL_ETH_Stop)
    i.HAL_ETH_TransmitFrame                  0x08000e48   Section        0  stm32f4xx_hal_eth.o(i.HAL_ETH_TransmitFrame)
    i.HAL_ETH_WritePHYRegister               0x08000f50   Section        0  stm32f4xx_hal_eth.o(i.HAL_ETH_WritePHYRegister)
    i.HAL_FLASHEx_Erase                      0x08000fc8   Section        0  stm32f4xx_hal_flash_ex.o(i.HAL_FLASHEx_Erase)
    i.HAL_FLASH_Program                      0x08001060   Section        0  stm32f4xx_hal_flash.o(i.HAL_FLASH_Program)
    i.HAL_FLASH_Unlock                       0x080010dc   Section        0  stm32f4xx_hal_flash.o(i.HAL_FLASH_Unlock)
    i.HAL_GPIO_EXTI_Callback                 0x08001104   Section        0  stm32f4xx_hal_gpio.o(i.HAL_GPIO_EXTI_Callback)
    i.HAL_GPIO_EXTI_IRQHandler               0x08001108   Section        0  stm32f4xx_hal_gpio.o(i.HAL_GPIO_EXTI_IRQHandler)
    i.HAL_GPIO_Init                          0x08001120   Section        0  stm32f4xx_hal_gpio.o(i.HAL_GPIO_Init)
    i.HAL_GPIO_ReadPin                       0x080012e0   Section        0  stm32f4xx_hal_gpio.o(i.HAL_GPIO_ReadPin)
    i.HAL_GPIO_WritePin                      0x080012ea   Section        0  stm32f4xx_hal_gpio.o(i.HAL_GPIO_WritePin)
    i.HAL_GetREVID                           0x080012f4   Section        0  stm32f4xx_hal.o(i.HAL_GetREVID)
    i.HAL_GetTick                            0x08001300   Section        0  stm32f4xx_hal.o(i.HAL_GetTick)
    i.HAL_I2C_DeInit                         0x0800130c   Section        0  stm32f4xx_hal_i2c.o(i.HAL_I2C_DeInit)
    i.HAL_I2C_GetState                       0x0800133e   Section        0  stm32f4xx_hal_i2c.o(i.HAL_I2C_GetState)
    i.HAL_I2C_Init                           0x08001344   Section        0  stm32f4xx_hal_i2c.o(i.HAL_I2C_Init)
    i.HAL_I2C_IsDeviceReady                  0x0800144c   Section        0  stm32f4xx_hal_i2c.o(i.HAL_I2C_IsDeviceReady)
    i.HAL_I2C_Mem_Write                      0x08001598   Section        0  stm32f4xx_hal_i2c.o(i.HAL_I2C_Mem_Write)
    i.HAL_I2C_MspDeInit                      0x0800168c   Section        0  stm32f4xx_hal_i2c.o(i.HAL_I2C_MspDeInit)
    i.HAL_I2C_MspInit                        0x0800168e   Section        0  stm32f4xx_hal_i2c.o(i.HAL_I2C_MspInit)
    i.HAL_IncTick                            0x08001690   Section        0  stm32f4xx_hal.o(i.HAL_IncTick)
    i.HAL_Init                               0x080016a0   Section        0  stm32f4xx_hal.o(i.HAL_Init)
    i.HAL_InitTick                           0x080016cc   Section        0  stm32f4xx_hal.o(i.HAL_InitTick)
    i.HAL_MspInit                            0x080016ee   Section        0  stm32f4xx_hal.o(i.HAL_MspInit)
    i.HAL_NVIC_EnableIRQ                     0x080016f0   Section        0  stm32f4xx_hal_cortex.o(i.HAL_NVIC_EnableIRQ)
    i.HAL_NVIC_SetPriority                   0x08001708   Section        0  stm32f4xx_hal_cortex.o(i.HAL_NVIC_SetPriority)
    i.HAL_NVIC_SetPriorityGrouping           0x08001748   Section        0  stm32f4xx_hal_cortex.o(i.HAL_NVIC_SetPriorityGrouping)
    i.HAL_RCC_ClockConfig                    0x0800176c   Section        0  stm32f4xx_hal_rcc.o(i.HAL_RCC_ClockConfig)
    i.HAL_RCC_GetHCLKFreq                    0x080018ac   Section        0  stm32f4xx_hal_rcc.o(i.HAL_RCC_GetHCLKFreq)
    i.HAL_RCC_GetPCLK1Freq                   0x080018e0   Section        0  stm32f4xx_hal_rcc.o(i.HAL_RCC_GetPCLK1Freq)
    i.HAL_RCC_GetSysClockFreq                0x0800190c   Section        0  stm32f4xx_hal_rcc.o(i.HAL_RCC_GetSysClockFreq)
    i.HAL_RCC_OscConfig                      0x08001980   Section        0  stm32f4xx_hal_rcc.o(i.HAL_RCC_OscConfig)
    i.HAL_SYSTICK_Config                     0x08001c64   Section        0  stm32f4xx_hal_cortex.o(i.HAL_SYSTICK_Config)
    i.HardFault_Handler                      0x08001c8c   Section        0  stm32f4xx_it.o(i.HardFault_Handler)
    i.I2C_Config                             0x08001c90   Section        0  main.o(i.I2C_Config)
    i.I2C_IsAcknowledgeFailed                0x08001cf8   Section        0  stm32f4xx_hal_i2c.o(i.I2C_IsAcknowledgeFailed)
    I2C_IsAcknowledgeFailed                  0x08001cf9   Thumb Code    40  stm32f4xx_hal_i2c.o(i.I2C_IsAcknowledgeFailed)
    i.I2C_RequestMemoryWrite                 0x08001d20   Section        0  stm32f4xx_hal_i2c.o(i.I2C_RequestMemoryWrite)
    I2C_RequestMemoryWrite                   0x08001d21   Thumb Code   146  stm32f4xx_hal_i2c.o(i.I2C_RequestMemoryWrite)
    i.I2C_WaitOnFlagUntilTimeout             0x08001db8   Section        0  stm32f4xx_hal_i2c.o(i.I2C_WaitOnFlagUntilTimeout)
    I2C_WaitOnFlagUntilTimeout               0x08001db9   Thumb Code   142  stm32f4xx_hal_i2c.o(i.I2C_WaitOnFlagUntilTimeout)
    i.I2C_WaitOnMasterAddressFlagUntilTimeout 0x08001e48   Section        0  stm32f4xx_hal_i2c.o(i.I2C_WaitOnMasterAddressFlagUntilTimeout)
    I2C_WaitOnMasterAddressFlagUntilTimeout  0x08001e49   Thumb Code   140  stm32f4xx_hal_i2c.o(i.I2C_WaitOnMasterAddressFlagUntilTimeout)
    i.I2C_WaitOnTXEFlagUntilTimeout          0x08001ed4   Section        0  stm32f4xx_hal_i2c.o(i.I2C_WaitOnTXEFlagUntilTimeout)
    I2C_WaitOnTXEFlagUntilTimeout            0x08001ed5   Thumb Code    82  stm32f4xx_hal_i2c.o(i.I2C_WaitOnTXEFlagUntilTimeout)
    i.IAP_HTTP_writedata                     0x08001f28   Section        0  httpserver.o(i.IAP_HTTP_writedata)
    IAP_HTTP_writedata                       0x08001f29   Thumb Code   130  httpserver.o(i.IAP_HTTP_writedata)
    i.IAP_httpd_init                         0x08001fb0   Section        0  httpserver.o(i.IAP_httpd_init)
    i.Init_Config                            0x08001fdc   Section        0  main.o(i.Init_Config)
    Init_Config                              0x08001fdd   Thumb Code   308  main.o(i.Init_Config)
    i.MemManage_Handler                      0x08002128   Section        0  stm32f4xx_it.o(i.MemManage_Handler)
    i.NMI_Handler                            0x0800212a   Section        0  stm32f4xx_it.o(i.NMI_Handler)
    i.NVIC_SetPriority                       0x0800212c   Section        0  stm32f4xx_hal_cortex.o(i.NVIC_SetPriority)
    NVIC_SetPriority                         0x0800212d   Thumb Code    32  stm32f4xx_hal_cortex.o(i.NVIC_SetPriority)
    i.NVIC_SystemReset                       0x0800214c   Section        0  httpserver.o(i.NVIC_SystemReset)
    NVIC_SystemReset                         0x0800214d   Thumb Code    26  httpserver.o(i.NVIC_SystemReset)
    i.Netif_Config                           0x08002170   Section        0  main.o(i.Netif_Config)
    Netif_Config                             0x08002171   Thumb Code    80  main.o(i.Netif_Config)
    i.Parse_Content_Length                   0x080021d8   Section        0  httpserver.o(i.Parse_Content_Length)
    Parse_Content_Length                     0x080021d9   Thumb Code   102  httpserver.o(i.Parse_Content_Length)
    i.SysTick_Handler                        0x08002248   Section        0  stm32f4xx_it.o(i.SysTick_Handler)
    i.SystemClock_Config                     0x0800224c   Section        0  main.o(i.SystemClock_Config)
    SystemClock_Config                       0x0800224d   Thumb Code   130  main.o(i.SystemClock_Config)
    i.SystemInit                             0x080022dc   Section        0  system_stm32f4xx.o(i.SystemInit)
    i.UsageFault_Handler                     0x08002330   Section        0  stm32f4xx_it.o(i.UsageFault_Handler)
    i.User_notification                      0x08002332   Section        0  app_ethernet.o(i.User_notification)
    i.__0sprintf$2                           0x08002334   Section        0  printf2.o(i.__0sprintf$2)
    i.__scatterload_copy                     0x0800235c   Section       14  handlers.o(i.__scatterload_copy)
    i.__scatterload_null                     0x0800236a   Section        2  handlers.o(i.__scatterload_null)
    i.__scatterload_zeroinit                 0x0800236c   Section       14  handlers.o(i.__scatterload_zeroinit)
    i._printf_core                           0x0800237a   Section        0  printf2.o(i._printf_core)
    _printf_core                             0x0800237b   Thumb Code   214  printf2.o(i._printf_core)
    i._sputc                                 0x08002450   Section        0  printf2.o(i._sputc)
    _sputc                                   0x08002451   Thumb Code    10  printf2.o(i._sputc)
    i.arp_timer                              0x0800245c   Section        0  lwip_timers.o(i.arp_timer)
    arp_timer                                0x0800245d   Thumb Code    22  lwip_timers.o(i.arp_timer)
    i.close_conn                             0x08002478   Section        0  httpserver.o(i.close_conn)
    close_conn                               0x08002479   Thumb Code    44  httpserver.o(i.close_conn)
    i.conn_err                               0x080024a4   Section        0  httpserver.o(i.conn_err)
    conn_err                                 0x080024a5   Thumb Code     4  httpserver.o(i.conn_err)
    i.dhcp_arp_reply                         0x080024a8   Section        0  dhcp.o(i.dhcp_arp_reply)
    i.dhcp_bind                              0x080024c6   Section        0  dhcp.o(i.dhcp_bind)
    dhcp_bind                                0x080024c7   Thumb Code   192  dhcp.o(i.dhcp_bind)
    i.dhcp_check                             0x08002586   Section        0  dhcp.o(i.dhcp_check)
    dhcp_check                               0x08002587   Thumb Code    48  dhcp.o(i.dhcp_check)
    i.dhcp_coarse_tmr                        0x080025b8   Section        0  dhcp.o(i.dhcp_coarse_tmr)
    i.dhcp_create_msg                        0x08002618   Section        0  dhcp.o(i.dhcp_create_msg)
    dhcp_create_msg                          0x08002619   Thumb Code   282  dhcp.o(i.dhcp_create_msg)
    i.dhcp_decline                           0x0800273c   Section        0  dhcp.o(i.dhcp_decline)
    dhcp_decline                             0x0800273d   Thumb Code   114  dhcp.o(i.dhcp_decline)
    i.dhcp_delete_msg                        0x080027b4   Section        0  dhcp.o(i.dhcp_delete_msg)
    dhcp_delete_msg                          0x080027b5   Thumb Code    22  dhcp.o(i.dhcp_delete_msg)
    i.dhcp_discover                          0x080027cc   Section        0  dhcp.o(i.dhcp_discover)
    dhcp_discover                            0x080027cd   Thumb Code   184  dhcp.o(i.dhcp_discover)
    i.dhcp_fine_tmr                          0x08002888   Section        0  dhcp.o(i.dhcp_fine_tmr)
    i.dhcp_option                            0x080028bc   Section        0  dhcp.o(i.dhcp_option)
    dhcp_option                              0x080028bd   Thumb Code    32  dhcp.o(i.dhcp_option)
    i.dhcp_option_byte                       0x080028dc   Section        0  dhcp.o(i.dhcp_option_byte)
    dhcp_option_byte                         0x080028dd   Thumb Code    16  dhcp.o(i.dhcp_option_byte)
    i.dhcp_option_long                       0x080028ec   Section        0  dhcp.o(i.dhcp_option_long)
    dhcp_option_long                         0x080028ed   Thumb Code    66  dhcp.o(i.dhcp_option_long)
    i.dhcp_option_short                      0x0800292e   Section        0  dhcp.o(i.dhcp_option_short)
    dhcp_option_short                        0x0800292f   Thumb Code    34  dhcp.o(i.dhcp_option_short)
    i.dhcp_option_trailer                    0x08002950   Section        0  dhcp.o(i.dhcp_option_trailer)
    dhcp_option_trailer                      0x08002951   Thumb Code    44  dhcp.o(i.dhcp_option_trailer)
    i.dhcp_rebind                            0x0800297c   Section        0  dhcp.o(i.dhcp_rebind)
    dhcp_rebind                              0x0800297d   Thumb Code   130  dhcp.o(i.dhcp_rebind)
    i.dhcp_reboot                            0x08002a04   Section        0  dhcp.o(i.dhcp_reboot)
    dhcp_reboot                              0x08002a05   Thumb Code   156  dhcp.o(i.dhcp_reboot)
    i.dhcp_release                           0x08002aa4   Section        0  dhcp.o(i.dhcp_release)
    i.dhcp_renew                             0x08002b48   Section        0  dhcp.o(i.dhcp_renew)
    i.dhcp_select                            0x08002bcc   Section        0  dhcp.o(i.dhcp_select)
    dhcp_select                              0x08002bcd   Thumb Code   228  dhcp.o(i.dhcp_select)
    i.dhcp_set_state                         0x08002cb4   Section        0  dhcp.o(i.dhcp_set_state)
    dhcp_set_state                           0x08002cb5   Thumb Code    16  dhcp.o(i.dhcp_set_state)
    i.dhcp_timeout                           0x08002cc4   Section        0  dhcp.o(i.dhcp_timeout)
    dhcp_timeout                             0x08002cc5   Thumb Code   136  dhcp.o(i.dhcp_timeout)
    i.dhcp_timer_coarse                      0x08002d4c   Section        0  lwip_timers.o(i.dhcp_timer_coarse)
    dhcp_timer_coarse                        0x08002d4d   Thumb Code    22  lwip_timers.o(i.dhcp_timer_coarse)
    i.dhcp_timer_fine                        0x08002d68   Section        0  lwip_timers.o(i.dhcp_timer_fine)
    dhcp_timer_fine                          0x08002d69   Thumb Code    22  lwip_timers.o(i.dhcp_timer_fine)
    i.etharp_arp_input                       0x08002d84   Section        0  etharp.o(i.etharp_arp_input)
    etharp_arp_input                         0x08002d85   Thumb Code   206  etharp.o(i.etharp_arp_input)
    i.etharp_cleanup_netif                   0x08002e54   Section        0  etharp.o(i.etharp_cleanup_netif)
    i.etharp_find_entry                      0x08002e84   Section        0  etharp.o(i.etharp_find_entry)
    etharp_find_entry                        0x08002e85   Thumb Code   216  etharp.o(i.etharp_find_entry)
    i.etharp_free_entry                      0x08002f60   Section        0  etharp.o(i.etharp_free_entry)
    etharp_free_entry                        0x08002f61   Thumb Code    50  etharp.o(i.etharp_free_entry)
    i.etharp_output                          0x08002f9c   Section        0  etharp.o(i.etharp_output)
    i.etharp_output_to_arp_index             0x080030a0   Section        0  etharp.o(i.etharp_output_to_arp_index)
    etharp_output_to_arp_index               0x080030a1   Thumb Code    62  etharp.o(i.etharp_output_to_arp_index)
    i.etharp_query                           0x080030e4   Section        0  etharp.o(i.etharp_query)
    i.etharp_raw                             0x080031d0   Section        0  etharp.o(i.etharp_raw)
    etharp_raw                               0x080031d1   Thumb Code   160  etharp.o(i.etharp_raw)
    i.etharp_request                         0x08003270   Section        0  etharp.o(i.etharp_request)
    i.etharp_send_ip                         0x08003294   Section        0  etharp.o(i.etharp_send_ip)
    etharp_send_ip                           0x08003295   Thumb Code    32  etharp.o(i.etharp_send_ip)
    i.etharp_tmr                             0x080032b4   Section        0  etharp.o(i.etharp_tmr)
    i.etharp_update_arp_entry                0x080032fc   Section        0  etharp.o(i.etharp_update_arp_entry)
    etharp_update_arp_entry                  0x080032fd   Thumb Code   118  etharp.o(i.etharp_update_arp_entry)
    i.ethernet_input                         0x08003378   Section        0  etharp.o(i.ethernet_input)
    i.ethernetif_init                        0x08003408   Section        0  ethernetif.o(i.ethernetif_init)
    i.ethernetif_input                       0x08003430   Section        0  ethernetif.o(i.ethernetif_input)
    i.ethernetif_notify_conn_changed         0x08003454   Section        0  app_ethernet.o(i.ethernetif_notify_conn_changed)
    i.ethernetif_update_config               0x08003494   Section        0  ethernetif.o(i.ethernetif_update_config)
    i.fs_open                                0x08003544   Section        0  httpserver.o(i.fs_open)
    fs_open                                  0x08003545   Thumb Code    42  httpserver.o(i.fs_open)
    i.http_accept                            0x08003574   Section        0  httpserver.o(i.http_accept)
    http_accept                              0x08003575   Thumb Code    62  httpserver.o(i.http_accept)
    i.http_poll                              0x080035c0   Section        0  httpserver.o(i.http_poll)
    http_poll                                0x080035c1   Thumb Code    26  httpserver.o(i.http_poll)
    i.http_recv                              0x080035dc   Section        0  httpserver.o(i.http_recv)
    http_recv                                0x080035dd   Thumb Code   874  httpserver.o(i.http_recv)
    i.http_sent                              0x08003a08   Section        0  httpserver.o(i.http_sent)
    http_sent                                0x08003a09   Thumb Code   100  httpserver.o(i.http_sent)
    i.icmp_dest_unreach                      0x08003a78   Section        0  icmp.o(i.icmp_dest_unreach)
    i.icmp_input                             0x08003a80   Section        0  icmp.o(i.icmp_input)
    i.icmp_send_response                     0x08003b7c   Section        0  icmp.o(i.icmp_send_response)
    icmp_send_response                       0x08003b7d   Thumb Code   100  icmp.o(i.icmp_send_response)
    i.icmp_time_exceeded                     0x08003be0   Section        0  icmp.o(i.icmp_time_exceeded)
    i.inet_chksum                            0x08003be8   Section        0  inet_chksum.o(i.inet_chksum)
    i.inet_chksum_pbuf                       0x08003bf4   Section        0  inet_chksum.o(i.inet_chksum_pbuf)
    i.ip4_addr_isbroadcast                   0x08003c3c   Section        0  ip_addr.o(i.ip4_addr_isbroadcast)
    i.ip_frag                                0x08003c6c   Section        0  ip_frag.o(i.ip_frag)
    i.ip_frag_free_pbuf_custom_ref           0x08003dd0   Section        0  ip_frag.o(i.ip_frag_free_pbuf_custom_ref)
    ip_frag_free_pbuf_custom_ref             0x08003dd1   Thumb Code     8  ip_frag.o(i.ip_frag_free_pbuf_custom_ref)
    i.ip_input                               0x08003dd8   Section        0  ip.o(i.ip_input)
    i.ip_output                              0x08003f54   Section        0  ip.o(i.ip_output)
    i.ip_output_if                           0x08003f88   Section        0  ip.o(i.ip_output_if)
    i.ip_reass                               0x08004030   Section        0  ip_frag.o(i.ip_reass)
    i.ip_reass_chain_frag_into_datagram_and_validate 0x080041bc   Section        0  ip_frag.o(i.ip_reass_chain_frag_into_datagram_and_validate)
    ip_reass_chain_frag_into_datagram_and_validate 0x080041bd   Thumb Code   228  ip_frag.o(i.ip_reass_chain_frag_into_datagram_and_validate)
    i.ip_reass_dequeue_datagram              0x080042a4   Section        0  ip_frag.o(i.ip_reass_dequeue_datagram)
    ip_reass_dequeue_datagram                0x080042a5   Thumb Code    30  ip_frag.o(i.ip_reass_dequeue_datagram)
    i.ip_reass_free_complete_datagram        0x080042c8   Section        0  ip_frag.o(i.ip_reass_free_complete_datagram)
    ip_reass_free_complete_datagram          0x080042c9   Thumb Code   108  ip_frag.o(i.ip_reass_free_complete_datagram)
    i.ip_reass_remove_oldest_datagram        0x08004338   Section        0  ip_frag.o(i.ip_reass_remove_oldest_datagram)
    ip_reass_remove_oldest_datagram          0x08004339   Thumb Code   104  ip_frag.o(i.ip_reass_remove_oldest_datagram)
    i.ip_reass_timer                         0x080043a4   Section        0  lwip_timers.o(i.ip_reass_timer)
    ip_reass_timer                           0x080043a5   Thumb Code    22  lwip_timers.o(i.ip_reass_timer)
    i.ip_reass_tmr                           0x080043c0   Section        0  ip_frag.o(i.ip_reass_tmr)
    i.ip_route                               0x080043ec   Section        0  ip.o(i.ip_route)
    i.ipfrag_free_pbuf_custom                0x0800442c   Section        0  ip_frag.o(i.ipfrag_free_pbuf_custom)
    ipfrag_free_pbuf_custom                  0x0800442d   Thumb Code    22  ip_frag.o(i.ipfrag_free_pbuf_custom)
    i.low_level_init                         0x08004444   Section        0  ethernetif.o(i.low_level_init)
    low_level_init                           0x08004445   Thumb Code   178  ethernetif.o(i.low_level_init)
    i.low_level_input                        0x08004510   Section        0  ethernetif.o(i.low_level_input)
    low_level_input                          0x08004511   Thumb Code   172  ethernetif.o(i.low_level_input)
    i.low_level_output                       0x080045c0   Section        0  ethernetif.o(i.low_level_output)
    low_level_output                         0x080045c1   Thumb Code   162  ethernetif.o(i.low_level_output)
    i.lwip_htonl                             0x08004668   Section        0  def.o(i.lwip_htonl)
    i.lwip_htons                             0x0800466c   Section        0  def.o(i.lwip_htons)
    i.lwip_init                              0x08004670   Section        0  init.o(i.lwip_init)
    i.lwip_ntohl                             0x0800468e   Section        0  def.o(i.lwip_ntohl)
    i.lwip_ntohs                             0x08004692   Section        0  def.o(i.lwip_ntohs)
    i.lwip_standard_chksum                   0x08004698   Section        0  inet_chksum.o(i.lwip_standard_chksum)
    lwip_standard_chksum                     0x08004699   Thumb Code    88  inet_chksum.o(i.lwip_standard_chksum)
    i.main                                   0x080046f0   Section        0  main.o(i.main)
    i.mem_free                               0x08004858   Section        0  mem.o(i.mem_free)
    i.mem_init                               0x08004884   Section        0  mem.o(i.mem_init)
    i.mem_malloc                             0x080048b8   Section        0  mem.o(i.mem_malloc)
    i.mem_trim                               0x08004960   Section        0  mem.o(i.mem_trim)
    i.memp_free                              0x08004a2c   Section        0  memp.o(i.memp_free)
    i.memp_init                              0x08004a44   Section        0  memp.o(i.memp_init)
    i.memp_malloc                            0x08004a9c   Section        0  memp.o(i.memp_malloc)
    i.netif_add                              0x08004abc   Section        0  netif.o(i.netif_add)
    i.netif_init                             0x08004b08   Section        0  netif.o(i.netif_init)
    i.netif_set_addr                         0x08004b0a   Section        0  netif.o(i.netif_set_addr)
    i.netif_set_default                      0x08004b2c   Section        0  netif.o(i.netif_set_default)
    i.netif_set_down                         0x08004b38   Section        0  netif.o(i.netif_set_down)
    i.netif_set_gw                           0x08004b52   Section        0  netif.o(i.netif_set_gw)
    i.netif_set_ipaddr                       0x08004b5c   Section        0  netif.o(i.netif_set_ipaddr)
    i.netif_set_link_callback                0x08004bc4   Section        0  netif.o(i.netif_set_link_callback)
    i.netif_set_netmask                      0x08004bcc   Section        0  netif.o(i.netif_set_netmask)
    i.netif_set_up                           0x08004bd4   Section        0  netif.o(i.netif_set_up)
    i.pbuf_alloc                             0x08004bf4   Section        0  pbuf.o(i.pbuf_alloc)
    i.pbuf_alloced_custom                    0x08004d0c   Section        0  pbuf.o(i.pbuf_alloced_custom)
    i.pbuf_cat                               0x08004d60   Section        0  pbuf.o(i.pbuf_cat)
    i.pbuf_chain                             0x08004d88   Section        0  pbuf.o(i.pbuf_chain)
    i.pbuf_clen                              0x08004d9a   Section        0  pbuf.o(i.pbuf_clen)
    i.pbuf_copy                              0x08004dac   Section        0  pbuf.o(i.pbuf_copy)
    i.pbuf_copy_partial                      0x08004e46   Section        0  pbuf.o(i.pbuf_copy_partial)
    i.pbuf_free                              0x08004eae   Section        0  pbuf.o(i.pbuf_free)
    i.pbuf_header                            0x08004efe   Section        0  pbuf.o(i.pbuf_header)
    i.pbuf_realloc                           0x08004f5e   Section        0  pbuf.o(i.pbuf_realloc)
    i.pbuf_ref                               0x08004fac   Section        0  pbuf.o(i.pbuf_ref)
    i.plug_holes                             0x08004fb8   Section        0  mem.o(i.plug_holes)
    plug_holes                               0x08004fb9   Thumb Code    78  mem.o(i.plug_holes)
    i.raw_input                              0x0800500c   Section        0  raw.o(i.raw_input)
    i.send_data                              0x08005080   Section        0  httpserver.o(i.send_data)
    send_data                                0x08005081   Thumb Code    44  httpserver.o(i.send_data)
    i.sys_check_timeouts                     0x080050ac   Section        0  lwip_timers.o(i.sys_check_timeouts)
    i.sys_now                                0x080050f4   Section        0  ethernetif.o(i.sys_now)
    i.sys_timeout                            0x080050f8   Section        0  lwip_timers.o(i.sys_timeout)
    i.sys_timeouts_init                      0x08005154   Section        0  lwip_timers.o(i.sys_timeouts_init)
    i.tcp_abandon                            0x080051a4   Section        0  tcp.o(i.tcp_abandon)
    i.tcp_abort                              0x08005230   Section        0  tcp.o(i.tcp_abort)
    i.tcp_accept                             0x08005236   Section        0  tcp.o(i.tcp_accept)
    i.tcp_accept_null                        0x0800523a   Section        0  tcp.o(i.tcp_accept_null)
    tcp_accept_null                          0x0800523b   Thumb Code     6  tcp.o(i.tcp_accept_null)
    i.tcp_alloc                              0x08005240   Section        0  tcp.o(i.tcp_alloc)
    i.tcp_arg                                0x08005338   Section        0  tcp.o(i.tcp_arg)
    i.tcp_bind                               0x0800533c   Section        0  tcp.o(i.tcp_bind)
    i.tcp_close                              0x080053c0   Section        0  tcp.o(i.tcp_close)
    i.tcp_close_shutdown                     0x080053d4   Section        0  tcp.o(i.tcp_close_shutdown)
    tcp_close_shutdown                       0x080053d5   Thumb Code   290  tcp.o(i.tcp_close_shutdown)
    i.tcp_create_segment                     0x080054fc   Section        0  tcp_out.o(i.tcp_create_segment)
    tcp_create_segment                       0x080054fd   Thumb Code   156  tcp_out.o(i.tcp_create_segment)
    i.tcp_eff_send_mss                       0x08005598   Section        0  tcp.o(i.tcp_eff_send_mss)
    i.tcp_enqueue_flags                      0x080055b8   Section        0  tcp_out.o(i.tcp_enqueue_flags)
    i.tcp_err                                0x0800565e   Section        0  tcp.o(i.tcp_err)
    i.tcp_fasttmr                            0x08005664   Section        0  tcp.o(i.tcp_fasttmr)
    i.tcp_init                               0x080056c4   Section        0  tcp.o(i.tcp_init)
    i.tcp_input                              0x080056c8   Section        0  tcp_in.o(i.tcp_input)
    i.tcp_keepalive                          0x080059dc   Section        0  tcp_out.o(i.tcp_keepalive)
    i.tcp_listen_input                       0x08005a18   Section        0  tcp_in.o(i.tcp_listen_input)
    tcp_listen_input                         0x08005a19   Thumb Code   208  tcp_in.o(i.tcp_listen_input)
    i.tcp_listen_with_backlog                0x08005afc   Section        0  tcp.o(i.tcp_listen_with_backlog)
    i.tcp_new                                0x08005b84   Section        0  tcp.o(i.tcp_new)
    i.tcp_new_port                           0x08005b8c   Section        0  tcp.o(i.tcp_new_port)
    tcp_new_port                             0x08005b8d   Thumb Code    82  tcp.o(i.tcp_new_port)
    i.tcp_next_iss                           0x08005be8   Section        0  tcp.o(i.tcp_next_iss)
    i.tcp_output                             0x08005bf8   Section        0  tcp_out.o(i.tcp_output)
    i.tcp_output_alloc_header                0x08005d84   Section        0  tcp_out.o(i.tcp_output_alloc_header)
    tcp_output_alloc_header                  0x08005d85   Thumb Code   106  tcp_out.o(i.tcp_output_alloc_header)
    i.tcp_output_segment                     0x08005df0   Section        0  tcp_out.o(i.tcp_output_segment)
    tcp_output_segment                       0x08005df1   Thumb Code   170  tcp_out.o(i.tcp_output_segment)
    i.tcp_parseopt                           0x08005ea0   Section        0  tcp_in.o(i.tcp_parseopt)
    tcp_parseopt                             0x08005ea1   Thumb Code   122  tcp_in.o(i.tcp_parseopt)
    i.tcp_pbuf_prealloc                      0x08005f20   Section        0  tcp_out.o(i.tcp_pbuf_prealloc)
    tcp_pbuf_prealloc                        0x08005f21   Thumb Code    78  tcp_out.o(i.tcp_pbuf_prealloc)
    i.tcp_pcb_purge                          0x08005f6e   Section        0  tcp.o(i.tcp_pcb_purge)
    i.tcp_pcb_remove                         0x08005fa8   Section        0  tcp.o(i.tcp_pcb_remove)
    i.tcp_poll                               0x08006000   Section        0  tcp.o(i.tcp_poll)
    i.tcp_process                            0x0800600c   Section        0  tcp_in.o(i.tcp_process)
    tcp_process                              0x0800600d   Thumb Code   788  tcp_in.o(i.tcp_process)
    i.tcp_process_refused_data               0x08006340   Section        0  tcp.o(i.tcp_process_refused_data)
    i.tcp_receive                            0x080063a8   Section        0  tcp_in.o(i.tcp_receive)
    tcp_receive                              0x080063a9   Thumb Code  1042  tcp_in.o(i.tcp_receive)
    i.tcp_recv                               0x080067ba   Section        0  tcp.o(i.tcp_recv)
    i.tcp_recv_null                          0x080067be   Section        0  tcp.o(i.tcp_recv_null)
    i.tcp_recved                             0x080067e2   Section        0  tcp.o(i.tcp_recved)
    i.tcp_rexmit                             0x0800681a   Section        0  tcp_out.o(i.tcp_rexmit)
    i.tcp_rexmit_fast                        0x0800686c   Section        0  tcp_out.o(i.tcp_rexmit_fast)
    i.tcp_rexmit_rto                         0x080068c4   Section        0  tcp_out.o(i.tcp_rexmit_rto)
    i.tcp_rst                                0x080068f2   Section        0  tcp_out.o(i.tcp_rst)
    i.tcp_seg_free                           0x08006968   Section        0  tcp.o(i.tcp_seg_free)
    i.tcp_segs_free                          0x08006984   Section        0  tcp.o(i.tcp_segs_free)
    i.tcp_send_empty_ack                     0x08006996   Section        0  tcp_out.o(i.tcp_send_empty_ack)
    i.tcp_send_fin                           0x080069de   Section        0  tcp_out.o(i.tcp_send_fin)
    i.tcp_sent                               0x08006a22   Section        0  tcp.o(i.tcp_sent)
    i.tcp_slowtmr                            0x08006a28   Section        0  tcp.o(i.tcp_slowtmr)
    i.tcp_timer_needed                       0x08006c84   Section        0  lwip_timers.o(i.tcp_timer_needed)
    i.tcp_timewait_input                     0x08006cb8   Section        0  tcp_in.o(i.tcp_timewait_input)
    tcp_timewait_input                       0x08006cb9   Thumb Code    92  tcp_in.o(i.tcp_timewait_input)
    i.tcp_tmr                                0x08006d24   Section        0  tcp.o(i.tcp_tmr)
    i.tcp_update_rcv_ann_wnd                 0x08006d44   Section        0  tcp.o(i.tcp_update_rcv_ann_wnd)
    i.tcp_write                              0x08006d78   Section        0  tcp_out.o(i.tcp_write)
    i.tcp_zero_window_probe                  0x08007074   Section        0  tcp_out.o(i.tcp_zero_window_probe)
    i.tcpip_tcp_timer                        0x08007100   Section        0  lwip_timers.o(i.tcpip_tcp_timer)
    tcpip_tcp_timer                          0x08007101   Thumb Code    40  lwip_timers.o(i.tcpip_tcp_timer)
    i.udp_bind                               0x08007138   Section        0  udp.o(i.udp_bind)
    i.udp_init                               0x080071d0   Section        0  udp.o(i.udp_init)
    i.udp_input                              0x080071d4   Section        0  udp.o(i.udp_input)
    i.udp_sendto_if                          0x0800734c   Section        0  udp.o(i.udp_sendto_if)
    .constdata                               0x08007402   Section       40  memp.o(.constdata)
    memp_sizes                               0x08007402   Data          20  memp.o(.constdata)
    memp_num                                 0x08007416   Data          20  memp.o(.constdata)
    .constdata                               0x0800742c   Section       84  tcp.o(.constdata)
    .constdata                               0x08007480   Section        4  ip_addr.o(.constdata)
    .constdata                               0x08007484   Section        4  ip_addr.o(.constdata)
    .constdata                               0x08007488   Section       12  etharp.o(.constdata)
    .constdata                               0x08007494   Section       16  stm32f4xx_hal_rcc.o(.constdata)
    .constdata                               0x080074a4   Section      662  httpserver.o(.constdata)
    data_index_html                          0x080074a4   Data         662  httpserver.o(.constdata)
    .constdata                               0x0800773a   Section      411  httpserver.o(.constdata)
    data_reset_html                          0x0800773a   Data         411  httpserver.o(.constdata)
    .constdata                               0x080078d5   Section      634  httpserver.o(.constdata)
    data_upload_html                         0x080078d5   Data         634  httpserver.o(.constdata)
    .constdata                               0x08007b4f   Section      571  httpserver.o(.constdata)
    data_uploaddone_html                     0x08007b4f   Data         571  httpserver.o(.constdata)
    .constdata                               0x08007d8c   Section       16  httpserver.o(.constdata)
    .constdata                               0x08007d9c   Section       16  httpserver.o(.constdata)
    .constdata                               0x08007dac   Section       16  httpserver.o(.constdata)
    .constdata                               0x08007dbc   Section       51  httpserver.o(.constdata)
    http_crnl_2                              0x08007dbc   Data           4  httpserver.o(.constdata)
    octet_stream                             0x08007dd0   Data          14  httpserver.o(.constdata)
    Content_Length                           0x08007dde   Data          17  httpserver.o(.constdata)
    .conststring                             0x08007df0   Section      117  tcp.o(.conststring)
    .data                                    0x20000000   Section       20  system_stm32f4xx.o(.data)
    .data                                    0x20000014   Section       28  tcp_in.o(.data)
    flags                                    0x20000014   Data           1  tcp_in.o(.data)
    recv_flags                               0x20000015   Data           1  tcp_in.o(.data)
    tcplen                                   0x20000016   Data           2  tcp_in.o(.data)
    tcphdr                                   0x20000018   Data           4  tcp_in.o(.data)
    iphdr                                    0x2000001c   Data           4  tcp_in.o(.data)
    seqno                                    0x20000020   Data           4  tcp_in.o(.data)
    ackno                                    0x20000024   Data           4  tcp_in.o(.data)
    recv_data                                0x20000028   Data           4  tcp_in.o(.data)
    .data                                    0x20000030   Section       12  lwip_timers.o(.data)
    next_timeout                             0x20000030   Data           4  lwip_timers.o(.data)
    timeouts_last_time                       0x20000034   Data           4  lwip_timers.o(.data)
    tcpip_tcp_timer_active                   0x20000038   Data           4  lwip_timers.o(.data)
    .data                                    0x2000003c   Section        4  dhcp.o(.data)
    xid                                      0x2000003c   Data           4  dhcp.o(.data)
    .data                                    0x20000040   Section        8  udp.o(.data)
    udp_port                                 0x20000040   Data           2  udp.o(.data)
    .data                                    0x20000048   Section       12  mem.o(.data)
    ram                                      0x20000048   Data           4  mem.o(.data)
    ram_end                                  0x2000004c   Data           4  mem.o(.data)
    lfree                                    0x20000050   Data           4  mem.o(.data)
    .data                                    0x20000054   Section       12  netif.o(.data)
    netif_num                                0x20000054   Data           1  netif.o(.data)
    .data                                    0x20000060   Section       36  tcp.o(.data)
    tcp_timer                                0x20000061   Data           1  tcp.o(.data)
    tcp_timer_ctr                            0x20000062   Data           1  tcp.o(.data)
    tcp_port                                 0x20000064   Data           2  tcp.o(.data)
    iss                                      0x20000068   Data           4  tcp.o(.data)
    .data                                    0x20000084   Section        4  raw.o(.data)
    raw_pcbs                                 0x20000084   Data           4  raw.o(.data)
    .data                                    0x20000088   Section        8  ip_frag.o(.data)
    ip_reass_pbufcount                       0x20000088   Data           2  ip_frag.o(.data)
    reassdatagrams                           0x2000008c   Data           4  ip_frag.o(.data)
    .data                                    0x20000090   Section       20  ip.o(.data)
    ip_id                                    0x20000090   Data           2  ip.o(.data)
    .data                                    0x200000a4   Section        1  etharp.o(.data)
    etharp_cached_entry                      0x200000a4   Data           1  etharp.o(.data)
    .data                                    0x200000a8   Section        4  stm32f4xx_hal.o(.data)
    .data                                    0x200000ac   Section       36  httpserver.o(.data)
    LeftBytes                                0x200000ac   Data           1  httpserver.o(.data)
    resetpage                                0x200000ad   Data           1  httpserver.o(.data)
    DataFlag                                 0x200000b0   Data           4  httpserver.o(.data)
    size                                     0x200000b4   Data           4  httpserver.o(.data)
    TotalReceived                            0x200000b8   Data           4  httpserver.o(.data)
    ContentLengthOffset                      0x200000bc   Data           4  httpserver.o(.data)
    BrowserFlag                              0x200000c0   Data           4  httpserver.o(.data)
    TotalData                                0x200000c4   Data           4  httpserver.o(.data)
    FlashWriteAddress                        0x200000c8   Data           4  httpserver.o(.data)
    LeftBytesTab                             0x200000cc   Data           4  httpserver.o(.data)
    .data                                    0x200000d0   Section       12  main.o(.data)
    .data                                    0x200000dc   Section        1  stm324xg_eval_eeprom.o(.data)
    .bss                                     0x200000e0   Section       20  tcp_in.o(.bss)
    inseg                                    0x200000e0   Data          20  tcp_in.o(.bss)
    .bss                                     0x200000f4   Section    18475  memp.o(.bss)
    memp_tab                                 0x200000f4   Data          40  memp.o(.bss)
    memp_memory                              0x2000011c   Data       18435  memp.o(.bss)
    .bss                                     0x2000491f   Section    10260  mem.o(.bss)
    .bss                                     0x20007134   Section      200  etharp.o(.bss)
    arp_table                                0x20007134   Data         200  etharp.o(.bss)
    .bss                                     0x200071fc   Section       32  stm32f4xx_hal_flash.o(.bss)
    .bss                                     0x2000721c   Section    12520  ethernetif.o(.bss)
    .bss                                     0x2000a304   Section      124  main.o(.bss)
    STACK                                    0x2000a380   Section     2048  startup_stm32f407xx.o(STACK)

    Global Symbols

    Symbol Name                              Value     Ov Type        Size  Object(Section)

    BuildAttributes$$THM_ISAv4$E$P$D$K$B$S$7EM$VFPi3$EXTD16$VFPS$VFMA$PE$A:L22UL41UL21$X:L11$S22US41US21$IEEE1$IW$USESV6$~STKCKD$USESV7$~SHL$OSPACE$ROPI$EBA8$MICROLIB$REQ8$PRES8$EABIv2 0x00000000   Number         0  anon$$obj.o ABSOLUTE
    __ARM_use_no_argv                        0x00000000   Number         0  main.o ABSOLUTE
    _printf_a                                0x00000000   Number         0  stubs.o ABSOLUTE
    _printf_c                                0x00000000   Number         0  stubs.o ABSOLUTE
    _printf_charcount                        0x00000000   Number         0  stubs.o ABSOLUTE
    _printf_d                                0x00000000   Number         0  stubs.o ABSOLUTE
    _printf_e                                0x00000000   Number         0  stubs.o ABSOLUTE
    _printf_f                                0x00000000   Number         0  stubs.o ABSOLUTE
    _printf_flags                            0x00000000   Number         0  stubs.o ABSOLUTE
    _printf_fp_dec                           0x00000000   Number         0  stubs.o ABSOLUTE
    _printf_fp_hex                           0x00000000   Number         0  stubs.o ABSOLUTE
    _printf_g                                0x00000000   Number         0  stubs.o ABSOLUTE
    _printf_i                                0x00000000   Number         0  stubs.o ABSOLUTE
    _printf_int_dec                          0x00000000   Number         0  stubs.o ABSOLUTE
    _printf_l                                0x00000000   Number         0  stubs.o ABSOLUTE
    _printf_lc                               0x00000000   Number         0  stubs.o ABSOLUTE
    _printf_ll                               0x00000000   Number         0  stubs.o ABSOLUTE
    _printf_lld                              0x00000000   Number         0  stubs.o ABSOLUTE
    _printf_lli                              0x00000000   Number         0  stubs.o ABSOLUTE
    _printf_llo                              0x00000000   Number         0  stubs.o ABSOLUTE
    _printf_llu                              0x00000000   Number         0  stubs.o ABSOLUTE
    _printf_llx                              0x00000000   Number         0  stubs.o ABSOLUTE
    _printf_longlong_dec                     0x00000000   Number         0  stubs.o ABSOLUTE
    _printf_longlong_hex                     0x00000000   Number         0  stubs.o ABSOLUTE
    _printf_longlong_oct                     0x00000000   Number         0  stubs.o ABSOLUTE
    _printf_ls                               0x00000000   Number         0  stubs.o ABSOLUTE
    _printf_mbtowc                           0x00000000   Number         0  stubs.o ABSOLUTE
    _printf_n                                0x00000000   Number         0  stubs.o ABSOLUTE
    _printf_o                                0x00000000   Number         0  stubs.o ABSOLUTE
    _printf_p                                0x00000000   Number         0  stubs.o ABSOLUTE
    _printf_percent                          0x00000000   Number         0  stubs.o ABSOLUTE
    _printf_pre_padding                      0x00000000   Number         0  stubs.o ABSOLUTE
    _printf_return_value                     0x00000000   Number         0  stubs.o ABSOLUTE
    _printf_s                                0x00000000   Number         0  stubs.o ABSOLUTE
    _printf_sizespec                         0x00000000   Number         0  stubs.o ABSOLUTE
    _printf_str                              0x00000000   Number         0  stubs.o ABSOLUTE
    _printf_truncate_signed                  0x00000000   Number         0  stubs.o ABSOLUTE
    _printf_truncate_unsigned                0x00000000   Number         0  stubs.o ABSOLUTE
    _printf_u                                0x00000000   Number         0  stubs.o ABSOLUTE
    _printf_wc                               0x00000000   Number         0  stubs.o ABSOLUTE
    _printf_wctomb                           0x00000000   Number         0  stubs.o ABSOLUTE
    _printf_widthprec                        0x00000000   Number         0  stubs.o ABSOLUTE
    _printf_x                                0x00000000   Number         0  stubs.o ABSOLUTE
    __cpp_initialize__aeabi_                  - Undefined Weak Reference
    __cxa_finalize                            - Undefined Weak Reference
    __decompress                              - Undefined Weak Reference
    _clock_init                               - Undefined Weak Reference
    _microlib_exit                            - Undefined Weak Reference
    __Vectors_Size                           0x00000188   Number         0  startup_stm32f407xx.o ABSOLUTE
    __Vectors                                0x08000000   Data           4  startup_stm32f407xx.o(RESET)
    __Vectors_End                            0x08000188   Data           0  startup_stm32f407xx.o(RESET)
    __main                                   0x08000189   Thumb Code     0  entry.o(.ARM.Collect$$$$00000000)
    _main_stk                                0x08000189   Thumb Code     0  entry2.o(.ARM.Collect$$$$00000001)
    _main_scatterload                        0x0800018d   Thumb Code     0  entry5.o(.ARM.Collect$$$$00000004)
    __main_after_scatterload                 0x08000191   Thumb Code     0  entry5.o(.ARM.Collect$$$$00000004)
    _main_clock                              0x08000191   Thumb Code     0  entry7b.o(.ARM.Collect$$$$00000008)
    _main_cpp_init                           0x08000191   Thumb Code     0  entry8b.o(.ARM.Collect$$$$0000000A)
    _main_init                               0x08000191   Thumb Code     0  entry9a.o(.ARM.Collect$$$$0000000B)
    __rt_final_cpp                           0x08000199   Thumb Code     0  entry10a.o(.ARM.Collect$$$$0000000D)
    __rt_final_exit                          0x08000199   Thumb Code     0  entry11a.o(.ARM.Collect$$$$0000000F)
    Reset_Handler                            0x0800019d   Thumb Code     8  startup_stm32f407xx.o(.text)
    SVC_Handler                              0x080001af   Thumb Code     2  startup_stm32f407xx.o(.text)
    PendSV_Handler                           0x080001b3   Thumb Code     2  startup_stm32f407xx.o(.text)
    ADC_IRQHandler                           0x080001b7   Thumb Code     0  startup_stm32f407xx.o(.text)
    CAN1_RX0_IRQHandler                      0x080001b7   Thumb Code     0  startup_stm32f407xx.o(.text)
    CAN1_RX1_IRQHandler                      0x080001b7   Thumb Code     0  startup_stm32f407xx.o(.text)
    CAN1_SCE_IRQHandler                      0x080001b7   Thumb Code     0  startup_stm32f407xx.o(.text)
    CAN1_TX_IRQHandler                       0x080001b7   Thumb Code     0  startup_stm32f407xx.o(.text)
    CAN2_RX0_IRQHandler                      0x080001b7   Thumb Code     0  startup_stm32f407xx.o(.text)
    CAN2_RX1_IRQHandler                      0x080001b7   Thumb Code     0  startup_stm32f407xx.o(.text)
    CAN2_SCE_IRQHandler                      0x080001b7   Thumb Code     0  startup_stm32f407xx.o(.text)
    CAN2_TX_IRQHandler                       0x080001b7   Thumb Code     0  startup_stm32f407xx.o(.text)
    DCMI_IRQHandler                          0x080001b7   Thumb Code     0  startup_stm32f407xx.o(.text)
    DMA1_Stream0_IRQHandler                  0x080001b7   Thumb Code     0  startup_stm32f407xx.o(.text)
    DMA1_Stream1_IRQHandler                  0x080001b7   Thumb Code     0  startup_stm32f407xx.o(.text)
    DMA1_Stream2_IRQHandler                  0x080001b7   Thumb Code     0  startup_stm32f407xx.o(.text)
    DMA1_Stream3_IRQHandler                  0x080001b7   Thumb Code     0  startup_stm32f407xx.o(.text)
    DMA1_Stream4_IRQHandler                  0x080001b7   Thumb Code     0  startup_stm32f407xx.o(.text)
    DMA1_Stream5_IRQHandler                  0x080001b7   Thumb Code     0  startup_stm32f407xx.o(.text)
    DMA1_Stream6_IRQHandler                  0x080001b7   Thumb Code     0  startup_stm32f407xx.o(.text)
    DMA1_Stream7_IRQHandler                  0x080001b7   Thumb Code     0  startup_stm32f407xx.o(.text)
    DMA2_Stream0_IRQHandler                  0x080001b7   Thumb Code     0  startup_stm32f407xx.o(.text)
    DMA2_Stream1_IRQHandler                  0x080001b7   Thumb Code     0  startup_stm32f407xx.o(.text)
    DMA2_Stream2_IRQHandler                  0x080001b7   Thumb Code     0  startup_stm32f407xx.o(.text)
    DMA2_Stream3_IRQHandler                  0x080001b7   Thumb Code     0  startup_stm32f407xx.o(.text)
    DMA2_Stream4_IRQHandler                  0x080001b7   Thumb Code     0  startup_stm32f407xx.o(.text)
    DMA2_Stream5_IRQHandler                  0x080001b7   Thumb Code     0  startup_stm32f407xx.o(.text)
    DMA2_Stream6_IRQHandler                  0x080001b7   Thumb Code     0  startup_stm32f407xx.o(.text)
    DMA2_Stream7_IRQHandler                  0x080001b7   Thumb Code     0  startup_stm32f407xx.o(.text)
    ETH_IRQHandler                           0x080001b7   Thumb Code     0  startup_stm32f407xx.o(.text)
    ETH_WKUP_IRQHandler                      0x080001b7   Thumb Code     0  startup_stm32f407xx.o(.text)
    EXTI0_IRQHandler                         0x080001b7   Thumb Code     0  startup_stm32f407xx.o(.text)
    EXTI1_IRQHandler                         0x080001b7   Thumb Code     0  startup_stm32f407xx.o(.text)
    EXTI2_IRQHandler                         0x080001b7   Thumb Code     0  startup_stm32f407xx.o(.text)
    EXTI3_IRQHandler                         0x080001b7   Thumb Code     0  startup_stm32f407xx.o(.text)
    EXTI4_IRQHandler                         0x080001b7   Thumb Code     0  startup_stm32f407xx.o(.text)
    EXTI9_5_IRQHandler                       0x080001b7   Thumb Code     0  startup_stm32f407xx.o(.text)
    FLASH_IRQHandler                         0x080001b7   Thumb Code     0  startup_stm32f407xx.o(.text)
    FMC_IRQHandler                           0x080001b7   Thumb Code     0  startup_stm32f407xx.o(.text)
    FPU_IRQHandler                           0x080001b7   Thumb Code     0  startup_stm32f407xx.o(.text)
    HASH_RNG_IRQHandler                      0x080001b7   Thumb Code     0  startup_stm32f407xx.o(.text)
    I2C1_ER_IRQHandler                       0x080001b7   Thumb Code     0  startup_stm32f407xx.o(.text)
    I2C1_EV_IRQHandler                       0x080001b7   Thumb Code     0  startup_stm32f407xx.o(.text)
    I2C2_ER_IRQHandler                       0x080001b7   Thumb Code     0  startup_stm32f407xx.o(.text)
    I2C2_EV_IRQHandler                       0x080001b7   Thumb Code     0  startup_stm32f407xx.o(.text)
    I2C3_ER_IRQHandler                       0x080001b7   Thumb Code     0  startup_stm32f407xx.o(.text)
    I2C3_EV_IRQHandler                       0x080001b7   Thumb Code     0  startup_stm32f407xx.o(.text)
    OTG_FS_IRQHandler                        0x080001b7   Thumb Code     0  startup_stm32f407xx.o(.text)
    OTG_FS_WKUP_IRQHandler                   0x080001b7   Thumb Code     0  startup_stm32f407xx.o(.text)
    OTG_HS_EP1_IN_IRQHandler                 0x080001b7   Thumb Code     0  startup_stm32f407xx.o(.text)
    OTG_HS_EP1_OUT_IRQHandler                0x080001b7   Thumb Code     0  startup_stm32f407xx.o(.text)
    OTG_HS_IRQHandler                        0x080001b7   Thumb Code     0  startup_stm32f407xx.o(.text)
    OTG_HS_WKUP_IRQHandler                   0x080001b7   Thumb Code     0  startup_stm32f407xx.o(.text)
    PVD_IRQHandler                           0x080001b7   Thumb Code     0  startup_stm32f407xx.o(.text)
    RCC_IRQHandler                           0x080001b7   Thumb Code     0  startup_stm32f407xx.o(.text)
    RTC_Alarm_IRQHandler                     0x080001b7   Thumb Code     0  startup_stm32f407xx.o(.text)
    RTC_WKUP_IRQHandler                      0x080001b7   Thumb Code     0  startup_stm32f407xx.o(.text)
    SDIO_IRQHandler                          0x080001b7   Thumb Code     0  startup_stm32f407xx.o(.text)
    SPI1_IRQHandler                          0x080001b7   Thumb Code     0  startup_stm32f407xx.o(.text)
    SPI2_IRQHandler                          0x080001b7   Thumb Code     0  startup_stm32f407xx.o(.text)
    SPI3_IRQHandler                          0x080001b7   Thumb Code     0  startup_stm32f407xx.o(.text)
    TAMP_STAMP_IRQHandler                    0x080001b7   Thumb Code     0  startup_stm32f407xx.o(.text)
    TIM1_BRK_TIM9_IRQHandler                 0x080001b7   Thumb Code     0  startup_stm32f407xx.o(.text)
    TIM1_CC_IRQHandler                       0x080001b7   Thumb Code     0  startup_stm32f407xx.o(.text)
    TIM1_TRG_COM_TIM11_IRQHandler            0x080001b7   Thumb Code     0  startup_stm32f407xx.o(.text)
    TIM1_UP_TIM10_IRQHandler                 0x080001b7   Thumb Code     0  startup_stm32f407xx.o(.text)
    TIM2_IRQHandler                          0x080001b7   Thumb Code     0  startup_stm32f407xx.o(.text)
    TIM3_IRQHandler                          0x080001b7   Thumb Code     0  startup_stm32f407xx.o(.text)
    TIM4_IRQHandler                          0x080001b7   Thumb Code     0  startup_stm32f407xx.o(.text)
    TIM5_IRQHandler                          0x080001b7   Thumb Code     0  startup_stm32f407xx.o(.text)
    TIM6_DAC_IRQHandler                      0x080001b7   Thumb Code     0  startup_stm32f407xx.o(.text)
    TIM7_IRQHandler                          0x080001b7   Thumb Code     0  startup_stm32f407xx.o(.text)
    TIM8_BRK_TIM12_IRQHandler                0x080001b7   Thumb Code     0  startup_stm32f407xx.o(.text)
    TIM8_CC_IRQHandler                       0x080001b7   Thumb Code     0  startup_stm32f407xx.o(.text)
    TIM8_TRG_COM_TIM14_IRQHandler            0x080001b7   Thumb Code     0  startup_stm32f407xx.o(.text)
    TIM8_UP_TIM13_IRQHandler                 0x080001b7   Thumb Code     0  startup_stm32f407xx.o(.text)
    UART4_IRQHandler                         0x080001b7   Thumb Code     0  startup_stm32f407xx.o(.text)
    UART5_IRQHandler                         0x080001b7   Thumb Code     0  startup_stm32f407xx.o(.text)
    USART1_IRQHandler                        0x080001b7   Thumb Code     0  startup_stm32f407xx.o(.text)
    USART2_IRQHandler                        0x080001b7   Thumb Code     0  startup_stm32f407xx.o(.text)
    USART3_IRQHandler                        0x080001b7   Thumb Code     0  startup_stm32f407xx.o(.text)
    USART6_IRQHandler                        0x080001b7   Thumb Code     0  startup_stm32f407xx.o(.text)
    WWDG_IRQHandler                          0x080001b7   Thumb Code     0  startup_stm32f407xx.o(.text)
    __aeabi_memcpy                           0x080001c1   Thumb Code    36  memcpya.o(.text)
    __aeabi_memcpy4                          0x080001c1   Thumb Code     0  memcpya.o(.text)
    __aeabi_memcpy8                          0x080001c1   Thumb Code     0  memcpya.o(.text)
    __aeabi_memset                           0x080001e5   Thumb Code    14  memseta.o(.text)
    __aeabi_memset4                          0x080001e5   Thumb Code     0  memseta.o(.text)
    __aeabi_memset8                          0x080001e5   Thumb Code     0  memseta.o(.text)
    __aeabi_memclr                           0x080001f3   Thumb Code     4  memseta.o(.text)
    __aeabi_memclr4                          0x080001f3   Thumb Code     0  memseta.o(.text)
    __aeabi_memclr8                          0x080001f3   Thumb Code     0  memseta.o(.text)
    _memset$wrapper                          0x080001f7   Thumb Code    18  memseta.o(.text)
    strcmp                                   0x08000209   Thumb Code    28  strcmp.o(.text)
    memcmp                                   0x08000225   Thumb Code    26  memcmp.o(.text)
    strncmp                                  0x0800023f   Thumb Code    30  strncmp.o(.text)
    __scatterload                            0x0800025d   Thumb Code    28  init.o(.text)
    __scatterload_rt2                        0x0800025d   Thumb Code     0  init.o(.text)
    BSP_EEPROM_TIMEOUT_UserCallback          0x08000281   Thumb Code     2  stm324xg_eval_eeprom.o(i.BSP_EEPROM_TIMEOUT_UserCallback)
    BSP_EEPROM_WriteBuffer                   0x08000283   Thumb Code   248  stm324xg_eval_eeprom.o(i.BSP_EEPROM_WriteBuffer)
    BusFault_Handler                         0x0800037b   Thumb Code     2  stm32f4xx_it.o(i.BusFault_Handler)
    DebugMon_Handler                         0x0800037d   Thumb Code     2  stm32f4xx_it.o(i.DebugMon_Handler)
    EEPROM_IO_IsDeviceReady                  0x08000381   Thumb Code    12  stm324xg_eval.o(i.EEPROM_IO_IsDeviceReady)
    EEPROM_IO_WriteData                      0x08000391   Thumb Code    40  stm324xg_eval.o(i.EEPROM_IO_WriteData)
    EXTI15_10_IRQHandler                     0x08000549   Thumb Code     8  stm32f4xx_it.o(i.EXTI15_10_IRQHandler)
    FLASH_Erase_Sector                       0x08000551   Thumb Code    84  stm32f4xx_hal_flash_ex.o(i.FLASH_Erase_Sector)
    FLASH_FlushCaches                        0x080005a9   Thumb Code    80  stm32f4xx_hal_flash_ex.o(i.FLASH_FlushCaches)
    FLASH_If_Erase                           0x080005fd   Thumb Code    46  flash_if.o(i.FLASH_If_Erase)
    FLASH_If_Init                            0x08000631   Thumb Code     4  flash_if.o(i.FLASH_If_Init)
    FLASH_If_Write                           0x08000635   Thumb Code    76  flash_if.o(i.FLASH_If_Write)
    FLASH_WaitForLastOperation               0x080007c5   Thumb Code    80  stm32f4xx_hal_flash.o(i.FLASH_WaitForLastOperation)
    HAL_Delay                                0x0800081d   Thumb Code    22  stm32f4xx_hal.o(i.HAL_Delay)
    HAL_ETH_ConfigMAC                        0x08000835   Thumb Code   300  stm32f4xx_hal_eth.o(i.HAL_ETH_ConfigMAC)
    HAL_ETH_DMARxDescListInit                0x08000965   Thumb Code   116  stm32f4xx_hal_eth.o(i.HAL_ETH_DMARxDescListInit)
    HAL_ETH_DMATxDescListInit                0x080009d9   Thumb Code   120  stm32f4xx_hal_eth.o(i.HAL_ETH_DMATxDescListInit)
    HAL_ETH_GetReceivedFrame                 0x08000a51   Thumb Code   122  stm32f4xx_hal_eth.o(i.HAL_ETH_GetReceivedFrame)
    HAL_ETH_Init                             0x08000acd   Thumb Code   450  stm32f4xx_hal_eth.o(i.HAL_ETH_Init)
    HAL_ETH_MspInit                          0x08000cb9   Thumb Code     2  ethernetif.o(i.HAL_ETH_MspInit)
    HAL_ETH_ReadPHYRegister                  0x08000cbd   Thumb Code   132  stm32f4xx_hal_eth.o(i.HAL_ETH_ReadPHYRegister)
    HAL_ETH_Start                            0x08000d41   Thumb Code   132  stm32f4xx_hal_eth.o(i.HAL_ETH_Start)
    HAL_ETH_Stop                             0x08000dc5   Thumb Code   132  stm32f4xx_hal_eth.o(i.HAL_ETH_Stop)
    HAL_ETH_TransmitFrame                    0x08000e49   Thumb Code   264  stm32f4xx_hal_eth.o(i.HAL_ETH_TransmitFrame)
    HAL_ETH_WritePHYRegister                 0x08000f51   Thumb Code   120  stm32f4xx_hal_eth.o(i.HAL_ETH_WritePHYRegister)
    HAL_FLASHEx_Erase                        0x08000fc9   Thumb Code   144  stm32f4xx_hal_flash_ex.o(i.HAL_FLASHEx_Erase)
    HAL_FLASH_Program                        0x08001061   Thumb Code   116  stm32f4xx_hal_flash.o(i.HAL_FLASH_Program)
    HAL_FLASH_Unlock                         0x080010dd   Thumb Code    28  stm32f4xx_hal_flash.o(i.HAL_FLASH_Unlock)
    HAL_GPIO_EXTI_Callback                   0x08001105   Thumb Code     2  stm32f4xx_hal_gpio.o(i.HAL_GPIO_EXTI_Callback)
    HAL_GPIO_EXTI_IRQHandler                 0x08001109   Thumb Code    18  stm32f4xx_hal_gpio.o(i.HAL_GPIO_EXTI_IRQHandler)
    HAL_GPIO_Init                            0x08001121   Thumb Code   398  stm32f4xx_hal_gpio.o(i.HAL_GPIO_Init)
    HAL_GPIO_ReadPin                         0x080012e1   Thumb Code    10  stm32f4xx_hal_gpio.o(i.HAL_GPIO_ReadPin)
    HAL_GPIO_WritePin                        0x080012eb   Thumb Code    10  stm32f4xx_hal_gpio.o(i.HAL_GPIO_WritePin)
    HAL_GetREVID                             0x080012f5   Thumb Code     8  stm32f4xx_hal.o(i.HAL_GetREVID)
    HAL_GetTick                              0x08001301   Thumb Code     6  stm32f4xx_hal.o(i.HAL_GetTick)
    HAL_I2C_DeInit                           0x0800130d   Thumb Code    50  stm32f4xx_hal_i2c.o(i.HAL_I2C_DeInit)
    HAL_I2C_GetState                         0x0800133f   Thumb Code     6  stm32f4xx_hal_i2c.o(i.HAL_I2C_GetState)
    HAL_I2C_Init                             0x08001345   Thumb Code   254  stm32f4xx_hal_i2c.o(i.HAL_I2C_Init)
    HAL_I2C_IsDeviceReady                    0x0800144d   Thumb Code   322  stm32f4xx_hal_i2c.o(i.HAL_I2C_IsDeviceReady)
    HAL_I2C_Mem_Write                        0x08001599   Thumb Code   236  stm32f4xx_hal_i2c.o(i.HAL_I2C_Mem_Write)
    HAL_I2C_MspDeInit                        0x0800168d   Thumb Code     2  stm32f4xx_hal_i2c.o(i.HAL_I2C_MspDeInit)
    HAL_I2C_MspInit                          0x0800168f   Thumb Code     2  stm32f4xx_hal_i2c.o(i.HAL_I2C_MspInit)
    HAL_IncTick                              0x08001691   Thumb Code    10  stm32f4xx_hal.o(i.HAL_IncTick)
    HAL_Init                                 0x080016a1   Thumb Code    40  stm32f4xx_hal.o(i.HAL_Init)
    HAL_InitTick                             0x080016cd   Thumb Code    34  stm32f4xx_hal.o(i.HAL_InitTick)
    HAL_MspInit                              0x080016ef   Thumb Code     2  stm32f4xx_hal.o(i.HAL_MspInit)
    HAL_NVIC_EnableIRQ                       0x080016f1   Thumb Code    22  stm32f4xx_hal_cortex.o(i.HAL_NVIC_EnableIRQ)
    HAL_NVIC_SetPriority                     0x08001709   Thumb Code    60  stm32f4xx_hal_cortex.o(i.HAL_NVIC_SetPriority)
    HAL_NVIC_SetPriorityGrouping             0x08001749   Thumb Code    26  stm32f4xx_hal_cortex.o(i.HAL_NVIC_SetPriorityGrouping)
    HAL_RCC_ClockConfig                      0x0800176d   Thumb Code   312  stm32f4xx_hal_rcc.o(i.HAL_RCC_ClockConfig)
    HAL_RCC_GetHCLKFreq                      0x080018ad   Thumb Code    38  stm32f4xx_hal_rcc.o(i.HAL_RCC_GetHCLKFreq)
    HAL_RCC_GetPCLK1Freq                     0x080018e1   Thumb Code    36  stm32f4xx_hal_rcc.o(i.HAL_RCC_GetPCLK1Freq)
    HAL_RCC_GetSysClockFreq                  0x0800190d   Thumb Code   104  stm32f4xx_hal_rcc.o(i.HAL_RCC_GetSysClockFreq)
    HAL_RCC_OscConfig                        0x08001981   Thumb Code   722  stm32f4xx_hal_rcc.o(i.HAL_RCC_OscConfig)
    HAL_SYSTICK_Config                       0x08001c65   Thumb Code    40  stm32f4xx_hal_cortex.o(i.HAL_SYSTICK_Config)
    HardFault_Handler                        0x08001c8d   Thumb Code     2  stm32f4xx_it.o(i.HardFault_Handler)
    I2C_Config                               0x08001c91   Thumb Code    88  main.o(i.I2C_Config)
    IAP_httpd_init                           0x08001fb1   Thumb Code    36  httpserver.o(i.IAP_httpd_init)
    MemManage_Handler                        0x08002129   Thumb Code     2  stm32f4xx_it.o(i.MemManage_Handler)
    NMI_Handler                              0x0800212b   Thumb Code     2  stm32f4xx_it.o(i.NMI_Handler)
    SysTick_Handler                          0x08002249   Thumb Code     4  stm32f4xx_it.o(i.SysTick_Handler)
    SystemInit                               0x080022dd   Thumb Code    66  system_stm32f4xx.o(i.SystemInit)
    UsageFault_Handler                       0x08002331   Thumb Code     2  stm32f4xx_it.o(i.UsageFault_Handler)
    User_notification                        0x08002333   Thumb Code     2  app_ethernet.o(i.User_notification)
    __0sprintf$2                             0x08002335   Thumb Code    34  printf2.o(i.__0sprintf$2)
    __1sprintf$2                             0x08002335   Thumb Code     0  printf2.o(i.__0sprintf$2)
    __2sprintf                               0x08002335   Thumb Code     0  printf2.o(i.__0sprintf$2)
    __scatterload_copy                       0x0800235d   Thumb Code    14  handlers.o(i.__scatterload_copy)
    __scatterload_null                       0x0800236b   Thumb Code     2  handlers.o(i.__scatterload_null)
    __scatterload_zeroinit                   0x0800236d   Thumb Code    14  handlers.o(i.__scatterload_zeroinit)
    dhcp_arp_reply                           0x080024a9   Thumb Code    30  dhcp.o(i.dhcp_arp_reply)
    dhcp_coarse_tmr                          0x080025b9   Thumb Code    90  dhcp.o(i.dhcp_coarse_tmr)
    dhcp_fine_tmr                            0x08002889   Thumb Code    46  dhcp.o(i.dhcp_fine_tmr)
    dhcp_release                             0x08002aa5   Thumb Code   160  dhcp.o(i.dhcp_release)
    dhcp_renew                               0x08002b49   Thumb Code   132  dhcp.o(i.dhcp_renew)
    etharp_cleanup_netif                     0x08002e55   Thumb Code    42  etharp.o(i.etharp_cleanup_netif)
    etharp_output                            0x08002f9d   Thumb Code   246  etharp.o(i.etharp_output)
    etharp_query                             0x080030e5   Thumb Code   228  etharp.o(i.etharp_query)
    etharp_request                           0x08003271   Thumb Code    32  etharp.o(i.etharp_request)
    etharp_tmr                               0x080032b5   Thumb Code    68  etharp.o(i.etharp_tmr)
    ethernet_input                           0x08003379   Thumb Code   138  etharp.o(i.ethernet_input)
    ethernetif_init                          0x08003409   Thumb Code    30  ethernetif.o(i.ethernetif_init)
    ethernetif_input                         0x08003431   Thumb Code    34  ethernetif.o(i.ethernetif_input)
    ethernetif_notify_conn_changed           0x08003455   Thumb Code    54  app_ethernet.o(i.ethernetif_notify_conn_changed)
    ethernetif_update_config                 0x08003495   Thumb Code   170  ethernetif.o(i.ethernetif_update_config)
    icmp_dest_unreach                        0x08003a79   Thumb Code     8  icmp.o(i.icmp_dest_unreach)
    icmp_input                               0x08003a81   Thumb Code   242  icmp.o(i.icmp_input)
    icmp_time_exceeded                       0x08003be1   Thumb Code     8  icmp.o(i.icmp_time_exceeded)
    inet_chksum                              0x08003be9   Thumb Code    12  inet_chksum.o(i.inet_chksum)
    inet_chksum_pbuf                         0x08003bf5   Thumb Code    72  inet_chksum.o(i.inet_chksum_pbuf)
    ip4_addr_isbroadcast                     0x08003c3d   Thumb Code    46  ip_addr.o(i.ip4_addr_isbroadcast)
    ip_frag                                  0x08003c6d   Thumb Code   352  ip_frag.o(i.ip_frag)
    ip_input                                 0x08003dd9   Thumb Code   372  ip.o(i.ip_input)
    ip_output                                0x08003f55   Thumb Code    52  ip.o(i.ip_output)
    ip_output_if                             0x08003f89   Thumb Code   164  ip.o(i.ip_output_if)
    ip_reass                                 0x08004031   Thumb Code   392  ip_frag.o(i.ip_reass)
    ip_reass_tmr                             0x080043c1   Thumb Code    40  ip_frag.o(i.ip_reass_tmr)
    ip_route                                 0x080043ed   Thumb Code    54  ip.o(i.ip_route)
    lwip_htonl                               0x08004669   Thumb Code     4  def.o(i.lwip_htonl)
    lwip_htons                               0x0800466d   Thumb Code     4  def.o(i.lwip_htons)
    lwip_init                                0x08004671   Thumb Code    30  init.o(i.lwip_init)
    lwip_ntohl                               0x0800468f   Thumb Code     4  def.o(i.lwip_ntohl)
    lwip_ntohs                               0x08004693   Thumb Code     4  def.o(i.lwip_ntohs)
    main                                     0x080046f1   Thumb Code   324  main.o(i.main)
    mem_free                                 0x08004859   Thumb Code    40  mem.o(i.mem_free)
    mem_init                                 0x08004885   Thumb Code    42  mem.o(i.mem_init)
    mem_malloc                               0x080048b9   Thumb Code   162  mem.o(i.mem_malloc)
    mem_trim                                 0x08004961   Thumb Code   200  mem.o(i.mem_trim)
    memp_free                                0x08004a2d   Thumb Code    18  memp.o(i.memp_free)
    memp_init                                0x08004a45   Thumb Code    78  memp.o(i.memp_init)
    memp_malloc                              0x08004a9d   Thumb Code    28  memp.o(i.memp_malloc)
    netif_add                                0x08004abd   Thumb Code    72  netif.o(i.netif_add)
    netif_init                               0x08004b09   Thumb Code     2  netif.o(i.netif_init)
    netif_set_addr                           0x08004b0b   Thumb Code    32  netif.o(i.netif_set_addr)
    netif_set_default                        0x08004b2d   Thumb Code     6  netif.o(i.netif_set_default)
    netif_set_down                           0x08004b39   Thumb Code    26  netif.o(i.netif_set_down)
    netif_set_gw                             0x08004b53   Thumb Code     8  netif.o(i.netif_set_gw)
    netif_set_ipaddr                         0x08004b5d   Thumb Code    96  netif.o(i.netif_set_ipaddr)
    netif_set_link_callback                  0x08004bc5   Thumb Code     8  netif.o(i.netif_set_link_callback)
    netif_set_netmask                        0x08004bcd   Thumb Code     8  netif.o(i.netif_set_netmask)
    netif_set_up                             0x08004bd5   Thumb Code    32  netif.o(i.netif_set_up)
    pbuf_alloc                               0x08004bf5   Thumb Code   280  pbuf.o(i.pbuf_alloc)
    pbuf_alloced_custom                      0x08004d0d   Thumb Code    84  pbuf.o(i.pbuf_alloced_custom)
    pbuf_cat                                 0x08004d61   Thumb Code    40  pbuf.o(i.pbuf_cat)
    pbuf_chain                               0x08004d89   Thumb Code    18  pbuf.o(i.pbuf_chain)
    pbuf_clen                                0x08004d9b   Thumb Code    18  pbuf.o(i.pbuf_clen)
    pbuf_copy                                0x08004dad   Thumb Code   154  pbuf.o(i.pbuf_copy)
    pbuf_copy_partial                        0x08004e47   Thumb Code   104  pbuf.o(i.pbuf_copy_partial)
    pbuf_free                                0x08004eaf   Thumb Code    80  pbuf.o(i.pbuf_free)
    pbuf_header                              0x08004eff   Thumb Code    96  pbuf.o(i.pbuf_header)
    pbuf_realloc                             0x08004f5f   Thumb Code    78  pbuf.o(i.pbuf_realloc)
    pbuf_ref                                 0x08004fad   Thumb Code    12  pbuf.o(i.pbuf_ref)
    raw_input                                0x0800500d   Thumb Code   104  raw.o(i.raw_input)
    sys_check_timeouts                       0x080050ad   Thumb Code    68  lwip_timers.o(i.sys_check_timeouts)
    sys_now                                  0x080050f5   Thumb Code     4  ethernetif.o(i.sys_now)
    sys_timeout                              0x080050f9   Thumb Code    88  lwip_timers.o(i.sys_timeout)
    sys_timeouts_init                        0x08005155   Thumb Code    60  lwip_timers.o(i.sys_timeouts_init)
    tcp_abandon                              0x080051a5   Thumb Code   136  tcp.o(i.tcp_abandon)
    tcp_abort                                0x08005231   Thumb Code     6  tcp.o(i.tcp_abort)
    tcp_accept                               0x08005237   Thumb Code     4  tcp.o(i.tcp_accept)
    tcp_alloc                                0x08005241   Thumb Code   236  tcp.o(i.tcp_alloc)
    tcp_arg                                  0x08005339   Thumb Code     4  tcp.o(i.tcp_arg)
    tcp_bind                                 0x0800533d   Thumb Code   122  tcp.o(i.tcp_bind)
    tcp_close                                0x080053c1   Thumb Code    20  tcp.o(i.tcp_close)
    tcp_eff_send_mss                         0x08005599   Thumb Code    32  tcp.o(i.tcp_eff_send_mss)
    tcp_enqueue_flags                        0x080055b9   Thumb Code   166  tcp_out.o(i.tcp_enqueue_flags)
    tcp_err                                  0x0800565f   Thumb Code     6  tcp.o(i.tcp_err)
    tcp_fasttmr                              0x08005665   Thumb Code    90  tcp.o(i.tcp_fasttmr)
    tcp_init                                 0x080056c5   Thumb Code     2  tcp.o(i.tcp_init)
    tcp_input                                0x080056c9   Thumb Code   758  tcp_in.o(i.tcp_input)
    tcp_keepalive                            0x080059dd   Thumb Code    60  tcp_out.o(i.tcp_keepalive)
    tcp_listen_with_backlog                  0x08005afd   Thumb Code   126  tcp.o(i.tcp_listen_with_backlog)
    tcp_new                                  0x08005b85   Thumb Code     6  tcp.o(i.tcp_new)
    tcp_next_iss                             0x08005be9   Thumb Code    12  tcp.o(i.tcp_next_iss)
    tcp_output                               0x08005bf9   Thumb Code   392  tcp_out.o(i.tcp_output)
    tcp_pcb_purge                            0x08005f6f   Thumb Code    58  tcp.o(i.tcp_pcb_purge)
    tcp_pcb_remove                           0x08005fa9   Thumb Code    82  tcp.o(i.tcp_pcb_remove)
    tcp_poll                                 0x08006001   Thumb Code    10  tcp.o(i.tcp_poll)
    tcp_process_refused_data                 0x08006341   Thumb Code   102  tcp.o(i.tcp_process_refused_data)
    tcp_recv                                 0x080067bb   Thumb Code     4  tcp.o(i.tcp_recv)
    tcp_recv_null                            0x080067bf   Thumb Code    36  tcp.o(i.tcp_recv_null)
    tcp_recved                               0x080067e3   Thumb Code    56  tcp.o(i.tcp_recved)
    tcp_rexmit                               0x0800681b   Thumb Code    82  tcp_out.o(i.tcp_rexmit)
    tcp_rexmit_fast                          0x0800686d   Thumb Code    88  tcp_out.o(i.tcp_rexmit_fast)
    tcp_rexmit_rto                           0x080068c5   Thumb Code    46  tcp_out.o(i.tcp_rexmit_rto)
    tcp_rst                                  0x080068f3   Thumb Code   118  tcp_out.o(i.tcp_rst)
    tcp_seg_free                             0x08006969   Thumb Code    28  tcp.o(i.tcp_seg_free)
    tcp_segs_free                            0x08006985   Thumb Code    18  tcp.o(i.tcp_segs_free)
    tcp_send_empty_ack                       0x08006997   Thumb Code    72  tcp_out.o(i.tcp_send_empty_ack)
    tcp_send_fin                             0x080069df   Thumb Code    68  tcp_out.o(i.tcp_send_fin)
    tcp_sent                                 0x08006a23   Thumb Code     4  tcp.o(i.tcp_sent)
    tcp_slowtmr                              0x08006a29   Thumb Code   588  tcp.o(i.tcp_slowtmr)
    tcp_timer_needed                         0x08006c85   Thumb Code    36  lwip_timers.o(i.tcp_timer_needed)
    tcp_tmr                                  0x08006d25   Thumb Code    28  tcp.o(i.tcp_tmr)
    tcp_update_rcv_ann_wnd                   0x08006d45   Thumb Code    52  tcp.o(i.tcp_update_rcv_ann_wnd)
    tcp_write                                0x08006d79   Thumb Code   764  tcp_out.o(i.tcp_write)
    tcp_zero_window_probe                    0x08007075   Thumb Code   138  tcp_out.o(i.tcp_zero_window_probe)
    udp_bind                                 0x08007139   Thumb Code   148  udp.o(i.udp_bind)
    udp_init                                 0x080071d1   Thumb Code     2  udp.o(i.udp_init)
    udp_input                                0x080071d5   Thumb Code   364  udp.o(i.udp_input)
    udp_sendto_if                            0x0800734d   Thumb Code   182  udp.o(i.udp_sendto_if)
    tcp_persist_backoff                      0x0800742c   Data           7  tcp.o(.constdata)
    tcp_state_str                            0x08007434   Data          44  tcp.o(.constdata)
    tcp_backoff                              0x08007460   Data          13  tcp.o(.constdata)
    tcp_pcb_lists                            0x08007470   Data          16  tcp.o(.constdata)
    ip_addr_any                              0x08007480   Data           4  ip_addr.o(.constdata)
    ip_addr_broadcast                        0x08007484   Data           4  ip_addr.o(.constdata)
    ethbroadcast                             0x08007488   Data           6  etharp.o(.constdata)
    ethzero                                  0x0800748e   Data           6  etharp.o(.constdata)
    APBAHBPrescTable                         0x08007494   Data          16  stm32f4xx_hal_rcc.o(.constdata)
    file_index_html                          0x08007d8c   Data          16  httpserver.o(.constdata)
    file_reset_html                          0x08007d9c   Data          16  httpserver.o(.constdata)
    file_upload_html                         0x08007dac   Data          16  httpserver.o(.constdata)
    file_uploaddone_html                     0x08007dc0   Data          16  httpserver.o(.constdata)
    Region$$Table$$Base                      0x08007e68   Number         0  anon$$obj.o(Region$$Table)
    Region$$Table$$Limit                     0x08007e88   Number         0  anon$$obj.o(Region$$Table)
    SystemCoreClock                          0x20000000   Data           4  system_stm32f4xx.o(.data)
    AHBPrescTable                            0x20000004   Data          16  system_stm32f4xx.o(.data)
    tcp_input_pcb                            0x2000002c   Data           4  tcp_in.o(.data)
    udp_pcbs                                 0x20000044   Data           4  udp.o(.data)
    netif_list                               0x20000058   Data           4  netif.o(.data)
    netif_default                            0x2000005c   Data           4  netif.o(.data)
    tcp_active_pcbs_changed                  0x20000060   Data           1  tcp.o(.data)
    tcp_ticks                                0x2000006c   Data           4  tcp.o(.data)
    tcp_bound_pcbs                           0x20000070   Data           4  tcp.o(.data)
    tcp_listen_pcbs                          0x20000074   Data           4  tcp.o(.data)
    tcp_active_pcbs                          0x20000078   Data           4  tcp.o(.data)
    tcp_tw_pcbs                              0x2000007c   Data           4  tcp.o(.data)
    tcp_tmp_pcb                              0x20000080   Data           4  tcp.o(.data)
    current_netif                            0x20000094   Data           4  ip.o(.data)
    current_header                           0x20000098   Data           4  ip.o(.data)
    current_iphdr_src                        0x2000009c   Data           4  ip.o(.data)
    current_iphdr_dest                       0x200000a0   Data           4  ip.o(.data)
    uwTick                                   0x200000a8   Data           4  stm32f4xx_hal.o(.data)
    htmlpage                                 0x200000ae   Data           1  httpserver.o(.data)
    Update_EPPROM                            0x200000d0   Data           1  main.o(.data)
    Jump_To_Application                      0x200000d4   Data           4  main.o(.data)
    JumpAddress                              0x200000d8   Data           4  main.o(.data)
    EEPROMDataWrite                          0x200000dc   Data           1  stm324xg_eval_eeprom.o(.data)
    ram_heap                                 0x2000491f   Data       10260  mem.o(.bss)
    pFlash                                   0x200071fc   Data          32  stm32f4xx_hal_flash.o(.bss)
    DMARxDscrTab                             0x2000721c   Data         128  ethernetif.o(.bss)
    DMATxDscrTab                             0x2000729c   Data         128  ethernetif.o(.bss)
    Rx_Buff                                  0x2000731c   Data        6096  ethernetif.o(.bss)
    Tx_Buff                                  0x20008aec   Data        6096  ethernetif.o(.bss)
    EthHandle                                0x2000a2bc   Data          72  ethernetif.o(.bss)
    gnetif                                   0x2000a304   Data          56  main.o(.bss)
    hi2c1                                    0x2000a33c   Data          68  main.o(.bss)
    __initial_sp                             0x2000ab80   Data           0  startup_stm32f407xx.o(STACK)



==============================================================================

Memory Map of the image

  Image Entry point : 0x08000189

  Load Region LR_IROM1 (Base: 0x08000000, Size: 0x00007f68, Max: 0x00080000, ABSOLUTE)

    Execution Region ER_IROM1 (Base: 0x08000000, Size: 0x00007e88, Max: 0x00080000, ABSOLUTE)

    Base Addr    Size         Type   Attr      Idx    E Section Name        Object

    0x08000000   0x00000188   Data   RO         3645    RESET               startup_stm32f407xx.o
    0x08000188   0x00000000   Code   RO         4173  * .ARM.Collect$$$$00000000  mc_w.l(entry.o)
    0x08000188   0x00000004   Code   RO         4451    .ARM.Collect$$$$00000001  mc_w.l(entry2.o)
    0x0800018c   0x00000004   Code   RO         4454    .ARM.Collect$$$$00000004  mc_w.l(entry5.o)
    0x08000190   0x00000000   Code   RO         4456    .ARM.Collect$$$$00000008  mc_w.l(entry7b.o)
    0x08000190   0x00000000   Code   RO         4458    .ARM.Collect$$$$0000000A  mc_w.l(entry8b.o)
    0x08000190   0x00000008   Code   RO         4459    .ARM.Collect$$$$0000000B  mc_w.l(entry9a.o)
    0x08000198   0x00000000   Code   RO         4461    .ARM.Collect$$$$0000000D  mc_w.l(entry10a.o)
    0x08000198   0x00000000   Code   RO         4463    .ARM.Collect$$$$0000000F  mc_w.l(entry11a.o)
    0x08000198   0x00000004   Code   RO         4452    .ARM.Collect$$$$00002712  mc_w.l(entry2.o)
    0x0800019c   0x00000024   Code   RO         3646    .text               startup_stm32f407xx.o
    0x080001c0   0x00000024   Code   RO         4176    .text               mc_w.l(memcpya.o)
    0x080001e4   0x00000024   Code   RO         4178    .text               mc_w.l(memseta.o)
    0x08000208   0x0000001c   Code   RO         4182    .text               mc_w.l(strcmp.o)
    0x08000224   0x0000001a   Code   RO         4184    .text               mc_w.l(memcmp.o)
    0x0800023e   0x0000001e   Code   RO         4186    .text               mc_w.l(strncmp.o)
    0x0800025c   0x00000024   Code   RO         4483    .text               mc_w.l(init.o)
    0x08000280   0x00000002   Code   RO         4081    i.BSP_EEPROM_TIMEOUT_UserCallback  stm324xg_eval_eeprom.o
    0x08000282   0x000000f8   Code   RO         4082    i.BSP_EEPROM_WriteBuffer  stm324xg_eval_eeprom.o
    0x0800037a   0x00000002   Code   RO         3959    i.BusFault_Handler  stm32f4xx_it.o
    0x0800037c   0x00000002   Code   RO         3960    i.DebugMon_Handler  stm32f4xx_it.o
    0x0800037e   0x00000002   PAD
    0x08000380   0x00000010   Code   RO         4132    i.EEPROM_IO_IsDeviceReady  stm324xg_eval.o
    0x08000390   0x0000002c   Code   RO         4134    i.EEPROM_IO_WriteData  stm324xg_eval.o
    0x080003bc   0x00000038   Code   RO         4083    i.EEPROM_WritePage  stm324xg_eval_eeprom.o
    0x080003f4   0x0000002e   Code   RO         3415    i.ETH_FlushTransmitFIFO  stm32f4xx_hal_eth.o
    0x08000422   0x00000002   PAD
    0x08000424   0x00000124   Code   RO         3416    i.ETH_MACDMAConfig  stm32f4xx_hal_eth.o
    0x08000548   0x00000008   Code   RO         3961    i.EXTI15_10_IRQHandler  stm32f4xx_it.o
    0x08000550   0x00000058   Code   RO         1761    i.FLASH_Erase_Sector  stm32f4xx_hal_flash_ex.o
    0x080005a8   0x00000054   Code   RO         1762    i.FLASH_FlushCaches  stm32f4xx_hal_flash_ex.o
    0x080005fc   0x00000034   Code   RO         3859    i.FLASH_If_Erase    flash_if.o
    0x08000630   0x00000004   Code   RO         3860    i.FLASH_If_Init     flash_if.o
    0x08000634   0x00000050   Code   RO         3861    i.FLASH_If_Write    flash_if.o
    0x08000684   0x00000028   Code   RO         1763    i.FLASH_MassErase   stm32f4xx_hal_flash_ex.o
    0x080006ac   0x00000020   Code   RO         1930    i.FLASH_Program_Byte  stm32f4xx_hal_flash.o
    0x080006cc   0x00000028   Code   RO         1931    i.FLASH_Program_DoubleWord  stm32f4xx_hal_flash.o
    0x080006f4   0x00000024   Code   RO         1932    i.FLASH_Program_HalfWord  stm32f4xx_hal_flash.o
    0x08000718   0x00000024   Code   RO         1933    i.FLASH_Program_Word  stm32f4xx_hal_flash.o
    0x0800073c   0x00000088   Code   RO         1934    i.FLASH_SetErrorCode  stm32f4xx_hal_flash.o
    0x080007c4   0x00000058   Code   RO         1935    i.FLASH_WaitForLastOperation  stm32f4xx_hal_flash.o
    0x0800081c   0x00000016   Code   RO         2055    i.HAL_Delay         stm32f4xx_hal.o
    0x08000832   0x00000002   PAD
    0x08000834   0x00000130   Code   RO         3418    i.HAL_ETH_ConfigMAC  stm32f4xx_hal_eth.o
    0x08000964   0x00000074   Code   RO         3419    i.HAL_ETH_DMARxDescListInit  stm32f4xx_hal_eth.o
    0x080009d8   0x00000078   Code   RO         3420    i.HAL_ETH_DMATxDescListInit  stm32f4xx_hal_eth.o
    0x08000a50   0x0000007a   Code   RO         3423    i.HAL_ETH_GetReceivedFrame  stm32f4xx_hal_eth.o
    0x08000aca   0x00000002   PAD
    0x08000acc   0x000001ec   Code   RO         3427    i.HAL_ETH_Init      stm32f4xx_hal_eth.o
    0x08000cb8   0x00000002   Code   RO         3778    i.HAL_ETH_MspInit   ethernetif.o
    0x08000cba   0x00000002   PAD
    0x08000cbc   0x00000084   Code   RO         3430    i.HAL_ETH_ReadPHYRegister  stm32f4xx_hal_eth.o
    0x08000d40   0x00000084   Code   RO         3432    i.HAL_ETH_Start     stm32f4xx_hal_eth.o
    0x08000dc4   0x00000084   Code   RO         3433    i.HAL_ETH_Stop      stm32f4xx_hal_eth.o
    0x08000e48   0x00000108   Code   RO         3434    i.HAL_ETH_TransmitFrame  stm32f4xx_hal_eth.o
    0x08000f50   0x00000078   Code   RO         3436    i.HAL_ETH_WritePHYRegister  stm32f4xx_hal_eth.o
    0x08000fc8   0x00000098   Code   RO         1764    i.HAL_FLASHEx_Erase  stm32f4xx_hal_flash_ex.o
    0x08001060   0x0000007c   Code   RO         1944    i.HAL_FLASH_Program  stm32f4xx_hal_flash.o
    0x080010dc   0x00000028   Code   RO         1946    i.HAL_FLASH_Unlock  stm32f4xx_hal_flash.o
    0x08001104   0x00000002   Code   RO         2196    i.HAL_GPIO_EXTI_Callback  stm32f4xx_hal_gpio.o
    0x08001106   0x00000002   PAD
    0x08001108   0x00000018   Code   RO         2197    i.HAL_GPIO_EXTI_IRQHandler  stm32f4xx_hal_gpio.o
    0x08001120   0x000001c0   Code   RO         2198    i.HAL_GPIO_Init     stm32f4xx_hal_gpio.o
    0x080012e0   0x0000000a   Code   RO         2200    i.HAL_GPIO_ReadPin  stm32f4xx_hal_gpio.o
    0x080012ea   0x0000000a   Code   RO         2202    i.HAL_GPIO_WritePin  stm32f4xx_hal_gpio.o
    0x080012f4   0x0000000c   Code   RO         2060    i.HAL_GetREVID      stm32f4xx_hal.o
    0x08001300   0x0000000c   Code   RO         2061    i.HAL_GetTick       stm32f4xx_hal.o
    0x0800130c   0x00000032   Code   RO         3024    i.HAL_I2C_DeInit    stm32f4xx_hal_i2c.o
    0x0800133e   0x00000006   Code   RO         3032    i.HAL_I2C_GetState  stm32f4xx_hal_i2c.o
    0x08001344   0x00000108   Code   RO         3033    i.HAL_I2C_Init      stm32f4xx_hal_i2c.o
    0x0800144c   0x0000014c   Code   RO         3034    i.HAL_I2C_IsDeviceReady  stm32f4xx_hal_i2c.o
    0x08001598   0x000000f4   Code   RO         3052    i.HAL_I2C_Mem_Write  stm32f4xx_hal_i2c.o
    0x0800168c   0x00000002   Code   RO         3055    i.HAL_I2C_MspDeInit  stm32f4xx_hal_i2c.o
    0x0800168e   0x00000002   Code   RO         3056    i.HAL_I2C_MspInit   stm32f4xx_hal_i2c.o
    0x08001690   0x00000010   Code   RO         2062    i.HAL_IncTick       stm32f4xx_hal.o
    0x080016a0   0x0000002c   Code   RO         2063    i.HAL_Init          stm32f4xx_hal.o
    0x080016cc   0x00000022   Code   RO         2064    i.HAL_InitTick      stm32f4xx_hal.o
    0x080016ee   0x00000002   Code   RO         2066    i.HAL_MspInit       stm32f4xx_hal.o
    0x080016f0   0x00000016   Code   RO         2666    i.HAL_NVIC_EnableIRQ  stm32f4xx_hal_cortex.o
    0x08001706   0x00000002   PAD
    0x08001708   0x00000040   Code   RO         2672    i.HAL_NVIC_SetPriority  stm32f4xx_hal_cortex.o
    0x08001748   0x00000024   Code   RO         2673    i.HAL_NVIC_SetPriorityGrouping  stm32f4xx_hal_cortex.o
    0x0800176c   0x00000140   Code   RO         1826    i.HAL_RCC_ClockConfig  stm32f4xx_hal_rcc.o
    0x080018ac   0x00000034   Code   RO         1831    i.HAL_RCC_GetHCLKFreq  stm32f4xx_hal_rcc.o
    0x080018e0   0x0000002c   Code   RO         1833    i.HAL_RCC_GetPCLK1Freq  stm32f4xx_hal_rcc.o
    0x0800190c   0x00000074   Code   RO         1835    i.HAL_RCC_GetSysClockFreq  stm32f4xx_hal_rcc.o
    0x08001980   0x000002e4   Code   RO         1838    i.HAL_RCC_OscConfig  stm32f4xx_hal_rcc.o
    0x08001c64   0x00000028   Code   RO         2677    i.HAL_SYSTICK_Config  stm32f4xx_hal_cortex.o
    0x08001c8c   0x00000002   Code   RO         3962    i.HardFault_Handler  stm32f4xx_it.o
    0x08001c8e   0x00000002   PAD
    0x08001c90   0x00000068   Code   RO         3895    i.I2C_Config        main.o
    0x08001cf8   0x00000028   Code   RO         3074    i.I2C_IsAcknowledgeFailed  stm32f4xx_hal_i2c.o
    0x08001d20   0x00000098   Code   RO         3081    i.I2C_RequestMemoryWrite  stm32f4xx_hal_i2c.o
    0x08001db8   0x0000008e   Code   RO         3084    i.I2C_WaitOnFlagUntilTimeout  stm32f4xx_hal_i2c.o
    0x08001e46   0x00000002   PAD
    0x08001e48   0x0000008c   Code   RO         3085    i.I2C_WaitOnMasterAddressFlagUntilTimeout  stm32f4xx_hal_i2c.o
    0x08001ed4   0x00000052   Code   RO         3088    i.I2C_WaitOnTXEFlagUntilTimeout  stm32f4xx_hal_i2c.o
    0x08001f26   0x00000002   PAD
    0x08001f28   0x00000088   Code   RO         3653    i.IAP_HTTP_writedata  httpserver.o
    0x08001fb0   0x0000002c   Code   RO         3654    i.IAP_httpd_init    httpserver.o
    0x08001fdc   0x0000014c   Code   RO         3896    i.Init_Config       main.o
    0x08002128   0x00000002   Code   RO         3963    i.MemManage_Handler  stm32f4xx_it.o
    0x0800212a   0x00000002   Code   RO         3964    i.NMI_Handler       stm32f4xx_it.o
    0x0800212c   0x00000020   Code   RO         2679    i.NVIC_SetPriority  stm32f4xx_hal_cortex.o
    0x0800214c   0x00000024   Code   RO         3655    i.NVIC_SystemReset  httpserver.o
    0x08002170   0x00000068   Code   RO         3897    i.Netif_Config      main.o
    0x080021d8   0x00000070   Code   RO         3656    i.Parse_Content_Length  httpserver.o
    0x08002248   0x00000004   Code   RO         3965    i.SysTick_Handler   stm32f4xx_it.o
    0x0800224c   0x00000090   Code   RO         3898    i.SystemClock_Config  main.o
    0x080022dc   0x00000054   Code   RO            5    i.SystemInit        system_stm32f4xx.o
    0x08002330   0x00000002   Code   RO         3966    i.UsageFault_Handler  stm32f4xx_it.o
    0x08002332   0x00000002   Code   RO         4028    i.User_notification  app_ethernet.o
    0x08002334   0x00000028   Code   RO         4259    i.__0sprintf$2      mc_w.l(printf2.o)
    0x0800235c   0x0000000e   Code   RO         4497    i.__scatterload_copy  mc_w.l(handlers.o)
    0x0800236a   0x00000002   Code   RO         4498    i.__scatterload_null  mc_w.l(handlers.o)
    0x0800236c   0x0000000e   Code   RO         4499    i.__scatterload_zeroinit  mc_w.l(handlers.o)
    0x0800237a   0x000000d6   Code   RO         4264    i._printf_core      mc_w.l(printf2.o)
    0x08002450   0x0000000a   Code   RO         4266    i._sputc            mc_w.l(printf2.o)
    0x0800245a   0x00000002   PAD
    0x0800245c   0x0000001c   Code   RO          277    i.arp_timer         lwip_timers.o
    0x08002478   0x0000002c   Code   RO         3657    i.close_conn        httpserver.o
    0x080024a4   0x00000004   Code   RO         3658    i.conn_err          httpserver.o
    0x080024a8   0x0000001e   Code   RO          452    i.dhcp_arp_reply    dhcp.o
    0x080024c6   0x000000c0   Code   RO          453    i.dhcp_bind         dhcp.o
    0x08002586   0x00000030   Code   RO          454    i.dhcp_check        dhcp.o
    0x080025b6   0x00000002   PAD
    0x080025b8   0x00000060   Code   RO          456    i.dhcp_coarse_tmr   dhcp.o
    0x08002618   0x00000124   Code   RO          457    i.dhcp_create_msg   dhcp.o
    0x0800273c   0x00000078   Code   RO          458    i.dhcp_decline      dhcp.o
    0x080027b4   0x00000016   Code   RO          459    i.dhcp_delete_msg   dhcp.o
    0x080027ca   0x00000002   PAD
    0x080027cc   0x000000bc   Code   RO          460    i.dhcp_discover     dhcp.o
    0x08002888   0x00000034   Code   RO          461    i.dhcp_fine_tmr     dhcp.o
    0x080028bc   0x00000020   Code   RO          465    i.dhcp_option       dhcp.o
    0x080028dc   0x00000010   Code   RO          466    i.dhcp_option_byte  dhcp.o
    0x080028ec   0x00000042   Code   RO          467    i.dhcp_option_long  dhcp.o
    0x0800292e   0x00000022   Code   RO          468    i.dhcp_option_short  dhcp.o
    0x08002950   0x0000002c   Code   RO          469    i.dhcp_option_trailer  dhcp.o
    0x0800297c   0x00000088   Code   RO          471    i.dhcp_rebind       dhcp.o
    0x08002a04   0x000000a0   Code   RO          472    i.dhcp_reboot       dhcp.o
    0x08002aa4   0x000000a4   Code   RO          474    i.dhcp_release      dhcp.o
    0x08002b48   0x00000084   Code   RO          475    i.dhcp_renew        dhcp.o
    0x08002bcc   0x000000e8   Code   RO          476    i.dhcp_select       dhcp.o
    0x08002cb4   0x00000010   Code   RO          477    i.dhcp_set_state    dhcp.o
    0x08002cc4   0x00000088   Code   RO          481    i.dhcp_timeout      dhcp.o
    0x08002d4c   0x0000001c   Code   RO          278    i.dhcp_timer_coarse  lwip_timers.o
    0x08002d68   0x0000001c   Code   RO          279    i.dhcp_timer_fine   lwip_timers.o
    0x08002d84   0x000000ce   Code   RO         1667    i.etharp_arp_input  etharp.o
    0x08002e52   0x00000002   PAD
    0x08002e54   0x00000030   Code   RO         1668    i.etharp_cleanup_netif  etharp.o
    0x08002e84   0x000000dc   Code   RO         1670    i.etharp_find_entry  etharp.o
    0x08002f60   0x0000003c   Code   RO         1671    i.etharp_free_entry  etharp.o
    0x08002f9c   0x00000104   Code   RO         1672    i.etharp_output     etharp.o
    0x080030a0   0x00000044   Code   RO         1673    i.etharp_output_to_arp_index  etharp.o
    0x080030e4   0x000000ec   Code   RO         1674    i.etharp_query      etharp.o
    0x080031d0   0x000000a0   Code   RO         1675    i.etharp_raw        etharp.o
    0x08003270   0x00000024   Code   RO         1676    i.etharp_request    etharp.o
    0x08003294   0x00000020   Code   RO         1677    i.etharp_send_ip    etharp.o
    0x080032b4   0x00000048   Code   RO         1678    i.etharp_tmr        etharp.o
    0x080032fc   0x0000007c   Code   RO         1679    i.etharp_update_arp_entry  etharp.o
    0x08003378   0x00000090   Code   RO         1680    i.ethernet_input    etharp.o
    0x08003408   0x00000028   Code   RO         3779    i.ethernetif_init   ethernetif.o
    0x08003430   0x00000022   Code   RO         3780    i.ethernetif_input  ethernetif.o
    0x08003452   0x00000002   PAD
    0x08003454   0x00000040   Code   RO         4029    i.ethernetif_notify_conn_changed  app_ethernet.o
    0x08003494   0x000000b0   Code   RO         3783    i.ethernetif_update_config  ethernetif.o
    0x08003544   0x00000030   Code   RO         3659    i.fs_open           httpserver.o
    0x08003574   0x0000004c   Code   RO         3660    i.http_accept       httpserver.o
    0x080035c0   0x0000001a   Code   RO         3661    i.http_poll         httpserver.o
    0x080035da   0x00000002   PAD
    0x080035dc   0x0000042c   Code   RO         3662    i.http_recv         httpserver.o
    0x08003a08   0x00000070   Code   RO         3663    i.http_sent         httpserver.o
    0x08003a78   0x00000008   Code   RO         1575    i.icmp_dest_unreach  icmp.o
    0x08003a80   0x000000fc   Code   RO         1576    i.icmp_input        icmp.o
    0x08003b7c   0x00000064   Code   RO         1577    i.icmp_send_response  icmp.o
    0x08003be0   0x00000008   Code   RO         1578    i.icmp_time_exceeded  icmp.o
    0x08003be8   0x0000000c   Code   RO         1436    i.inet_chksum       inet_chksum.o
    0x08003bf4   0x00000048   Code   RO         1437    i.inet_chksum_pbuf  inet_chksum.o
    0x08003c3c   0x0000002e   Code   RO         1382    i.ip4_addr_isbroadcast  ip_addr.o
    0x08003c6a   0x00000002   PAD
    0x08003c6c   0x00000164   Code   RO         1474    i.ip_frag           ip_frag.o
    0x08003dd0   0x00000008   Code   RO         1475    i.ip_frag_free_pbuf_custom_ref  ip_frag.o
    0x08003dd8   0x0000017c   Code   RO         1536    i.ip_input          ip.o
    0x08003f54   0x00000034   Code   RO         1537    i.ip_output         ip.o
    0x08003f88   0x000000a8   Code   RO         1538    i.ip_output_if      ip.o
    0x08004030   0x0000018c   Code   RO         1476    i.ip_reass          ip_frag.o
    0x080041bc   0x000000e8   Code   RO         1477    i.ip_reass_chain_frag_into_datagram_and_validate  ip_frag.o
    0x080042a4   0x00000024   Code   RO         1478    i.ip_reass_dequeue_datagram  ip_frag.o
    0x080042c8   0x00000070   Code   RO         1479    i.ip_reass_free_complete_datagram  ip_frag.o
    0x08004338   0x0000006c   Code   RO         1480    i.ip_reass_remove_oldest_datagram  ip_frag.o
    0x080043a4   0x0000001c   Code   RO          280    i.ip_reass_timer    lwip_timers.o
    0x080043c0   0x0000002c   Code   RO         1481    i.ip_reass_tmr      ip_frag.o
    0x080043ec   0x00000040   Code   RO         1539    i.ip_route          ip.o
    0x0800442c   0x00000016   Code   RO         1482    i.ipfrag_free_pbuf_custom  ip_frag.o
    0x08004442   0x00000002   PAD
    0x08004444   0x000000cc   Code   RO         3784    i.low_level_init    ethernetif.o
    0x08004510   0x000000b0   Code   RO         3785    i.low_level_input   ethernetif.o
    0x080045c0   0x000000a8   Code   RO         3786    i.low_level_output  ethernetif.o
    0x08004668   0x00000004   Code   RO          247    i.lwip_htonl        def.o
    0x0800466c   0x00000004   Code   RO          248    i.lwip_htons        def.o
    0x08004670   0x0000001e   Code   RO         1226    i.lwip_init         init.o
    0x0800468e   0x00000004   Code   RO          249    i.lwip_ntohl        def.o
    0x08004692   0x00000004   Code   RO          250    i.lwip_ntohs        def.o
    0x08004696   0x00000002   PAD
    0x08004698   0x00000058   Code   RO         1440    i.lwip_standard_chksum  inet_chksum.o
    0x080046f0   0x00000168   Code   RO         3899    i.main              main.o
    0x08004858   0x0000002c   Code   RO          713    i.mem_free          mem.o
    0x08004884   0x00000034   Code   RO          714    i.mem_init          mem.o
    0x080048b8   0x000000a8   Code   RO          715    i.mem_malloc        mem.o
    0x08004960   0x000000cc   Code   RO          716    i.mem_trim          mem.o
    0x08004a2c   0x00000018   Code   RO          393    i.memp_free         memp.o
    0x08004a44   0x00000058   Code   RO          394    i.memp_init         memp.o
    0x08004a9c   0x00000020   Code   RO          395    i.memp_malloc       memp.o
    0x08004abc   0x0000004c   Code   RO          763    i.netif_add         netif.o
    0x08004b08   0x00000002   Code   RO          765    i.netif_init        netif.o
    0x08004b0a   0x00000020   Code   RO          767    i.netif_set_addr    netif.o
    0x08004b2a   0x00000002   PAD
    0x08004b2c   0x0000000c   Code   RO          768    i.netif_set_default  netif.o
    0x08004b38   0x0000001a   Code   RO          769    i.netif_set_down    netif.o
    0x08004b52   0x00000008   Code   RO          770    i.netif_set_gw      netif.o
    0x08004b5a   0x00000002   PAD
    0x08004b5c   0x00000068   Code   RO          771    i.netif_set_ipaddr  netif.o
    0x08004bc4   0x00000008   Code   RO          772    i.netif_set_link_callback  netif.o
    0x08004bcc   0x00000008   Code   RO          775    i.netif_set_netmask  netif.o
    0x08004bd4   0x00000020   Code   RO          776    i.netif_set_up      netif.o
    0x08004bf4   0x00000118   Code   RO         1250    i.pbuf_alloc        pbuf.o
    0x08004d0c   0x00000054   Code   RO         1251    i.pbuf_alloced_custom  pbuf.o
    0x08004d60   0x00000028   Code   RO         1252    i.pbuf_cat          pbuf.o
    0x08004d88   0x00000012   Code   RO         1253    i.pbuf_chain        pbuf.o
    0x08004d9a   0x00000012   Code   RO         1254    i.pbuf_clen         pbuf.o
    0x08004dac   0x0000009a   Code   RO         1256    i.pbuf_copy         pbuf.o
    0x08004e46   0x00000068   Code   RO         1257    i.pbuf_copy_partial  pbuf.o
    0x08004eae   0x00000050   Code   RO         1259    i.pbuf_free         pbuf.o
    0x08004efe   0x00000060   Code   RO         1261    i.pbuf_header       pbuf.o
    0x08004f5e   0x0000004e   Code   RO         1264    i.pbuf_realloc      pbuf.o
    0x08004fac   0x0000000c   Code   RO         1265    i.pbuf_ref          pbuf.o
    0x08004fb8   0x00000054   Code   RO          717    i.plug_holes        mem.o
    0x0800500c   0x00000074   Code   RO         1166    i.raw_input         raw.o
    0x08005080   0x0000002c   Code   RO         3664    i.send_data         httpserver.o
    0x080050ac   0x00000048   Code   RO          281    i.sys_check_timeouts  lwip_timers.o
    0x080050f4   0x00000004   Code   RO         3787    i.sys_now           ethernetif.o
    0x080050f8   0x0000005c   Code   RO          283    i.sys_timeout       lwip_timers.o
    0x08005154   0x00000050   Code   RO          284    i.sys_timeouts_init  lwip_timers.o
    0x080051a4   0x0000008c   Code   RO          859    i.tcp_abandon       tcp.o
    0x08005230   0x00000006   Code   RO          860    i.tcp_abort         tcp.o
    0x08005236   0x00000004   Code   RO          861    i.tcp_accept        tcp.o
    0x0800523a   0x00000006   Code   RO          862    i.tcp_accept_null   tcp.o
    0x08005240   0x000000f8   Code   RO          863    i.tcp_alloc         tcp.o
    0x08005338   0x00000004   Code   RO          864    i.tcp_arg           tcp.o
    0x0800533c   0x00000084   Code   RO          865    i.tcp_bind          tcp.o
    0x080053c0   0x00000014   Code   RO          866    i.tcp_close         tcp.o
    0x080053d4   0x00000128   Code   RO          867    i.tcp_close_shutdown  tcp.o
    0x080054fc   0x0000009c   Code   RO         1072    i.tcp_create_segment  tcp_out.o
    0x08005598   0x00000020   Code   RO          870    i.tcp_eff_send_mss  tcp.o
    0x080055b8   0x000000a6   Code   RO         1073    i.tcp_enqueue_flags  tcp_out.o
    0x0800565e   0x00000006   Code   RO          871    i.tcp_err           tcp.o
    0x08005664   0x00000060   Code   RO          872    i.tcp_fasttmr       tcp.o
    0x080056c4   0x00000002   Code   RO          873    i.tcp_init          tcp.o
    0x080056c6   0x00000002   PAD
    0x080056c8   0x00000314   Code   RO          135    i.tcp_input         tcp_in.o
    0x080059dc   0x0000003c   Code   RO         1074    i.tcp_keepalive     tcp_out.o
    0x08005a18   0x000000e4   Code   RO          136    i.tcp_listen_input  tcp_in.o
    0x08005afc   0x00000088   Code   RO          874    i.tcp_listen_with_backlog  tcp.o
    0x08005b84   0x00000006   Code   RO          875    i.tcp_new           tcp.o
    0x08005b8a   0x00000002   PAD
    0x08005b8c   0x0000005c   Code   RO          876    i.tcp_new_port      tcp.o
    0x08005be8   0x00000010   Code   RO          877    i.tcp_next_iss      tcp.o
    0x08005bf8   0x0000018c   Code   RO         1075    i.tcp_output        tcp_out.o
    0x08005d84   0x0000006a   Code   RO         1076    i.tcp_output_alloc_header  tcp_out.o
    0x08005dee   0x00000002   PAD
    0x08005df0   0x000000b0   Code   RO         1077    i.tcp_output_segment  tcp_out.o
    0x08005ea0   0x00000080   Code   RO          137    i.tcp_parseopt      tcp_in.o
    0x08005f20   0x0000004e   Code   RO         1078    i.tcp_pbuf_prealloc  tcp_out.o
    0x08005f6e   0x0000003a   Code   RO          878    i.tcp_pcb_purge     tcp.o
    0x08005fa8   0x00000058   Code   RO          879    i.tcp_pcb_remove    tcp.o
    0x08006000   0x0000000a   Code   RO          880    i.tcp_poll          tcp.o
    0x0800600a   0x00000002   PAD
    0x0800600c   0x00000334   Code   RO          138    i.tcp_process       tcp_in.o
    0x08006340   0x00000066   Code   RO          881    i.tcp_process_refused_data  tcp.o
    0x080063a6   0x00000002   PAD
    0x080063a8   0x00000412   Code   RO          139    i.tcp_receive       tcp_in.o
    0x080067ba   0x00000004   Code   RO          882    i.tcp_recv          tcp.o
    0x080067be   0x00000024   Code   RO          883    i.tcp_recv_null     tcp.o
    0x080067e2   0x00000038   Code   RO          884    i.tcp_recved        tcp.o
    0x0800681a   0x00000052   Code   RO         1079    i.tcp_rexmit        tcp_out.o
    0x0800686c   0x00000058   Code   RO         1080    i.tcp_rexmit_fast   tcp_out.o
    0x080068c4   0x0000002e   Code   RO         1081    i.tcp_rexmit_rto    tcp_out.o
    0x080068f2   0x00000076   Code   RO         1082    i.tcp_rst           tcp_out.o
    0x08006968   0x0000001c   Code   RO          885    i.tcp_seg_free      tcp.o
    0x08006984   0x00000012   Code   RO          886    i.tcp_segs_free     tcp.o
    0x08006996   0x00000048   Code   RO         1083    i.tcp_send_empty_ack  tcp_out.o
    0x080069de   0x00000044   Code   RO         1084    i.tcp_send_fin      tcp_out.o
    0x08006a22   0x00000004   Code   RO          887    i.tcp_sent          tcp.o
    0x08006a26   0x00000002   PAD
    0x08006a28   0x0000025c   Code   RO          890    i.tcp_slowtmr       tcp.o
    0x08006c84   0x00000034   Code   RO          286    i.tcp_timer_needed  lwip_timers.o
    0x08006cb8   0x0000006c   Code   RO          140    i.tcp_timewait_input  tcp_in.o
    0x08006d24   0x00000020   Code   RO          891    i.tcp_tmr           tcp.o
    0x08006d44   0x00000034   Code   RO          892    i.tcp_update_rcv_ann_wnd  tcp.o
    0x08006d78   0x000002fc   Code   RO         1085    i.tcp_write         tcp_out.o
    0x08007074   0x0000008a   Code   RO         1086    i.tcp_zero_window_probe  tcp_out.o
    0x080070fe   0x00000002   PAD
    0x08007100   0x00000038   Code   RO          287    i.tcpip_tcp_timer   lwip_timers.o
    0x08007138   0x00000098   Code   RO          623    i.udp_bind          udp.o
    0x080071d0   0x00000002   Code   RO          626    i.udp_init          udp.o
    0x080071d2   0x00000002   PAD
    0x080071d4   0x00000178   Code   RO          627    i.udp_input         udp.o
    0x0800734c   0x000000b6   Code   RO          633    i.udp_sendto_if     udp.o
    0x08007402   0x00000028   Data   RO          397    .constdata          memp.o
    0x0800742a   0x00000002   PAD
    0x0800742c   0x00000054   Data   RO          893    .constdata          tcp.o
    0x08007480   0x00000004   Data   RO         1389    .constdata          ip_addr.o
    0x08007484   0x00000004   Data   RO         1390    .constdata          ip_addr.o
    0x08007488   0x0000000c   Data   RO         1682    .constdata          etharp.o
    0x08007494   0x00000010   Data   RO         1839    .constdata          stm32f4xx_hal_rcc.o
    0x080074a4   0x00000296   Data   RO         3665    .constdata          httpserver.o
    0x0800773a   0x0000019b   Data   RO         3666    .constdata          httpserver.o
    0x080078d5   0x0000027a   Data   RO         3667    .constdata          httpserver.o
    0x08007b4f   0x0000023b   Data   RO         3668    .constdata          httpserver.o
    0x08007d8a   0x00000002   PAD
    0x08007d8c   0x00000010   Data   RO         3669    .constdata          httpserver.o
    0x08007d9c   0x00000010   Data   RO         3670    .constdata          httpserver.o
    0x08007dac   0x00000010   Data   RO         3671    .constdata          httpserver.o
    0x08007dbc   0x00000033   Data   RO         3672    .constdata          httpserver.o
    0x08007def   0x00000001   PAD
    0x08007df0   0x00000075   Data   RO          894    .conststring        tcp.o
    0x08007e65   0x00000003   PAD
    0x08007e68   0x00000020   Data   RO         4495    Region$$Table       anon$$obj.o


    Execution Region RW_IRAM1 (Base: 0x20000000, Size: 0x0000ab80, Max: 0x00020000, ABSOLUTE)

    Base Addr    Size         Type   Attr      Idx    E Section Name        Object

    0x20000000   0x00000014   Data   RW            6    .data               system_stm32f4xx.o
    0x20000014   0x0000001c   Data   RW          142    .data               tcp_in.o
    0x20000030   0x0000000c   Data   RW          288    .data               lwip_timers.o
    0x2000003c   0x00000004   Data   RW          483    .data               dhcp.o
    0x20000040   0x00000008   Data   RW          634    .data               udp.o
    0x20000048   0x0000000c   Data   RW          719    .data               mem.o
    0x20000054   0x0000000c   Data   RW          777    .data               netif.o
    0x20000060   0x00000024   Data   RW          895    .data               tcp.o
    0x20000084   0x00000004   Data   RW         1172    .data               raw.o
    0x20000088   0x00000008   Data   RW         1483    .data               ip_frag.o
    0x20000090   0x00000014   Data   RW         1540    .data               ip.o
    0x200000a4   0x00000001   Data   RW         1683    .data               etharp.o
    0x200000a5   0x00000003   PAD
    0x200000a8   0x00000004   Data   RW         2069    .data               stm32f4xx_hal.o
    0x200000ac   0x00000024   Data   RW         3673    .data               httpserver.o
    0x200000d0   0x0000000c   Data   RW         3901    .data               main.o
    0x200000dc   0x00000001   Data   RW         4086    .data               stm324xg_eval_eeprom.o
    0x200000dd   0x00000003   PAD
    0x200000e0   0x00000014   Zero   RW          141    .bss                tcp_in.o
    0x200000f4   0x0000482b   Zero   RW          396    .bss                memp.o
    0x2000491f   0x00002814   Zero   RW          718    .bss                mem.o
    0x20007133   0x00000001   PAD
    0x20007134   0x000000c8   Zero   RW         1681    .bss                etharp.o
    0x200071fc   0x00000020   Zero   RW         1947    .bss                stm32f4xx_hal_flash.o
    0x2000721c   0x000030e8   Zero   RW         3788    .bss                ethernetif.o
    0x2000a304   0x0000007c   Zero   RW         3900    .bss                main.o
    0x2000a380   0x00000800   Zero   RW         3643    STACK               startup_stm32f407xx.o


==============================================================================

Image component sizes


      Code (inc. data)   RO Data    RW Data    ZI Data      Debug   Object Name

        66         10          0          0          0       1237   app_ethernet.o
        16          0          0          0          0       3052   def.o
      2208         50          0          4          0      18363   dhcp.o
      1666         68         12          1        200      16108   etharp.o
       804         52          0          0      12520       7126   ethernetif.o
       136         10          0          0          0       2414   flash_if.o
      1750        260       2377         36          0      42641   httpserver.o
       368         10          0          0          0       4138   icmp.o
         0          0          0          0          0       3960   inet.o
       172          0          0          0          0       3241   inet_chksum.o
        30          0          0          0          0        648   init.o
       664         22          0         20          0       8381   ip.o
        46          0          8          0          0       7822   ip_addr.o
      1314         30          0          8          0      10744   ip_frag.o
       464         84          0         12          0      22873   lwip_timers.o
      1044        114          0         12        124       9599   main.o
       552         30          0         12      10260       5817   mem.o
       144         20         40          0      18475       5614   memp.o
       308         18          0         12          0      10225   netif.o
       964          0          0          0          0      11027   pbuf.o
       116         12          0          4          0       1936   raw.o
        36          8        392          0       2048        860   startup_stm32f407xx.o
        60          8          0          0          0       2824   stm324xg_eval.o
       306          6          0          1          0       3738   stm324xg_eval_eeprom.o
       142         20          0          4          0       5992   stm32f4xx_hal.o
       194         14          0          0          0      30971   stm32f4xx_hal_cortex.o
      2272         72          0          0          0      13594   stm32f4xx_hal_eth.o
       532         60          0          0         32       6937   stm32f4xx_hal_flash.o
       364         22          0          0          0       4454   stm32f4xx_hal_flash_ex.o
       494         56          0          0          0       4895   stm32f4xx_hal_gpio.o
      1456         34          0          0          0      13045   stm32f4xx_hal_i2c.o
      1272         60         16          0          0       5908   stm32f4xx_hal_rcc.o
        24          0          0          0          0       4082   stm32f4xx_it.o
        84         18          0         20          0     394769   system_stm32f4xx.o
      2334         96        201         36          0      34698   tcp.o
      3114        126          0         28         20      31618   tcp_in.o
      2514         10          0          0          0      17387   tcp_out.o
       712         16          0          8          0      14953   udp.o

    ----------------------------------------------------------------------
     28798       1416       3086        224      43680     787691   Object Totals
         0          0         32          0          0          0   (incl. Generated)
        56          0          8          6          1          0   (incl. Padding)

    ----------------------------------------------------------------------

      Code (inc. data)   RO Data    RW Data    ZI Data      Debug   Library Member Name

         0          0          0          0          0          0   entry.o
         0          0          0          0          0          0   entry10a.o
         0          0          0          0          0          0   entry11a.o
         8          4          0          0          0          0   entry2.o
         4          0          0          0          0          0   entry5.o
         0          0          0          0          0          0   entry7b.o
         0          0          0          0          0          0   entry8b.o
         8          4          0          0          0          0   entry9a.o
        30          0          0          0          0          0   handlers.o
        36          8          0          0          0         68   init.o
        26          0          0          0          0         80   memcmp.o
        36          0          0          0          0         68   memcpya.o
        36          0          0          0          0        108   memseta.o
       264          6          0          0          0        244   printf2.o
        28          0          0          0          0         76   strcmp.o
        30          0          0          0          0         80   strncmp.o

    ----------------------------------------------------------------------
       508         22          0          0          0        724   Library Totals
         2          0          0          0          0          0   (incl. Padding)

    ----------------------------------------------------------------------

      Code (inc. data)   RO Data    RW Data    ZI Data      Debug   Library Name

       506         22          0          0          0        724   mc_w.l

    ----------------------------------------------------------------------
       508         22          0          0          0        724   Library Totals

    ----------------------------------------------------------------------

==============================================================================


      Code (inc. data)   RO Data    RW Data    ZI Data      Debug   

     29306       1438       3086        224      43680     763407   Grand Totals
     29306       1438       3086        224      43680     763407   ELF Image Totals
     29306       1438       3086        224          0          0   ROM Totals

==============================================================================

    Total RO  Size (Code + RO Data)                32392 (  31.63kB)
    Total RW  Size (RW Data + ZI Data)             43904 (  42.88kB)
    Total ROM Size (Code + RO Data + RW Data)      32616 (  31.85kB)

==============================================================================

